:020000040000FA
:1000000092EF01F01200FFFF10EF04F01200FFFF6B
:1000100000000901C80E526F62806250010B06E0B9
:100020000901525103E009015207F7D712000000FD
:100030000901C80E526F62846250040B06E0090188
:10004000525103E009015207F7D71200D9CFE6FF5A
:10005000E1CFD9FF3F0E6416636A626AFE0EDB5081
:100060006312FD0EDB506412638AE552E7CFD9FFBD
:100070001200D9CFE6FFE1CFD9FFFE0EDB50666E4E
:1000800063AE02D0FF0E30D00F0E631408080CE0F0
:100090000F0E63140B0808E06450040B03E1645076
:1000A000010B1FE0000E20D00F0E6314080804E0BF
:1000B0000F0E63140B0818E10901C80E526F64504B
:1000C000010B04E0525102E05207F9D76450040BCF
:1000D00001E0010E4A6E1F0E62144A10F7E162AC95
:1000E00002D0FE0E01D0000EE552E7CFD9FF12007C
:1000F000D9CFE6FFE1CFD9FF0000FE0EDBCFE6FF50
:10010000B8DFE552006E005003E091DF005000D0F0
:10011000E552E7CFD9FF120000007ADF700EE66EDD
:10012000E7DFE552000901E028D0800EE66EE0DF4F
:10013000E552000901E021D0E66ADADFE552000964
:1001400001E01BD0400EE66ED3DFE552000901E06E
:1001500014D0016A1E0E015C0FE20150EA6A000F22
:10016000E96E060EEA22EF50E66EC2DFE5520009A4
:1001700001E003D0012AEED75ADF12000000016A25
:100180001E0E015C09E20150EA6A000FE96E060EDC
:10019000EA22EF68012AF4D712000000016A1E0E5D
:1001A000015C09E20150EA6A000FE96E060EEA22DC
:1001B000EF6A012AF4D712000000EFDFE66A080EAA
:1001C000E66E44DFE552E552090E656E21DF700EE2
:1001D000E66E8EDFE552000901E01CD0800EE66E6F
:1001E00087DFE552000901E015D0C80EE66E80DF1A
:1001F000E552000901E00ED0E66A7ADFE552000917
:1002000001E008D0E00EE66E73DFE552000901E080
:1002100001D00DDF12000000CFDF06010F6B0601D9
:10022000106B06019C0E116F0601100E126F060175
:10023000136B0601150E146F0601156B0601166B84
:100240000601090E176F0601010E186F0601500E08
:10025000196F0601810E1A6F06015D0E1B6F0601F4
:10026000040E1C6F0601500E1D6F56DF12000000B9
:10027000810EC96E37D8FC0EC96E34D88E8E000040
:100280000000000000008E9E120009014E6B090163
:100290004A07000E4B5B09014D5109014C5D01E01D
:1002A000C96A4E2FFED709014D5109014C5D02E08C
:1002B0004CC9C9FF4E2FFED78E8E8E8E8E9E4CC996
:1002C0004DF9120000000900F5CF49F90900F5CFFA
:1002D00048F9090148510901462709014951090115
:1002E0004723120000000901486B496B0901540EB5
:1002F000485D3D0E495905E20901482B000E49238E
:10030000F5D712000000210EC26EC09EC28200000E
:10031000C2B2FED7C4504D0802E2010E02D0000E58
:1003200000D01200C16A210EC26E896A300E8A6E38
:10033000030E8B6E100E8C6E320E8D6E040E8E6E52
:100340008F6A830E906E916A92680F0E936E900E74
:10035000946E600E956E9D0E966E7B0E976E070ED8
:10036000986E300E996E9A688D8CC79EC698C78C11
:10037000F00EC616C680C68A240EAC6E190EAF6E7D
:10038000900EAB6E19DFC8DE72DF0901516BBADF68
:10039000000904E10A0E0901515D09E2640E090138
:1003A000515D05E29FDF9EDF0901512BF0D7090166
:1003B0005151630802E2FDEF01F00901466B476B02
:1003C000F66A080EF76EF86A7DDF000009014851F1
:1003D000491102E102EF04F075DF800EF61805E125
:1003E000FD0EF71802E1010EF81801E0F5D709013A
:1003F0004651471102E102EF04F001D8120000005B
:100400000ADF09014C6B09014BA703D00901010E5A
:100410004C6F3BDF9EAA29D0ABA209D0AB9800005D
:1004200000000000000000000000AB881ED0AECF2E
:100430004FF9ACA2FED7490E09014F5D0BE14B0EFF
:10044000AD6EACA2FED7330EAD6EACA2FED7420E9F
:10045000AD6E06D0FF0E09014F5D02E04FC9ADFF42
:10046000440E09014F5D01E101D0CBD709014A6B70
:100470004B6B0901020E4C6F09014AA902D0090118
:100480004C6B03DF2FD8020EF85C05E1420EAD6E17
:10049000F86A0ED8FF000CD8410EAD6EEAD71200F4
:1004A0000000550EA76EAA0EA76EA68200001200CD
:1004B000940EA66EF5DF000EE96E090EEA6E0A00D4
:1004C0000901080E446F0901080E456FEE50F56EE4
:1004D0000F00452FFBD7840EA66EE2DF442FF3D723
:1004E000A694120000000901506B0901446B440EF0
:1004F0000901445D1FE29EAAFED7ABA209D0AB98CA
:10050000000000000000000000000000AB8802D0E6
:10051000AECF4FF909014451EA6A000FE96E090EA6
:10052000EA224FC9EFFF09014F5109015027090184
:10053000442BDDD7090150510BE1030E0901425D47
:1005400007E240C9F6FF41C9F7FF42C9F8FF03D0EF
:100550004E0EAD6EC8D71200FFFFFFFFFFFFFFFF7B
:10056000FFFFFFFFFFFFFFFFFFFFFFFFFFFFFFFF9B
:10057000FFFFFFFFFFFFFFFFFFFFFFFFFFFFFFFF8B
:10058000FFFFFFFFFFFFFFFFFFFFFFFFFFFFFFFF7B
:10059000FFFFFFFFFFFFFFFFFFFFFFFFFFFFFFFF6B
:1008000000001200280EE66EAEECFDF0E55262EF3D
:10081000FDF01200FFFFFFFFFFFFFFFFFFFFFFFFE5
:10082000FBEF2AF01200FFFFFFFFFFFFFFFFFFFFBC
:100830000000FAECE4F04C0E4A6EEF0E4B6E010E27
:1008400099EFEFF0FAECE4F0BF0E4A6EEF0E4B6E4C
:10085000010E99EFEFF0FAECE4F09A0E4C6EF00E08
:100860004D6E010E4E6EFE0EDBCF4FF0506A516A98
:10087000D8904F36503651364C504F24F36E4D5071
:100880005020F46E4E505120FAECEFF00900F5CFF5
:100890004AF00800F5CF4BF01AECF3F0FFEFE4F06C
:1008A00065ECEFF0010EE66EFD0EDB500301A725AF
:1008B0004A6EFE0EDB50A821000127ECF4F01AEC82
:1008C000EEF014ECEDF0DF50E552FFEFE4F08DECCC
:1008D000EFF04B6A020F4A6E010EB7ECEFF0FFEF3C
:1008E000E4F0FAECE4F0EF0E4A6EEE0E4B6E010E01
:1008F00099EFEFF08DECEFF001ECF2F0FD0EDB5034
:10090000E0ECE5F0EF50FFEFE4F02FC1E6FFA3DFEE
:10091000E5521200100E8AEFEBF0FAECE4F00F0E45
:100920004A6EEB0E4B6E010E99EFEFF069503FEC03
:10093000F4F0D7ECEFF0006E1200D9EFE9F00A0EF8
:100940004A6E4B6AC5EFF4F0FBECEEF0C5EFF4F045
:10095000E80E4A6E030E4B6EC5EFF4F0FBECEEF0C2
:100960004AC23EF04BC23FF0B0ECE5F03E50006EA4
:10097000120001012B51010B1CE07851200B19E0F2
:10098000E251010B16E0CA51080B13E0100E2C5D6A
:1009900010E22C5105080DE23C51100B0BE011EC5C
:1009A000E9F008E0100E0101615D03E26151050804
:1009B00001E3000C010C17ECEBF00EE00201BB515F
:1009C000100B0AE03450400B08E00101D751010B35
:1009D00003E011ECE9F001E1000C010CE66A6FECB8
:1009E0002EF0E5521200300EE66EED0EE66E010EB0
:1009F00090ECEBF0E5521200010E27EFE5F0020E4D
:100A000027EFE5F0B2C2E6FFE50E0FEFE5F0E66A8C
:100A1000E50E0FEFE5F07EEC14F0000918E07EEC37
:100A200014F0000914E0960E85ECE5F06CEC0FF084
:100A30002BB00DD07EEC14F0000909E07EEC14F030
:100A4000000905E0DB0E98ECE5F083EC0FF01200F6
:100A50000101E151010B03E05751080B02E1000EC7
:100A600001D0010E000903E00201B9511200020198
:100A7000B5511200FAECE4F00101E151010B07E07D
:100A80005751080B04E0FE0EDBCFB9F203D0FE0E87
:100A9000DBCFB5F2FFEFE4F002011881178B17816D
:100AA0000501BF0E3B6F12000301D2510201EF5D41
:100AB0000301D3510201F05913E3EF510301D45D57
:100AC0000201F0510301D5590BE3D2510201ED5D52
:100AD0000301D3510201EE5903E37DECECF008E28F
:100AE000D2C3EFF2D3C3F0F2D2C3EDF2D3C3EEF22E
:100AF000120089ECEFF0FF0805E117ECE5F0090EB4
:100B0000D3ECE8F01FECF3F04A6E0A0E4A5C0BE3FC
:100B100017ECE5F00F0EEF140009BEECF3F0090E30
:100B20002DECF0F0EF8E12007DECE7F003E1040E07
:100B3000495D12004951120096ECEBF013941396A4
:100B4000198C04908EEC55F001018F51400B09E196
:100B50004A51320806E2320E4A6FE9EC7FF0020198
:100B600017870C500EE101018FAD09D09BECEBF023
:100B70000A01D76BE66A08EC91F0E5521200B3EC7B
:100B80004BF01200800E081406E02150010B03E127
:100B90000201315101E0000C010C800E081403E049
:100BA0002150010B01E0000C010C0C500AE1010185
:100BB0008F51400B06E03550400B03E12150800B74
:100BC00001E0000C010C0201010E4D6FE20E98ECE9
:100BD000E5F01E0E096E12001BEFEDF08DECEFF04C
:100BE00004080FE017ECE6F00EE0FE0EDB500A08FA
:100BF00008E0FE0EDB500D0804E0FE0EDB50090895
:100C000002E1010E01D0000EFFEFE4F00701C7077B
:100C1000C551C52BEA6A000FE96E0C0EEA22EF50AF
:100C200012000101E051100B03E00401BA510AE186
:100C3000420EE66E460EE66E6EECCCF0E552E552E4
:100C40000101E0891200D9CFE6FFE1CFD9FFFE0E06
:100C5000DB50D80805E1300EF36EFE0EF3CFDBFF5C
:100C6000060EAB1406E0AB98000000000000AB8855
:100C70008ED1FE0EDB50100805E0FE0EDB50110891
:100C800001E02AD10201050E296FFE0EDB5011088A
:100C900037E1020134510DE12150800B0AE10501D9
:100CA00005013B51010B0AE1050105013B51400BD8
:100CB00005E1100EE66E85D9E55222D00501050149
:100CC0003B51400B02E00F0E01D0060EE66E79D9C3
:100CD000E552BFC1E6FF75D9E552C0C1E6FF71D943
:100CE000E552C1C1E6FF6DD9E5520A0E0101C2030A
:100CF000F3500101C325E66E64D9E55205013B912D
:100D00000401B0514A6E4B6AD8904B5004E6D30EA2
:100D10004A5C000E4B5801E3DED005013B5101E176
:100D2000DAD00201345101E0D6D02150800B01E02D
:100D3000D2D0049005013BA11AD001010101E0517C
:100D4000080B03E00401BA510DE1410EE66E460EB8
:100D5000E66E6EECCCF0E552E5520101E08705014C
:100D60003BB35FDF05013B9305013B91B4D0050127
:100D70003BA304D056DF05013B93ADD005013BA753
:100D800024D0440EE66E4D0EE66E6EECCCF0E552CD
:100D9000E5520480440EE66E4D0EE66E6EECCCF02D
:100DA000E552E552030E0C5C03E0030E7D5C08E1A6
:100DB000540EE66E440EE66E6EECCCF0E552E55253
:100DC00005013B9705013B8586D005013BA524D055
:100DD000570EE66E420EE66E6EECCCF0E552E55232
:100DE0000480570EE66E420EE66E6EECCCF0E552D5
:100DF000E552530EE66E490EE66E6EECCCF0E5520F
:100E0000E552490EE66E460EE66E6EECCCF0E5520B
:100E1000E55205013B955FD005013BA90BD0410E82
:100E2000E66E500EE66E6EECCCF0E552E552050132
:100E30003B9951D005013BAB0BD0410EE66E520EF3
:100E4000E66E6EECCCF0E552E55205013B9B43D0DB
:100E500005013BAD13D04F0EE66E520EE66E6EEC02
:100E6000CCF0E552E552540EE66E520EE66E6EEC94
:100E7000CCF0E552E55205013B9D2DD005013BAF7D
:100E80002AD04E0EE66E4C0EE66E6EECCCF0E552BD
:100E9000E552560EE66E440EE66E6EECCCF0E55270
:100EA000E552420EE66E530EE66E6EECCCF0E55265
:100EB000E552570EE66E430EE66E6EECCCF0E55250
:100EC000E5524E0EE66E420EE66E6EECCCF0E5524A
:100ED000E55205013B9F5BD0200EF36EFE0EDBCF8B
:100EE000F4FFF350F45C04E3FE0EDB507E0807E2EF
:100EF000FE0EDBCFE6FF72DEE552000948E0FE0E93
:100F0000DB503B0804E0FE0EDB507C0802E10401EC
:100F1000B92B01010101E351800B0BE0FE0EDB5008
:100F20003B0807E17EC1E6FFBAEC0EF0E552010195
:100F3000E39FFE0EDB50210804E0FE0EDB5040086C
:100F40000AE13B0E0401BE5D04E07C0E0401BE5DBF
:100F500002E10401B92BFE0EDBCFBEF40401B15156
:100F6000EA6A000FE96E0B0EEA22FE0EDBCFEFFFFE
:100F70000401B12B0401B02B0401B05108E10401BC
:100F8000BE6BBEC4B9F4BEC4B1F4BEC4B2F4E55283
:100F9000E7CFD9FF1200ACA212000401B8510EEC49
:100FA000F0F0006E0050E66E1DECFDF0E5523B0ED9
:100FB000005C03E07C0E005C01E12A900401B82B88
:100FC0001200FAECE4F0ACA2FED794ECE5F01DECD4
:100FD000FDF0E552FFEFE4F089EC13F095EC13F02F
:100FE000F29EF66A080EF76EF86A940EA66E550E1B
:100FF000A76EAA0EA76EA682000000EC00F01200F9
:101000000401B007B251B3ECE8F0EF50006EB22B20
:101010001200050E0C5C0AE12050020B07E10201F0
:10102000B451020B04E1B451010B01E1000C010CBD
:10103000040E0C5C04E10101CD51080B01E1000C30
:10104000010CC70E70ECF4F0320803E33050400B93
:1010500009E0309C89EC13F095EC13F079ECB5F0D5
:10106000DAEC13F0120069ECEFF09C0EDE6E030E6A
:10107000DD6E0301A551A61127E0090EE66EFD0EF7
:10108000DB50090DF350A5254A6EF450A62127EC3C
:10109000F4F09C0EE66E030EE66E14ECEDF0DFCF7E
:1010A000E9FFDF2A010EDBCFEAFF01E3DB2AEFCF06
:1010B00000F0EF5024E0FE0EDB5003E10EEC97F061
:1010C000EED737EC97F0EBD7FE0EDB500BE1A2EC3E
:1010D00093F0E60EE66EF20EE66E010EE66E25EC7D
:1010E00097F00AD0AEEC93F0DE0EE66EF20EE66EEE
:1010F000010EE66E4AEC97F0E552E552E552020E1B
:10110000E15C02E2E16AE552E16EFFEFE4F0049097
:1011100074ECF4F038E004800101DEAB34D017EC5D
:10112000E5F00492EF50010B01E0048223ECF3F0B0
:10113000016E050EEB50026EEF50080B01E0010E40
:101140006AECF2F0FE0EEF14F310BEECF3F0070EB3
:10115000EB50E66E040E8FECF4F0080EEB50E66EEA
:10116000050E8FECF4F00450020B02E0EF8601D084
:10117000EF9617ECE5F0070E01C0EBFF17ECE5F07A
:10118000080E02C0EBFF12000501005102012A11F6
:101190003D1107E11C50010B03E14A514B1101E1E4
:1011A000000C010CFAECE4F00101DE9D0701108552
:1011B0006DEC5EF094ECE5F035EC29F0E5520701BA
:1011C00010956DEC5EF0080E85ECE5F0FFEFE4F0B5
:1011D00000000000000000008C98000000000000EB
:1011E0000000120000000000000000008C880000D9
:1011F000000000000000120052EC29F002016A6BAE
:101200006AC22AF23D6B4A514B1102E021949CD9EB
:1012100050EF80F00701EF51010B07E0030E0C5C6B
:1012200004E0050E0C5C01E0000C010C0101279D9F
:10123000010E0E6E27BF0E681200030E27ECE5F0BC
:10124000268E12004D0E12EFE5F04E0E12EFE5F075
:1012500001018F51010B08E0C8EC11F0000904E016
:1012600001013C51800B01E0000C010C040E27EC45
:10127000E5F03C0E096E1200268E050E27EFE5F014
:10128000FEECF1F0FEECF1F000010F6EFEECF1F07F
:10129000106E120078ECF4F088C1E6FFDD0E0FEC62
:1012A000E5F094C100F0FFECEEF005E1090E01015C
:1012B0009603F350006E0050E66EDE0E0FECE5F084
:1012C00078EFEFF0FAECE4F0490EB6ECF1F00F50E5
:1012D00010100BE0FE0EDB50EA6A900FE96E010E73
:1012E000EA220FC0EEFF10C0EDFFFFEFE4F025A8EB
:1012F00006D0010E696E020EE66EE4DFE552696A01
:10130000E66AE0DFE5521200FAECE4F0FE0EDB5094
:10131000D4ECE5F0EF5010E1FE0EDBCF4AF0FD0E0D
:10132000DB50D8804A5408E3FE0E1FECEEF0D4ECFC
:10133000E5F0100EEF6EEAD7FFEFE4F0830E0A6ED1
:10134000FA0EBDECE5F000500F6E0FC010F00F6A02
:10135000FB0E7CECF4F00050BAEFF1F00101CB5140
:10136000800B01E0010EA1ECEBF03BC1EFFF12009E
:101370000101CB51800B01E0010EA1ECEBF0EFCFAE
:101380003BF13B51140804E2010E3B6F2CA63B6B72
:1013900008EFC5F0FAECE4F0E2ECECF002E1EBC7A8
:1013A000EAF7FE0EDB0402E1EAC7EBF7FFEFE4F039
:1013B000695003E03450400B02E00C5012007D50A5
:1013C00012000C50FDECE5F085EFECF043C1E1F2CA
:1013D00043C1E0F20C504CECF2F0400B03E0020190
:1013E000040EE06F7D504CECF2F0400B03E0020184
:1013F000040EE16F120065ECEFF02950010B29E1BA
:101400002A0E675C06E10850A5ECEAF001E14B50BA
:1014100020E00C0E675C0AE108504C6E4D6A810EAC
:101420004C1804E14D5002E16F5013E08FECB5F021
:10143000000909E01A50400B06E11850080B03E1BF
:101440002150100B06E0190E675C05E15BECE8F03B
:1014500002E1000E01D0010EDF6E2D50800B03E182
:101460002D50400B02E0010EDF6E2990DF50E55257
:10147000FFEFE4F01B9C248A1200010137AF05D076
:1014800004A002D01B8812001B8A120078ECF4F032
:10149000580E12ECE5F01DBE02D001ECECF078EF36
:1014A000EFF0010137AF07D0060E3BECF1F0280E4C
:1014B00085ECE5F0EBDF12000601980ED880B455FC
:1014C0003A0EB55509E20F50B45D0101D26F1050CC
:1014D0000601B559010108D0B4510F240101D26FA2
:1014E0000601B55110200101D36F12000101DFBFC9
:1014F00011D0160E1CECE9F0050E436E446A4AC288
:101500003EF04BC23FF078ECFDF03EC04AF23FC0E7
:101510004BF21200110E1CECE9F0020E0F0B02014F
:1015200005E0D8904B334A33E806FBE112001AB4C9
:1015300004D0370EC1ECF3F0000C010C970E28EC30
:10154000F3F0980E2BEFE5F00101E0931C921C9054
:101550001A9A149220EC1EF002014A6B4B6B54DB7A
:101560009EEF0AF069ECEFF0580EDE6E050EDD6EB0
:10157000560E0F6E010E106E0101DFAF07D0A80EE0
:10158000DE6E030EDD6EEA0E0F6E106A0D044A6EFB
:101590004B6A19ECF4F0C5ECEFF0CBECF8F03CC082
:1015A000D2F13DC0D3F101018BA706D009ECE6F0E2
:1015B000EE50D227EE50D323020EE15C02E2E16A44
:1015C000E552E16EFFEFE4F0320E85ECE5F09F0EA0
:1015D00009EFF2F0FAECE4F0F7DF2250800B08E0BC
:1015E000350E675C05E10F681068410E27ECE5F0E9
:1015F000049001018BB70480C4EC8EF000C70AF0A0
:10160000FC0E016E10C000F0FFEC4CF0012A0FC080
:1016100000F0FFEC4CF00A6AFFEFE4F065ECEFF04D
:10162000010EDF6E21AC06D0030EDF6E0101E083F8
:1016300020EC1EF0800E80ECF4F0980E2BECE5F020
:10164000D6C30FF0D7C310F0950E8CECF0F0E55236
:10165000FFEFE4F0550E12ECE5F01A801200540E84
:1016600012ECE5F01A90120065ECEFF0FCEC26F0BD
:10167000DF6E1BECEBF007E01AA00ED0F0DFDF50BE
:101680000BE1006A07D01AB007D0E4DFDF5004E1B5
:10169000010E006E36EC91F0E552FFEFE4F001012F
:1016A00060B702D02CC161F157ECE7F024EFEEF007
:1016B000D5ECEAF005E02050020B02E189ECE6F0FF
:1016C0001200F4ECE8F009E02150800B06E13C51F7
:1016D000100B03E02050080B01E1000C010CD5ECCD
:1016E000EAF00EE02150800B0BE12050080B08E0DF
:1016F0003C51200B05E12E50400B02E1095001E066
:10170000000C010CB4ECE5F003E03550400B04E0B4
:1017100001015851040B01E1000C010C65ECEFF0E4
:1017200001018BA10AD0FCEC26F0DF6EDF0403E0A0
:10173000020EDF5C02E1010E01D0000EE552FFEF68
:10174000E4F007ECEFF005E1FCEC26F0040801E022
:10175000000C010CF6DF000904E10BECEFF001E0F6
:10176000000C010C8150080B0DE08150010B0AE0C8
:10177000B4ECE5F003E0E6ECECF004E11A50020B07
:1017800001E1000C010C8150080B19E08150020BA3
:1017900016E08150040B13E08150010B10E00501AD
:1017A00000510DE12150040B0AE12150010B07E12A
:1017B000B4ECE5F003E0E6ECECF001E1000C010C28
:1017C000810E15ECE9F0010137BF268E120010C220
:1017D000E6FF0FC2E6FFC80E2BEFE5F01E9C076A7E
:1017E000796A33DDEA0E15ECE9F0268E12008DECF5
:1017F000EFF00A0DF3CF5AF3F4CF5BF3000E0301C1
:101800005A27030E5B23FFEFE4F00F0E07010E13C0
:101810000E990E9F040E0101445D02E107010E8F37
:10182000100E01012C5D14E2020E815D25E22C51A7
:1018300002E107010E9101012C0502E107010E935F
:1018400001012C51020818E22C1D07010E1714D0BB
:10185000815112E0100E2C5D3DECE8F08BC200F0DF
:101860000A0E005C01E1006A001C07010E17DDECA6
:10187000F4F0020B01E10E89049007010EB7048019
:101880000E970EB30E870E9304B00E831200F3EC86
:10189000F0F004E68A0E4A5C000E4B5802E2E0EFDC
:1018A0000BF0F3ECF0F004E6A90E4A5C000E4B5886
:1018B00004E20201E051795E1200F3ECF0F002E67E
:1018C00028ECEEF003E20201E05179261200140E3A
:1018D0005CECE7F0D4ECEFF000501C0806E3145089
:1018E000100B04E000500C0801E2010C000CF4ECB9
:1018F000E8F003E1D951100B07E18B51400B03E0F5
:10190000D951040B01E1000C010C11ECE9F002E0EB
:10191000060E01D0070E27EFE5F069CFC7F2696A1E
:1019200079C101F07AC102F0D9ECEAF004E20701D2
:101930000551026E016E01900142029002424D0E6D
:10194000012471ECF2F0010E696E4D0E022471EC6F
:10195000F2F0C7C269FF120007010E9B0101CCAB78
:1019600002D007010E8B12A007D007010E9B0101C8
:10197000CCAD02D007010E8B1200695006E0345046
:10198000400B03E10201B15112000101E2A903D0B1
:101990000201B05112000A01D55112000201630E7A
:1019A000C36F010EC46F695004E05D0EC36F010E7A
:1019B000C46F1200BEECF1F00FC1DFFF010E10C1C9
:1019C000DBFF34AC05D0DB50DF6E010E0FC1DBFF57
:1019D00064ECE6F0F4ECE8F037E107011051200B7D
:1019E00033E01051010B07E0DF500A0804E2010E5A
:1019F000DB500A0829E3010EDB50DF5C25E00A0E0C
:101A0000DF5C22E0DF50070804E20A0E36ECE5F066
:101A10001BE3DF50050804E2080E36ECE5F014E3A2
:101A2000DF50030804E2060E36ECE5F00DE3DF506C
:101A3000010804E2040E36ECE5F006E3DF0406E1FB
:101A4000020E36ECE5F002E2020EDB6A020EDB501B
:101A500007E0080E27ECE5F0FA0E096E19861C88DF
:101A6000030EE15C02E2E16AE552E16EFFEFE4F0B1
:101A70000701079711ECE9F006E074ECE9F003E0E8
:101A80000701078797DF1FEFEBF0FAECE4F02BA4D8
:101A900009D0F1ECEAF065EC2EF0FCECF3F0500E1E
:101AA000096E2B94FFEFE4F0159E0A01DA51800BCA
:101AB00006E1050E0C5C03E0A8ECE6F001E0158EF3
:101AC00012000C50080D61ECE7F0010E0FECEFF086
:101AD000E806FCE10250080D4C50F3244A6E4D50CC
:101AE000F4204A50016E12000A01DA8FDDDF020194
:101AF0009651F6ECE5F01AE24A509608000E4B5467
:101B000015E20268950501E1026A030E955D02E1A6
:101B1000010E026EFF0E025C10E021ECEDF0C3EC52
:101B2000F1F0015056ECF0F00A6A07D088ECE9F0C9
:101B300069ECECF0178B05013B850201956B188E63
:101B4000500E096E2596328C12000201C669C6C27B
:101B5000C5F2C6C2BCF7C6C2BBF7C6C2BAF7C6C298
:101B6000B9F7C6C2B8F7C6C2B7F70701C369C469F7
:101B7000C169C269C1C7BFF7C2C7C0F7C1C7BDF756
:101B8000C2C7BEF712000101470503E18450100BE4
:101B900007E0020E475D03E18450100B01E1000CE9
:101BA000010C96880101475101E19698120065ECFD
:101BB000EFF00101A45103E19A51200821E2DF6A0C
:101BC000090EDF5C10E2DF502FECE6F0EF50040B63
:101BD00008E0100EDF24E66E08EC35F0E55200094F
:101BE00002E1DF2AEDD7090EDF5C0AE2100EDF26E4
:101BF0002A86DFCFE6FFC7EC34F0E552DF5001D094
:101C0000000EE552FFEFE4F02086076A796A189823
:101C1000189A2682248A1200010138BB02D09092C1
:101C200001D09090000000000050E66E12EC7AF0B7
:101C3000E5520000C950006E000090809082030EB3
:101C4000E66ECAECFDF0E55212002C880701108107
:101C5000108D10990101E0A502D00701108907013C
:101C6000129712002C9807011091109D109912875D
:101C700012001FEC7AF0F00EC616C680C68A12005B
:101C8000800EE66EE66A010EE66E54ECFBF0FCECAC
:101C9000F3F039EF0EF0138213800601109F02015A
:101CA0001E0E406F1200139020A21380139220B2D8
:101CB000138212004EECF4F04CECF2F013ECEFF067
:101CC000DF6E000EDF94DF96DF98DF9ADF9CDF9EE9
:101CD0000A0E006EFE0EDB5009E1030EDF5C02E22D
:101CE000050E006EDF5043E1010E40D0FE0EDB50CA
:101CF000030804E1DF5002E1010E006EFE0EDB502E
:101D000004080EE1DF0402E1320E006E020EDF5C19
:101D100002E15A0E006E030EDF5C02E1640E006EFB
:101D2000FE0EDB50050810E1320E006EDF0402E10A
:101D3000640E006E020EDF5C02E17D0E006E030E8B
:101D4000DF5C02E1FA0E006EFE0EDB0403E0E2EC63
:101D5000ECF00DE1DF5002E1010E006EDF0402E164
:101D6000050E006E030EDF5C02E1190E006EE552F7
:101D7000FFEFE4F0FAECE4F0F00E07010F17FE0EAF
:101D8000DB50320FB8ECE5F007010F1396EC5EF074
:101D9000FFEFE4F0695010ECF2F0D7ECEFF0050D36
:101DA000F350006E8EECE8F0EF50200B02E0050ED1
:101DB00000260701BB51005C07E000C0BBF70050E4
:101DC000E66EAE0E0FECE5F01200139A20B2138A05
:101DD0006ADFB3EC4BF0E5EC1CF02050020B05E0A1
:101DE0007D500C5C02E01B8C12001BAC02D03AEC64
:101DF0000AF01200FAECE4F02050020B06E026ECA8
:101E0000B9F0000902E120922ED02050020B08E028
:101E1000A8ECE6F005E0B7ECB8F0BFECB8F0208233
:101E20002050020B06E0F4ECE8F003E0139E3C9334
:101E3000CA99FE0EDB5004E120B204803DEC0AF0AA
:101E4000C4DF050E0C5C08E12050020B05E0020126
:101E5000B493B4916AEC38F0C8ECB8F0FE0EDB50E5
:101E600002E102011783FFEFE4F065ECEFF0CFC170
:101E7000DFFF7DECE7F002E1040EDF2682ECE6F006
:101E800003E00D0EDF5C11E382ECE6F00CE17DEC8B
:101E9000E7F003E0140ECF5D08E30A0E2C5D03E1CA
:101EA0000A0ECF5D02E3000E01D0010EE552FFEFF6
:101EB000E4F00A6A700EE66E290EE66E010EE66E1A
:101EC000E66A5AEFE5F07E0E0A6E0F0EE66EED0E34
:101ED000E66E020E76EFF1F0F00E8C162EECF4F0BA
:101EE00011E282ECE6F00EE02B50010B0BE1320E1A
:101EF00085ECE5F02EECF4F005E22B807B0E9CECFB
:101F0000E5F001D812000101320E496FD7ECE8F07C
:101F10007FEF28F00701875106E14C0E66ECE7F0F1
:101F20000501141501E1000C010C2D9E2D9C6AEC9D
:101F300038F0F7EFB5F007011D891D9782ECE6F048
:101F400009E001012C0506E16051400B03E10701A6
:101F50001D991D871200FAECE4F02BECEEF007E17E
:101F60002C50010B04E101018B51200B09E155C2FA
:101F700058F254C257F253C256F228ECEDF009D091
:101F8000FE0EDB5006E058C255F257C254F256C25C
:101F900053F2198C04802CA002D004902C908EEC6B
:101FA00055F0320E096EFFEFE4F0006A01013A517C
:101FB000060802E2DDC700F000AE02D007011CD027
:101FC0002BA002D007013ED00701DF5106E10050EF
:101FD000240825E3E05140E022D0DF050FE1005066
:101FE000290803E3E051010802E2020EDF6F230E2D
:101FF000005C32E2E05130E1DF6B2ED0020EDF5D9B
:1020000010E10050310803E3E051020802E2030E40
:10201000DF6F280E005C20E2020EE05D1DE2010E83
:102020001AD0030EDF5D10E10050360803E3E051E3
:10203000030802E2040EDF6F300E005C0DE2030EB7
:10204000E05D0AE2020E07D0350E005C05E2040EE8
:10205000E05D02E2030EDF6F070E1315006EF80E4F
:102060001317DF0501E11385020EDF5D01E1138324
:10207000030EDF5D02E113851383040EDF5D01E1D2
:102080001381070E1315005C08E0050E06ECECF05A
:102090002D907BEC5EF0F00E8C161200FAECE4F062
:1020A00021B814D0FE0EDB503EECF1F0016EFE0EB6
:1020B000DB50040F3EECF1F0026EFF0E015C08E114
:1020C000FF0E025C05E1199A17B8198A000E09D0B3
:1020D0000150006E17A802D00250006E02EC9BF077
:1020E000010EFFEFE4F00301916B926B936B946B25
:1020F00091C38DF392C38EF393C38FF394C390F384
:10210000030E016EFF0E015C32E0056A030E026EE3
:10211000FF0E025C22E00250EA6A890FE96E030EAC
:10212000EA22EF504C6E4D6A0150EA6A850FE96E63
:10213000030EEA22EF501BECE6F035ECEBF0EF502B
:10214000BAECF1F00550BAECF1F035ECEBF00FC061
:10215000EFFF10C005F00206DBD70150EA6A8D0FD1
:10216000E96E030EEA2205C0EFFF0106CBD712008D
:1021700000AE04D0006C01010E0E146F8EECE9F07D
:10218000010115510AE114C115F1100E146F165119
:1021900004E115C116F1100E156F130E186F120021
:1021A000BEECF1F06950A7ECEBF0EFCFDFFF010ED2
:1021B000BFC1DBFF020EC0C1DBFF010178B738D021
:1021C000695006E0010EC4C1DBFF020EC5C1DBFF92
:1021D000DFCFE6FF19EC04F0E552E66E5EECEAF0C4
:1021E0000EECE6F00B0EDF24B8ECE5F0E66E69507D
:1021F000EA6AE60FE96E020EEA220EECE6F0DF5024
:1022000011E165ECEAF0010EEF6EDB0404E1500E23
:1022100095ECE8F007E25EECEAF0020EEF6E65EC9A
:10222000EAF0EF6A5EECEAF0EF50E66E92ECE9F06D
:10223000030EE15C02E2E16AE552E16EFFEFE4F0D9
:1022400069ECEFF0BFC1DFFF010EC0C1DBFF010190
:1022500078B71ED0695005E0C4C1DFFF010EC5C1CB
:10226000DBFF6950A7ECEBF0EF5012E165ECEAF010
:10227000EF5007E0DF040BE1500E36ECE5F008E22A
:1022800006D0DF0405E1010EDB504F0801E288DFD4
:10229000020EE15C02E2E16AE552E16EFFEFE4F07A
:1022A000030E0C5C03E1030E785C01E0000C010CF2
:1022B000030E0C5C05E1020E785C03E0780401E09B
:1022C000000C010C030E0C5C03E1020E785C01E0D3
:1022D000000C010C030E0C5C08E1785006E10101D2
:1022E000CA51040B01E0020C010C000C030E0C5C43
:1022F0000DE1020E785C04E101013D51010B07E1A3
:10230000780404E101013D51020B01E1000C010CD4
:102310000601F25106E0030E0C5C03E17850000860
:1023200001E3000C010C030E0C5C04E1780403E0F3
:10233000785001E0000C010C030E0C5C06E1020E6B
:10234000785C04E0030E785C01E0000C010C0101F4
:102350003D51080B03E0030E0C5C09E03D51040BFA
:1023600005E00C0404E0020E0C5C01E0000C010C22
:10237000CEEC0CF012ECE6F0EF9C23ECEBF007E077
:1023800012ECE6F0EF8C0701E26B56C1D5FA1200B1
:10239000B4ECE5F003E027ECEBF001E1000C010CFC
:1023A0000C5004E10A01DA51040B01E1000C010CAC
:1023B0000C5003E117ECEFF001E1000C010CEAEC2A
:1023C000ECF00CE0F8ECE8F009E00301D851E1ECA6
:1023D000F4F05DECE9F0E80E2BECE5F0120084EC93
:1023E000F4F00C5005E117ECEFF002E0020EDF6EA6
:1023F000010178B9DF84DFCFE6FFEB0E0FECE5F0EB
:102400000C5004E10A01DAB7DA95D9DFE552FFEFA3
:10241000E4F0030E0C5C11E10101CB51040B05E06B
:1024200078040CE0020E785C09E0CA51040B05E068
:10243000785004E0030E785C01E0000C010C0C50B5
:1024400003E1DDECEAF004E11BECEFF001E1000C4C
:10245000010CC9ECE9F001E0040C78ECE9F001E0D2
:10246000080C040E0C5C01E11B0C0C5009E0030E7F
:102470000C5C05E1785004E0030E785C01E0030C8D
:10248000010CC9ECE9F001E00A0C78ECE9F001E09C
:10249000380C040E0C5C01E1640C0C5001E0500C93
:1024A000380CEFDFE66ED5DFE66ED60EE66E0A0E6E
:1024B00021EFE5F034EC56F0190E01240A01D88022
:1024C000D75503E2190E0124D76FEEECECF0D75D7F
:1024D00003E2EEECECF0D76FD46B348800EFF0F051
:1024E000A8ECE6F00DE1C9ECE9F00AE178ECE9F0DE
:1024F00007E123ECEBF004E15FECE8F001E1000C14
:10250000010C896A700E8A6E030E8B6E100E8C6E33
:10251000320E8D6E040E8E6E8F6A830E906E916AEF
:1025200092688F0E936E900E946E600E956E9D0E57
:10253000966E7B0E976E070E986E300E996E9A68A7
:1025400012002098268A189A02012B5114E00701E4
:10255000EF9BEF9B33BCEF8BE1EC09F002012B6B9F
:10256000F1C600F00C5002E0F3C600F00050E66E39
:10257000E20E0FECE5F02682120095ECF4F030EC60
:10258000EEF0C9ECF4F0C9ECF4F0C9ECF4F0C09E44
:10259000F00E8C16020E0F0B05E0D89010320F32A1
:1025A000E806FBE16BECE7F0030E50ECF2F0FDE126
:1025B0004A500F5E4B50105A2BAA0DD00A0E3E6E99
:1025C0003F6ADBC743F0DCC744F0CBECF8F03C508B
:1025D0000F263D501022AEEC93F0A8EC04F0300F23
:1025E0000101196F36ECE9F001011A6F3A500F6ED4
:1025F000106A9FEC04F0300F01011B6F300E3A247B
:102600001C6F300E195D02E1200E196F1B8F410EF9
:102610001E6F1200FAECE4F005010151EA6A000FA6
:10262000E96E080E2DECF3F0012B015179ECE5F089
:1026300002E635ECEEF001E3016B002BFFEFE4F076
:10264000020E42EFE8F032EFF3F094928B90949008
:10265000B9EFE8F08B9232ECF3F082B0FF0C000C93
:10266000EFDFEEDF82A2FE0C000C0701080EC96F3F
:102670008B9232ECF3F082B207D0F2DF000904E073
:10268000FE0EF36EF46812000701C89FC847C89198
:1026900082B0C881C907EDE1C8513CEFE9F0D9CF5C
:1026A000E6FFE1CFD9FF0701080EC96FFE0EDBCFB1
:1026B000C8F78B9282B206D0D3DF000902E0FF0E8A
:1026C00017D011D0C837D8A006D094929480B8DF24
:1026D0009482B6DF06D094928B909490B1DF94826E
:1026E000AFDF0701C9070701C951E4E1000E00D0BF
:1026F000E552E7CFD9FF12008B9294928B90949081
:10270000B9ECE8F0948020EF13F08B90949020EFD8
:1027100013F09EECE6F059EC0FF020EC5FF063EC68
:102720000FF02AEC5FF052EF9BF0E2EC18F0909C77
:10273000908E31EC2CF00101776B2FEC0BF077ECE5
:1027400009F0020EE66EF50EADECEBF046EC0AF089
:102750000701010E066F076B086B096B0A6B0B6BA9
:102760000C6B0D6BF00E0E170F6B106B116B126B69
:10277000600E136F146B156B166B186B18C717F779
:102780001B6B1C6B206B1D6B1E6B1F6B96EC5EF046
:102790000601526B52C650F6547115EC51F08A98EE
:1027A00067EC98F0D6EC97F00601556B55C654F6D9
:1027B0000B6A1200F29E9D0E966E8D9CFCD7E7EC84
:1027C00026F00701F10504E14C0E005C06E203D09F
:1027D0005A0E005C02E2A9DFEDDF000C46EC0AF0C5
:1027E000E9EC18F03488B3EF4BF08B8A010160B14B
:1027F0008B9AC69A8B96F00E8C1407098C6E93EC0C
:102800005EF08A9AE8EC08F08B8600000000000079
:102810008B960000F2EC08F000008A8AC68A12004B
:102820001A50800B01E0010EA7ECEBF0EF50090805
:1028300001E2000C010CF00E8C16050E8C12C08EFD
:10284000D4ECEFF0C3CF4AF0C4CF4BF029ECE8F062
:1028500029ECE8F0C3CF4CF0C4CF4DF0060ED89071
:102860004D324C32E804FBE14A504C240701DB6F47
:102870004B504D20DC6FC09EF00E8C1612008F0E58
:10288000FAECE5F0030E0002F3CF0CF20050200842
:1028900001E3000C010C0101DD51040B2EE05BECA7
:1028A000E8F02BE02150200B28E03450400B25E1CC
:1028B000E6DF000922E00A0E85ECE5F0E0DF000922
:1028C0001CE0FA0E85ECE5F0DADF000916E0090EEF
:1028D00027ECE5F012AE04D0129E3AECEEF008D0F0
:1028E00012BC06D0128C3FECEEF00201020EBC6F5F
:1028F0003CEC27F04FEC27F0258A1200F00E8C16E6
:10290000070E8C12C08ED4ECEFF0C3CF4CF0C4CFC6
:102910004DF00FECEFF00FECEFF04C50C3244A6E8B
:102920004D50C4204B6E4A50C3240F6E4B50C420F0
:10293000106E110EC8ECF1F0C09EF00E8C16010165
:102940005F514C6E4D6A3B0E4C26010E4D220F50CE
:102950004C5C4A6E10504D584B6E4AC0DDF7070173
:10296000DD5154080BE2DD5179ECE5F002E670EC44
:10297000E7F004E282ECE6F001E0010C000CC08E0E
:10298000870EFAECE5F030ECEEF0D8900F3610360A
:10299000D8900F3610360BECECF0C09ED9C74AF039
:1029A000DAC74BF0030E50ECF2F0FDE14A5007019C
:1029B000D95F4B50DA5B0F50D9271050DA23120041
:1029C000860E010164254C6E4D6A000E4D22D9C75A
:1029D0004EF0DAC74FF0600E436E446A4EC03EF0D0
:1029E0004FC03FF078ECFDF03EC04EF03FC04FF0DE
:1029F0004E504C5C4A6E4F504D584B6E4A50006ED4
:102A000012008DECEFF00EE1F00E0201131507013C
:102A10000D6F0F0E02011315006E0038F00B070149
:102A20000C6F0DD0F00E020114150701096F0F0E87
:102A300002011415006E0038F00B0701086FFFEF5C
:102A4000E4F0C00E016E82ECE6F002E0B00E016E22
:102A50002CA802D0D00E016E01010F5101263EEFCD
:102A60004DF0FAECE4F0E2ECECF002E1FE0EDB06F5
:102A70006950060D64ECE5F0140E4A260A0E4B224E
:102A8000FE0EDB5036ECF3F0FFEFE4F065ECEFF018
:102A9000A5EC0DF0050E0C5C06E10701E26B0A01E6
:102AA000D56BDA931CD0CAECE7F0EFCFE2F70C500D
:102AB000DF6ED5CA00F0F2ECECF0DF5031ECF0F054
:102AC000C3ECF1F0C3ECE7F0020E6F5C0CE19A0E80
:102AD0000B5C09E30B509E0806E300C0D5FAE66ADA
:102AE000A7EC90F003D0DFCFE6FFBBDFE5526950E3
:102AF00003E0D5CAB1F20BD0A8ECE6F008E00A0179
:102B0000D76B060150850A01DA81C5EC1EF0159CD1
:102B10000701E25101E0158CC30E060150170A01AE
:102B2000DAA102D0140E01D0280E060150130A01BA
:102B3000DAA304D0D8CAE7F7D9CAE8F78BEC1EF0BD
:102B40000C50FDECE5F0EFCFEFF7ADEC25F0010E0A
:102B5000E66EE66A99ECE6F07CEC95F037EC2CF04A
:102B6000E6EC09F0E552FFEFE4F0F2ECECF0C3EC38
:102B7000F1F00C5031ECF0F0C3EFE7F00C50FDEC4D
:102B8000E5F085ECECF0050E0C5C0CE00A01DAA334
:102B900006D0E7C7D8FAE8C7D9FA8BEC1EF0E5DF14
:102BA0003BECF3F0120065ECEFF0DF6A080EDF5C3F
:102BB00005E247ECE6F0EF68DF2AF8D7E552FFEFD1
:102BC000E4F065ECEFF0DF6A080EDF5C0CE247EC46
:102BD000E6F0EFCF4AF0FE0EDB504A5C02E1010E58
:102BE00003D0DF2AF1D7000EE552FFEFE4F065ECE9
:102BF000EFF00301D95104E0DB2B030ED95D17E39D
:102C000094ECE5F0DEDFE552000911E1DF6A080E21
:102C1000DF5C0DE247ECE6F0EF50FF0806E147EC21
:102C2000E6F0FE0EDBCFEFFF02D0DF2AF0D7E55251
:102C3000FFEFE4F065ECEFF0DF6A080EDF5C0BE21B
:102C400047ECE6F0EF50FF0804E047ECE6F0EF5009
:102C500003D0DF2AF2D7FF0EE552FFEFE4F069EC74
:102C6000EFF0DF6A080EDF5C10E247ECE6F0010EE1
:102C7000EFCFDBFFDB50FF0806E047ECE6F0EF6844
:102C8000010EDB5003D0DF2AEDD7000EE1ECEAF0B5
:102C900002E2E16AE552E16E4A50FFEFE4F065ECD2
:102CA000EFF0318A00ECF4F0FEECF1F0FEECF1F024
:102CB000DF6E319ADF50E552FFEFE4F065ECEFF0A4
:102CC00007018B6B8C6B2EA802D0010E2AD00C0E44
:102CD00066ECE7F0DF6E07018B2B000E8C23DF50D4
:102CE00008E0FF0EDF5C05E0580E8B5D020E8C598C
:102CF000EEE38B518D5D8C518E5904E28BC78DF7BD
:102D00008CC78EF7580E8B5D020E8C5909E30101BA
:102D10008C5103E15A0E9CECE5F02E88000E01D098
:102D2000010EE552FFEFE4F0FAECE4F005ECF0F010
:102D3000FFEFE4F07CECF1F003E21FECEFF004D0E5
:102D4000FE0EDB50F60F410FFFEFE4F023ECEFF047
:102D500004E001013651E82402D001013651E66E4B
:102D6000C40E0FEFE5F065ECEFF0FCEC26F0DF6E43
:102D70000F0EE66EDF5007E0030EDF5C04E001019A
:102D80008B51020B02E1000E01D0010E000905E09B
:102D90000A0E01017B03F35001D0000EE66ED90E3E
:102DA0002BECE5F0E552FFEFE4F065C18EF227EC85
:102DB000EBF002E166C18EF2006A02018EA302D03E
:102DC000008807D08E51010B04E08E51800B01E08A
:102DD000008C0050AAECEAF002018EA502D05F0E32
:102DE00005D08EA702D04F0E01D05E0E006E0050AF
:102DF00012ECE5F002018EB508D08E51400B02E0D6
:102E00004B0E01D04A0E12ECE5F007010F9D0201B6
:102E10008E51020B05E08E51200B02E007010F8D51
:102E20000601529523ECEFF005E08E51100B02E005
:102E300006015285258A120027ECEBF003E18EC2D1
:102E400066F102D08EC265F1D5EF16F0FAECE4F02F
:102E50003250080B35E10101DD51100B31E1060163
:102E6000BA6B020EBB6F328601018C5129E1450E0F
:102E700069ECE5F02A0E69ECE5F0440E69ECE5F04A
:102E8000530E69ECE5F0450E69ECE5F0300E69246F
:102E900069ECE5F03B0E69ECE5F05D0E9CECE5F0CD
:102EA000FE0EDBCF2CF789C72DF788C72EF701015F
:102EB00039A906D02A0E49ECEEF02A0E49ECEEF0C4
:102EC000FFEFE4F065ECEFF02E50100B06E132500E
:102ED000100B03E00701F10502E1000E17D001011C
:102EE0003951100B0AE03150200B07E1695002E024
:102EF000400E01D0210E49ECEEF007018A6BFE0E68
:102F0000DBCF88F794ECE5F019D8E552E552FFEFF6
:102F1000E4F0FAECE4F00601B82B000EB923BA5144
:102F2000B81909E1BB51B91906E194ECE5F08EDF5F
:102F3000E552010E01D0000EFFEFE4F0D9CFE6FF1D
:102F4000E1CFD9FF020EE1262E50100B03E107015D
:102F5000F10502E1000E9AD0FE0EDBCF89F70101E8
:102F600001013951100B19E03150200B16E1FE0E12
:102F7000DB380F0BE66EDEDEE552E66ED5DEE5529F
:102F8000FE0EDB500F0BE66ED5DEE552E66ECCDEB4
:102F9000E5522E0EE66EC8DEE552695027E10601C5
:102FA000B86BB96B84B007D0E66AB3DFE5520009AD
:102FB00001E001D0F7D790920000FE0EDBCFE6FFD4
:102FC00012EC7AF0E5520000C950DF6E00009082EA
:102FD0000601B86BB96B84A008D0010EE66E99DFCC
:102FE000E552000901E001D0F6D731D0010101011D
:102FF0003851080B05E101010101DD51100B27E0FB
:103000000601B86BB96B86B008D0020EE66E81DFA0
:10301000E552000901E001D0F6D790900000FE0EC5
:10302000DBCFE6FF12EC7AF0E5520000C950DF6E0C
:10303000000090800601B86BB96B86A008D0030E23
:10304000E66E67DFE552000901E001D0F6D707011F
:103050008A5103E107018A2B14D007018A0511E187
:103060000701881DDF5C0AE0695003E02550100B62
:1030700005E0040E6924E66EE9DEE5520701020E62
:103080008A6F010EDFCFDBFFDF5000D04A6E020EE9
:10309000E15C02E2E16AE552E16E4A50E552E7CFB7
:1030A000D9FF120091ECEFF0FFEFE4F091ECEFF0BC
:1030B000FC0ECCECF1F0FFEFE4F091ECEFF0FC0E45
:1030C000CCECF1F0FB0ECCECF1F0FFEFE4F070ECA7
:1030D000EFF001013CA904D0010E696E00ECF4F0A0
:1030E000696A00ECF4F078EFEFF070ECEFF00101BA
:1030F0003CA906D0010E696EA1ECEFF040ECF3F0B4
:10310000696AA1ECEFF040ECF3F078EFEFF070ECCF
:10311000EFF001013CA90BD0010E696E53ECF4F005
:1031200094ECE6F0FA0EDBCFE6FF08DFE552696AC1
:1031300053ECF4F094ECE6F0FA0ECCECF1F078EF0E
:10314000EFF0FAECE4F000ECF4F0D2C1E6FF6EEC44
:10315000E6F0D3C1E6FF6EECE6F00FC0E6FF6EECE2
:10316000E6F010C0E6FF6EECE6F0FFEFE4F078EC7E
:10317000F4F001013CA902D0010E696EF00EB6EC2C
:10318000F1F078EFEFF078ECF4F001013CA902D017
:10319000010E696EF10EB6ECF1F078EFEFF0D9CFD9
:1031A000E6FFE1CFD9FFFE0EDBCFE6FF12EC7AF0AF
:1031B000E55200008C8E000000008C9EE552E7CFA7
:1031C000D9FF12002BB203D0740E73ECE7F02B8200
:1031D00012002BA203D0760E73ECE7F02B921200B4
:1031E0002BB203D0750E73ECE7F02B8212002BA2EA
:1031F00003D0770E73ECE7F02B921200FAECE4F0B8
:1032000032B206D0790E12ECE5F0FE0EDBCF2CF2D6
:10321000FFEFE4F0FAECE4F002015ABF07D07EECD5
:10322000E5F05951EE265A51ED2208D0FF0E5915FE
:103230004A6E7F0E5A154B6E77ECF2F0FC0EDBCF28
:10324000E6FF6CECEAF04A6E4B6A4ABE4B680A0E27
:1032500074ECE8F077ECF2F0FB0EDB5069E0010172
:103260000B6B0C6B69502DE1FF0E0A01DF5D29E04D
:10327000030EDE5D03E10101CE0E21D0050EDE5D01
:1032800002E1320E14D0020EDE5D03E101019C0E5C
:1032900016D0060EDE5D02E1640E09D0DE0503E104
:1032A00001016A0E0CD0070EDE5D05E1960E0101EC
:1032B0000B6F0C6B06D0DE5104E10101380E0B6F71
:1032C0000C69FB0EDB0416E1E5ECEAF006E3D0EC5A
:1032D000F1F0EE26E451ED2205D0D0ECF1F0EE5EF7
:1032E000E451ED5A7EECE5F001010B51EE260C5154
:1032F000ED2215D0E5ECEAF006E3D0ECF1F0EE5E5D
:10330000E451ED5A05D0D0ECF1F0EE26E451ED2277
:103310007EECE5F001010B51EE5E0C51ED5A9BEC99
:10332000F4F0FD0EDBCFEEFFFE0EDBCFEDFF06D09F
:10333000FD0EDBCFB4F6FE0EDBCFB5F694ECE5F078
:1033400066ECE8F0E4ECF4F0FFEFE4F065ECEFF0AD
:10335000140EDF6E010178A302D0230EDF6E78A178
:1033600002D00A0EDF6EDF50E552FFEFE4F00A0EE6
:10337000036E0C5002E1EADF036E0050320D64EC84
:10338000E5F0010E0F0B03E054ECF2F0FDE1035009
:103390000A0DD1ECE7F001010F50D25D1050D35966
:1033A0000BE2D2510F5C02015B6F0101D351105847
:1033B00002015C6F10ECECF0120004B007D098EC46
:1033C000E9F0010101ECF1F0110E03D0A1ECF4F0F1
:1033D000100E12EFE5F0B0C6B4F6B1C6B5F681EC4A
:1033E000F1F0CBBD06D00F500601B45F1050B55BB5
:1033F00005D00F500601B4271050B523B5C6E6FF1F
:10340000B4C6E6FFE4ECF4F0056A0101CBAD02D0EE
:10341000060E05266A0E0524D1EFF0F0FCEC26F02E
:10342000056E055003E1DDECEAF003E11BECEFF083
:1034300002E0060E05266AEC11F0006E005002E074
:103440000050056EF6ECF0F003E14FC101F00ED034
:10345000A1EC0BF0000903E085C101F007D0050ED7
:10346000005C02E1016A02D056C101F0040E05249D
:10347000E66E2BEC04F0E552D5ECF0F0030E005CA8
:1034800010E178040EE125ECE7F0CBB505D0980EFD
:10349000D2273A0ED32305D0980ED880D2573A0EB1
:1034A000D35707ECEFF00CE0000405E10101B40E86
:1034B000D26F460E04D001017C0ED26F2E0ED36F58
:1034C000E66A0150E66ED2C1E6FFD3C1E6FF4EECDC
:1034D000E6F06A0E0524D1EFF0F002015B6B5C6B45
:1034E00021AC02D00101E28996EC04F00101E299DD
:1034F0000C5011E12A519EECE9F039DF0101CBBDFE
:1035000006D098ECE9F001ECF1F0130E69D0A1ECD3
:10351000F4F0120E65D0E9ECEAF00CE00101F20ED5
:10352000D26F030ED36F23DF04900101CAA50CD024
:1035300004800AD081ECE7F009E025ECE7F017DF22
:1035400004900101CBB5048038DF4DD0DC0E0F6E46
:10355000050E106E45ECF1F0780E4A1806E14B505E
:1035600004E1400E0F26060E1022050E0C5C0BE146
:10357000010EE66EE66A980EE66E3A0EE66E4ADEDA
:10358000FCECF3F02FD0040E0C5C11E198ECE9F0A8
:10359000E66E3A0EE66E4EECE6F00101CDA723D0C2
:1035A000CD51020B02E0180E1BD0190E19D00C04DD
:1035B00004E06AEC11F001080CE198ECE9F00F244A
:1035C0004A6E3A0E102027ECF4F04EECE6F0110EA5
:1035D00007D04EECEEF06BECE7F0BCECEFF0100E29
:1035E000E66E70DCE552695004E05BC263F25CC2D7
:1035F00064F2120072DF695006E1A8ECE6F002E026
:10360000EBEF19F00BDF1200FAECE4F00701B45114
:10361000320DD5ECF0F0E5ECEAF011E1FE0EDB50F6
:103620000EE10C5004E101012A519EECE9F0E9ECB5
:10363000EAF005E00101F20ED26F030ED36FFFEF47
:10364000E4F065ECEFF0695004E02550100B01E167
:10365000B9D1CEEC0CF0D6CAB3F707011E0EB46F89
:103660000C5005E17DECE8F03FC0B4F710D0030E3C
:103670000C5C0DE1030E785C02E1140E07D081ECC6
:10368000E7F005E0260E49ECF0F00701B46FD7CA69
:1036900000F00701EFAF10D0190E006E0A01D75DE0
:1036A00006E2F6ECECF086ECF1F0005E05D0190EC7
:1036B000D75D86ECF1F00026190E005C05E3190ECB
:1036C000005C0701B42705D0190ED880005407010B
:1036D000B45F040E006E0C5005E138DE86ECF1F0AC
:1036E000006E09D00C0406E0020E0C5C03E0040E30
:1036F0000C5C01E1006A0701B351FE0BE8420024B3
:10370000056EDF6A0550B45D13E2DF2AB351FE0B8C
:10371000E842B425016E01500024FE0BE842B46F6C
:103720000050015C02E20050016E0050015CB36F7A
:10373000B3C7B2F7040E0C5C03E1B351E824B26FD7
:10374000050E0C5C05E1320EB36F1F0EB46FB2694B
:103750009BECF4F0EECFB5F7EDCFB6F7040E0C5CB2
:1037600020E2DFCFE6FF50DFE552020E0C5C08E0FE
:103770006AEC11F0020804E01FEC12F0000909E005
:103780000101D2510701B5270101D3510701B62329
:1037900008D00101D2510701B55F0101D3510701E2
:1037A000B65BF8ECE8F001E109D112ECE6F0EF9637
:1037B0000701B251F6ECE5F004E24A500A08000EA7
:1037C0004B5403E312ECE6F0EF86C5ECF3F0080B84
:1037D00002E0B60E01D0B00E006E5FECE8F002E041
:1037E000B30E006E0701B751005C09E1BD51B51978
:1037F00006E1BE51B61903E1B851B25D1AE000C04E
:10380000B7F7B5C7BDF7B6C7BEF7B2C7B8F7B5C704
:10381000D2F1B6C7D3F1B251320D8AECE5F0050E04
:103820000C5C04E1C80E0F6E320E106E005052ECAC
:10383000E7F0F8ECE8F001E1C1D012ECE6F0EF9A25
:1038400012ECE6F0EF8E78ECE9F018E10701B351E5
:10385000020814E301013DAB04D012ECE6F0EF8A5C
:103860000DD00701B451F6ECE5F004E24A501E0811
:10387000000E4B5403E312ECE6F0EF9EE4EC23F071
:103880000C5003E0030E0C5C2EE10701EF51800B9E
:1038900003E1E5ECEAF027E1DF5025E1E7DB10EC9E
:1038A000ECF00A01D751190808E2190ED75D93EC24
:1038B000E7F00101D2274B50D323E5ECEAF008E210
:1038C000F6ECECF093ECE7F00101D25F4B50D35BE8
:1038D00001010A0ED303F3CFD3F1D203F3CFD2F118
:1038E000F450D32704D0DFCFE6FF8EDEE552070188
:1038F000B351320D8AECE5F078ECE9F007E0010114
:103900002A519EECE9F0960E0F6E106AD8EC09F081
:10391000030802E10101D38FC5ECF3F0200B02E0B4
:10392000B70E01D0B10E006E0701B951005C10E175
:10393000BF510101D2190CE10701C0510101D31996
:1039400007E10701C1510F1802E1C25110180DE043
:1039500000C0B9F7D2C1BFF7D3C1C0F70FC0C1F7DC
:1039600010C0C2F7005052ECE7F078ECE9F024E028
:10397000F8ECE8F021E00701C3510101D21909E197
:103980000701C4510101D31904E10701BA51B35D24
:1039900013E0D2C1C3F7D3C1C4F7B3C7BAF7070165
:1039A000B351320D8AECE5F0B20E52ECE7F0100E96
:1039B000E66E9EEC17F0E552DFEC11F0CAEC0EF06B
:1039C00094EC68F0E552FFEFE4F0F6ECF0F001E182
:1039D0001200F8ECE8F047E0040E005C05E3B4C622
:1039E000D2F1B5C6D3F117D0030E005C07E178041D
:1039F00005E1B5C7D2F1B6C7D3F10DD0DC0E0F6E1D
:103A0000050E106E07ECEFF004E0400E0F6E060E90
:103A1000106E5CEC0AF0F00E0F6E0A0E106E0004D1
:103A200003E0020E005C0EE101018BA105D08A517A
:103A30006E0D8AECE5F006D0355104E0C80E0F5E3D
:103A4000000E105A040E005C04E1700E0F6E170E8B
:103A5000106E050E005C04E1C80E0F6E320E106E83
:103A6000CB0E52ECE7F0F8ECE8F03EE00101DC0EA2
:103A7000D26F050ED36FF00E0F6E0A0E106E030E8E
:103A8000005C0CE1780409E18E51400B06E025EC66
:103A9000E7F0900E0F6E010E106ED38F07ECEFF073
:103AA00014E001018A516E0D8AECE5F010ECECF0A7
:103AB000010E0F0B05E0D890D333D233E806FBE1BB
:103AC000640E0101D227000ED323050E0C5C09E120
:103AD00001010E0ED26F060ED36FC40E0F6E090ECB
:103AE000106ECF0E52ECE7F01200530E006EE66A35
:103AF000005045ECF3F0695003E15C0E12ECE5F088
:103B00005B0E12ECE5F0A70E016E026A58ECEEF0C7
:103B1000C20E2BECE5F05D0E12ECE5F001EFECF0DF
:103B200001013CA905D0570EE66E67EC18F004D0F1
:103B3000570EE66E62EC17F0E552120069ECEFF0FA
:103B4000B4ECE5F02BE017ECE6F028E10701875133
:103B500025E101013C51800B03E1050E0C5C1EE1E7
:103B60004C0E66ECE7F0DF6E050E0C5C11E1010116
:103B7000DE9FDFA8DE8F3CA90BD0010E696E4C0ED4
:103B800066ECE7F0AFECEAF0696A3398DBA83388BB
:103B900001013CAF03D0010EDF1401D0000EE1ECB7
:103BA000EAF002E2E16AE552E16E4A50FFEFE4F02A
:103BB00001013C51800B06E0B4ECE5F003E017ECAA
:103BC000E6F001E0000C010CF3DF000902E0510E09
:103BD00001D0500E12EFE5F06FC1E6FFD00E0FECF2
:103BE000E5F054C1E6FFD10E0FECE5F070C1E6FF41
:103BF000D30E0FECE5F0E4EF1DF001013CA905D078
:103C0000560EE66E67EC18F004D0560EE66E62ECC7
:103C100017F0E552120001013851100B02E0140EAA
:103C200001D0050EE66EAC0E0FEFE5F02150400B13
:103C300006E00101DF51040B02E1DF8501D812002B
:103C400065ECEFF055C1DFFF27ECEBF003E159C164
:103C5000DFFF09D00101E051020B05E09751040B91
:103C600002E098C1DFFF040EDF02F350E66EC70EDC
:103C70000FECE5F001019751080B03E0DF51040B55
:103C800002E0000E01D0010E000902E06F0E01D02B
:103C90006E0E12ECE5F00201FB51E824E66ED40E44
:103CA0000FECE5F0E552FFEFE4F0020EE66EBC0E1D
:103CB00045ECF3F07C0E12ECE5F0070EE66E6C0EB0
:103CC00045ECF3F07D0E12ECE5F0BC0E0F6E020E2B
:103CD00096ECF0F07E0E12ECE5F06C0E0F6E070E17
:103CE00096ECF0F07F0E12ECE5F001ECECF046C142
:103CF000E6FFC10E0FEFE5F0620E006E07010E9DAC
:103D0000010158AD03D0002A07010E8D005012ECBE
:103D1000E5F0258A12000701E7510C0803E3E8519A
:103D20000C0805E2E76B0C0EE86F0A01DA9312004B
:103D3000016A0D0E015C07E07CECE9F002E0015045
:103D40001200012AF6D7000C0C0E016E015007E09C
:103D50007CECE9F002E0015012000106F7D7000CFC
:103D60000701E56BE66BD7DFE7C701F00701E85114
:103D7000D880015409E38AEC04F0F3500701E513FD
:103D8000F450E613012AF2D71200016AC9ECE9F0F7
:103D90000BE00BECF0F006E24A500508000E4B5425
:103DA00001E2012A1D0E0DD078ECE9F011E00BECD8
:103DB000F0F006E24A501408000E4B5401E2012ACA
:103DC0001F0E8AECEBF0F3CFE5F7F4CFE6F7120025
:103DD0000BECF0F016E24A504608000E4B5411E28C
:103DE0005FECE8F00EE107011F0EE56FE669050ED6
:103DF0000C5C01E1C7D0E76B0C0EE86F0A01DA83B7
:103E0000C1D0006A0A01D751F6ECE5F006E24A504B
:103E10000D08000E4B5401E2002AD751F6ECE5F0F4
:103E200006E24A501308000E4B5401E2002AD75113
:103E3000180801E2002AD751190801E2002AD751D7
:103E4000F6ECE5F006E24A501F08000E4B5401E282
:103E5000002AD751F6ECE5F006E24A502508000E9C
:103E60004B5401E2002A5FECE8F007E0020E006E1E
:103E70000101CDA302D0040E006E0C5003E0030E2E
:103E80000C5C1CE10BECF0F006E24A500508000E59
:103E90004B5401E2012AE7ECF4F006E24A500A082A
:103EA000000E4B5401E2012AE7ECF4F022E24A5002
:103EB0001308000E4B541DE2012A1BD00BECF0F04E
:103EC00006E24A501E08000E4B5401E2012AE7ECBC
:103ED000F4F006E24A502808000E4B5401E2012A91
:103EE000E7ECF4F006E24A503208000E4B5401E2CF
:103EF000012A040E4D6EEF0E4E6E010E4F6E0050F5
:103F0000506E516A526A030ED8905036513652366E
:103F1000E806FAE14D5050244A6E4E5051204B6E47
:103F20004F5052204C6E0150536E546A556AD890CF
:103F30005336543655364A505324F36E4B50542062
:103F4000F46E4C505520FAECEFF00900F5CFE5F790
:103F50000A00F5CFE6F7EAECECF005E00701E589A9
:103F6000E687E591E695030E0A01D45D02E0D4519F
:103F700009E1DEDE0701E76FE7DE0701E86F0A010E
:103F8000DA83C9DE0A01D40514E10701E805056EEC
:103F90000A0EE85D01E20506CBDE0701E76F05507A
:103FA000D880E75502E205C0E7F7DADE0A01DA83D6
:103FB0001200020ED45D12E10701E729056EE751F8
:103FC000020801E2052AC0DE0701E86F0550E85D3E
:103FD00002E205C0E8F7C4DE0A01DA8312001E0E11
:103FE000006E0C5004E17DECE8F03F500BD0E9ECA2
:103FF000EAF002E0140E06D081ECE7F004E0260EB1
:1040000049ECF0F0006E0A01D651FE0BE842056E55
:104010001200170E98ECE5F0050E0A01D803F350D4
:10402000006E0101012BA0EC96F00101200E1C6F27
:104030001E8F12001A0E98ECE5F00A01D951E1EC3E
:10404000F4F08DECECF01E8F1200D5ECF1F0F3ECF7
:104050007EF02BEC2EF0300E01011C5D02E1200EF3
:104060001C6F1E8F016B700EDCEFE8F00C5003E14B
:1040700001012A510BD0030E0C5C10E1030E785C99
:1040800002E1650E03D0785004E1960E0F6E106ABF
:1040900012002A0E49ECF0F00F6E106A12009FDF3A
:1040A0000701EFAF15D0DAECF0F0E0DF0A01D751ED
:1040B000190807E2190ED75D93ECE7F00F264B5075
:1040C0001022190ED75D17E2F6ECECF08CEFF1F050
:1040D0000A01D751190803E2190ED75D0026190EFF
:1040E000D75D03E2F6ECECF0005EDAECF0F0190ECE
:1040F000D75D01E1BBDF12005FECE8F00AE00101EF
:10410000CD930A01D751190802E20101CD830A01BA
:10411000D76B12005FECE8F009E00A0E27ECE5F03F
:104120000101CDA32BD00B0E27EFE5F0AB0E98ECE1
:10413000E5F0B5DFEAECECF00BE00101410E196FA0
:10414000500E1A6F0301D851106AE8307F0B0F6EC2
:104150008DECECF0EAECECF009E00101460E1B6F8F
:104160002A51E8240301D85D07E103D0E5ECEAF029
:1041700003E101012A0E1C6F01011E8F1200FAECEF
:10418000E4F0070EE12629EC12F00A01D65D04E204
:1041900029EC12F00A01D66F41EC12F00A01D88026
:1041A000D65504E241EC12F00A01D66F70EC12F021
:1041B000000903E00A01190ED76F11DFE5ECEAF000
:1041C00004E3190ED75D002603D0F6ECECF00526CB
:1041D0000550005C03E30550005E0AD0006AD40578
:1041E00007E1DC51D75D04E2DCCAD7FADDCAD6FAB2
:1041F00000C0D8FAF4DE05500026E5ECEAF004E34E
:10420000190ED75D002609D0F6ECECF0056E0550CE
:10421000D880005402E20550005E59ECF0F00BE249
:104220004A505408000E4B5406E2540E006EDCCA8D
:10423000D7FADDCAD6FA00C0D9FA190ED75D03E362
:10424000190ED75D03D0190ED880D7550701E36F3B
:10425000E46BEFAF02D00A0E01D0320EE403F3CFCD
:10426000E4F7E303F3CFE3F7F450E427695002E007
:10427000D7CA60F2A8ECE6F004E0060150850A0116
:10428000DA81FE0EDB5014E02150800B11E10A01AF
:10429000D45102E1DADE0AD0D40502E1BADE06D05A
:1042A000020ED45D02E1C6DE01D034DF960E096E47
:1042B0003550040B13E10A01DA51020B0FE0A8ECB0
:1042C000E6F00CE1C9ECE9F009E178ECE9F006E18F
:1042D000EAECECF003E15FECE8F003E056DD359446
:1042E00001D03EDDF3EC7EF0040E0C5C04E1010E27
:1042F0005DECEEF0FDE10C500AE10E0ED8800F549B
:10430000010E105404E20E0E0F6E010E106EFD0E23
:10431000DB5001E195D01950020B01E091D0050E60
:104320000C5C01E18DD023ECEBF001E089D0D5CA23
:10433000DFFF026802C0D5FA050EDB68060EDB68F7
:10434000D950030FE96EDACFEAFFEE68ED68016A33
:10435000050E015C5DE2010E01C0E7FFE75204E0DB
:10436000E846FE0BE706FCE10701E1154FE0695066
:104370003FECF4F001500F01E0ECE5F0EF50050DDB
:10438000DE52F3CFDEFFF4CFDDFFDD52E4ECE9F0E7
:104390001FE2010EDB500F5C4C6E020EDB5010581A
:1043A0004D6E050EDBCF4EF0060E2FECEDF010E259
:1043B000010EDB500F5C4A6E020EDB5010584B6E44
:1043C000050E4AC0DBFF060E4BC0DBFF0150026E3C
:1043D000E4ECE9F01BE33EECEBF04C6E10503F5880
:1043E0004D6E030EDBCF4EF0040E2FECEDF00EE21F
:1043F0003EECEBF04A6E10503F584B6E030E4AC035
:10440000DBFF040E4BC0DBFF01C0D5FA012AA0D7A9
:10441000FF0E0A01D55D07E1FF0E025C02E1D56BDC
:1044200002D002C0D5FA695002E0D5CAB1F2DF501D
:10443000D55D06E07CEC95F0B3ECEBF0B4ECEAF083
:10444000B3EC4BF0070EE15C02E2E16AE552E16E8B
:10445000FFEFE4F0006A800E066E056E055005025F
:10446000F350015CF4500258D8B008D000C005F0F9
:1044700006420650051206BE09D0F0D705C000F06E
:1044800006420650051206BE01D0E8D700D0120041
:10449000FAECE4F02B8421EC15F049C102F082EC37
:1044A000E6F004E094EC05F0940F026E00504C6EC0
:1044B0004D6A02501BECE6F00F50016E10C002F086
:1044C000C9DF036AFCEC26F0016E1D50040B2FE0DF
:1044D000010403E0020E015C2AE13550400B27E1A4
:1044E000FE0EDB5024E010C202F0025020E0025029
:1044F00079ECE5F002E670ECE7F019E20250FE0B11
:10450000E842D880005413E20250E824005C0FE235
:10451000FE0EDB0406E1320E02010F27000E10230F
:1045200005D0320E02010F5F000E105B032A03500C
:104530000EE102010F6B59ECF0F007E24A507108EE
:10454000000E4B5402E2710E006E00C010F22550B6
:10455000020B06E12350400B03E03250800B0AE0CF
:10456000036A006A32AE06D0000E0201116F126BB0
:104570000F6F106B035007E10050E66EE66AC80E3D
:104580002BECE5F002D0E7EC0BF0FFEFE4F05DEC94
:10459000E9F0C20E2BEFE5F0FAECE4F081ECF1F07B
:1045A000F6DF1D8EFE0EDB5005E0695003E1680E5C
:1045B00012ECE5F0FFEFE4F065ECEFF035C1DFFF62
:1045C0000101355108E02150400B05E01C50020B61
:1045D00002E0010EDF6EFCEC26F0026E036ADF5093
:1045E00006E0030E025C03E0050E025C02E1010E30
:1045F000036E8C0E006E035001E000683C0E27EC49
:10460000EFF0C50E2BECE5F0C60E016EDF50006E2C
:10461000040E025C04E1100E0026D80E016E035059
:1046200006E0006A040E025C02E1100E006E00500B
:10463000E66E01500FECE5F0046A035001E0048ED1
:104640000450E66ECE0E0FECE5F0E552FFEFE4F01D
:1046500036ECEDF003E00101355106E00201DE51D8
:1046600005E10101355102E0E5EC1CF02B8412005C
:10467000016A7DECE7F001E1012A006A3290015005
:1046800037ECE6F015ECECF0EF50800B06E0015053
:1046900037ECE6F0EF50006E3280E66A0050E66ECE
:1046A000DF0E2BEFE5F0FAECE4F0695014E1040EB4
:1046B00001012903F350006EFE0EDB5002E00050B2
:1046C00001D0000EE66EC30E0FECE5F00050E66E72
:1046D000AD0E0FECE5F0FFEFE4F0DAECF1F04D0E8B
:1046E0000A6E695003E0DE52800EDD6E010EDB5073
:1046F000BDECE5F0FF0E005C14E0BC0E12ECE5F042
:10470000DF6ADF5079ECE5F002E670ECE7F009E2F1
:10471000010EDB5089ECF0F0005058ECF2F0DF2A8B
:10472000F0D70A6A020EE15C02E2E16AE552E16E4C
:10473000FFEFE4F0FAECE4F0016A080E015C10E22D
:10474000FE0EDB50012462ECEEF0026E100E025CF5
:10475000040DF350006E005058ECF2F0012AEDD732
:10476000FFEFE4F0F8ECE8F00DE0AB0E12ECE5F052
:10477000D8EC09F0000902E1180E01D0080EE66E2F
:10478000D9DFE5521200F8ECE8F00DE0CA0E12ECA9
:10479000E5F0AAEC0BF0000902E0100E01D0000ECB
:1047A000E66EC8DFE552120070ECEFF00A0E0B5C0B
:1047B00008E125A803D0010E696ED4DF696AD2DF53
:1047C00001D0E1DF78EFEFF0CEEC0CF012ECE6F088
:1047D000EFCF4AF03DECEDF0EF5000014A5C0EE007
:1047E000C5ECF3F0E66E3DECEDF00EECE6F0C5EC5A
:1047F000F3F0800AE66EB40E0FECE5F0120084ECE4
:10480000F4F00701F1054EE001013851080B03E116
:104810003851200B02E0010EDF6E006A07018705A8
:1048200007E1695002E1008203D0DF5001E0008619
:1048300002018EB300880050AAECEAF0695002E150
:10484000010E03D0DF5004E0040E0010AAECEAF0E1
:10485000010E78ECE6F00050AAECEAF0280E78ECB5
:10486000E6F0070187051EE0020E12ECE5F0020EED
:1048700012ECE5F0006E020E005C08E1695002E106
:10488000510E0ED0DF500EE0570E0AD0FD0E005C28
:1048900009E0695002E14E0E03D0DF5003E0540EF0
:1048A0009CECE5F0E552FFEFE4F00701F10501E1D2
:1048B00012002B92E2EC18F0695006E0100EE66E42
:1048C000A60E0FECE5F00AD0E66AA60E0FECE5F0B6
:1048D000E66ABF0E0FECE5F00BEC1EF0E668A70EE3
:1048E0000FECE5F0695013E1610E12ECE5F0620E99
:1048F00012ECE5F07CEC1EF0650E28ECF3F0660E91
:104900002BECE5F0E66AE66A660E2BECE5F0220E8B
:1049100012ECE5F0695003E1420E12ECE5F021ECF7
:104920001BF0FDEC1DF08DEC0CF0695002E14AEC3F
:1049300009F013D9C80EE66EB50E0FECE5F0700E57
:1049400012ECE5F0020EE66EE66AE00E2BECE5F006
:10495000800EE66EE20E0FECE5F0010163855D95D9
:10496000B8EC11F031DF280EE66E110EE66EE66847
:10497000A90EC9ECF3F0360E28ECF3F0C00EE66E8B
:10498000A40EC9ECF3F0695002E172D866D894EC39
:1049900068F0A3DE695023E1D5EC16F0A6EC16F022
:1049A0007CC1E6FFCC0E0FECE5F055EC1EF0345068
:1049B000040B02E0530E01D0520E12ECE5F020EC95
:1049C0001EF0E1DED7ECE8F0F7DD7DC1E6FFD60EA4
:1049D0000FECE5F0B3EC16F0ECEC1DF049DE75ECF5
:1049E0001DF0010EE66ED8DDE552A1ECE9F00601FE
:1049F000B66B090EB76FB6DE640EE66EF20E0FEF01
:104A0000E5F001010A0E8C6F89EC13F0248A2A0E5E
:104A1000CCECF3F02E880701010E876F696A010163
:104A200038BB696EA5EC0DF0EADE696A1200046A13
:104A3000010160AF04D012BC048012BE04823DB9F3
:104A400004845FECE8F001E004880101E0B504862D
:104A50000450E66EBA0EADEFEBF0695008E10101CB
:104A60008051E824E66EA10E0FECE5F0E0DF1200C5
:104A7000695018E101013229080DF350E66E050E68
:104A8000325D02E2020E01D0010EE66EAA0E2BECA0
:104A9000E5F001013C51400B02E0390E01D0380E27
:104AA00012ECE5F01200016A0701EFB302D04CC12D
:104AB00001F04DC102F0EF51020B08E00C5004E18F
:104AC0000601F051010802E34EC102F00150E66E0A
:104AD00062C1E6FF48C1E6FFA80EC9ECF3F0025040
:104AE00058ECF2F042C100F0F3ECF0F004E6F20E04
:104AF0004A5C000E4B5802E2F20E006E005058EC79
:104B0000F2F03C0E006E0701EFA102D03D0E006EE8
:104B1000005012ECE5F074C1E6FF73C1E6FF72C10C
:104B2000E6FFA00EC9ECF3F071C1E6FFF30E0FEC47
:104B3000E5F00701EFB110D057ECF4F004E073ECAE
:104B400068F094EC68F01550100B06E01550200B3F
:104B500003E11598C1EC6AF0120078ECF4F0A3DFE1
:104B600001013CA904D0010E696E9DDF696A78EFEE
:104B7000EFF065ECEFF00C5003E1010EE66E84D02F
:104B800017ECE6F001E182D0020E785C67E185EC7B
:104B900004F08AECE5F0AA0E01010F24D26F000E9A
:104BA0001020D36F39BD0BD085EC04F0D5ECF0F0BC
:104BB000AA0E0101106AD2250F6ED3511022E7DC34
:104BC0007D0E12ECE5F0680E12ECE5F067ECEEF00D
:104BD000DEDC7C0E12ECE5F0690E7EECF2F00101F9
:104BE0003951400B400A01E0010E4A6ECB51040BD3
:104BF000040A01E0010E4A1805E0550E0F26000ECA
:104C0000102204D0550E0F5E000E105A49ECF1F040
:104C100001013951400B400A01E0010E4A6ECB51AF
:104C2000040B040A01E0010E4A1805E0AA0E0F5E0B
:104C3000000E105A04D0AA0E0F26000E10225DECB2
:104C4000E9F0E4ECF4F07F0E12ECE5F0030EDF6E19
:104C5000010197A113D0070EDF6E10D06CECEEF0BF
:104C600096DC7C0E12ECE5F0680E7EECF2F049EC7E
:104C7000F1F0010EDF6E010178BDDF2A92ECF1F058
:104C80000501040E146FE66A87DCE552E552FFEF7A
:104C9000E4F065ECEFF0CEEC0CF002013F6B0601A6
:104CA000C26BC2C6C0F6339E0C5022E1F05101081F
:104CB00003E31450010B17E0010E016EF0510208DE
:104CC00002E2030E016E040EF05D02E1020E016EBF
:104CD00001505BECF2F0E00E2BECE5F0F1C6E6FFE4
:104CE00018ECF2F003D0700E12ECE5F036DF6AD06B
:104CF000030E0C5C64E112ECE6F0EF981450010B2B
:104D000006E1C9ECE9F003E12BECEFF053E081ECB4
:104D1000E7F015E02E0E49ECF0F0016E020E026E87
:104D20002D0EDF6E010197A104D0040E026E4B0E12
:104D3000DF6E14A016D00201010E3F6F12D0E9EC15
:104D4000EAF00FE0030E016E010E026E1F0EDF6E21
:104D5000010178AD06D0040E016E030E026E3F0E07
:104D6000DF6E58ECEEF0E00E2BECE5F0F3C6E6FF5C
:104D700018ECF2F0C9ECE9F003E012ECE6F0EF8891
:104D80000701200E7E6F3F0EDF5C02E1100E7E6F8A
:104D9000640EDF5C02E10A0E7E6F4B0EDF5C02E107
:104DA0000D0E7E6F2D0EDF5C02E1160E7E6F7B6BAB
:104DB0007F6B03D0700E12ECE5F006DD03D0700EB1
:104DC00012ECE5F040EC4BF0E552FFEFE4F01C8410
:104DD0009F0EFAECE5F01C94005013ECEFF0005C31
:104DE00002011E6F0050E00BE838E8401E27050E58
:104DF0001E271EC200F0120020B202D00C5012007A
:104E00007D5012000A0EB6EFF1F014A205D0E2C2F6
:104E10000FF0E3C210F012009A0E09ECF2F00FC08E
:104E2000E2F210C0E3F212004C6B4D6B4E6B4F6B15
:104E3000400E506FD8904737463745374437433791
:104E40004237413740374F374E374D374C374B514C
:104E50004F5D4A514E5949514D5948514C5909E3FA
:104E60004B514F5F4A514E5B49514D5B48514C5B32
:104E7000472B502FE0D7120012A409D00101CB9983
:104E800012BECB89CC9712AC09D0CC87120001019D
:104E9000CB9712BECB87CC9912BCCC891200125092
:104EA000040B04E00101CB51100B09E11250040B7B
:104EB00004E10101CB51080B02E1000E01D0010E0B
:104EC0000490E8B004801250040B04E00101CC51BE
:104ED000080B09E11250040B04E10101CC51100B45
:104EE00002E1000E01D0010E0492E8B0048217EC3A
:104EF000EBF004E00201BB51100B02E1000E01D007
:104F0000010E0494E8B0048434AC09D0129E01016F
:104F1000D7B1128E129CD7A308D0128C06D0129E45
:104F200004B0128E129C04B2128C0450040B040ABA
:104F300001E0010E4A6E0450010B4A140496E8B0D9
:104F4000048607011D9904B61D891D9704A61D87B7
:104F50000101E3B906D007010B9904A218D00B890F
:104F600016D007010B990450020B06E0020E020155
:104F7000BC1502E007010B8907010B910450020BDD
:104F800006E0010E0201BC1502E007010B8104508E
:104F9000040B05E011ECE9F002E0000E01D0010E77
:104FA0004A6E0101D751010B4A140498E8B00488F5
:104FB00007011B9904B81B891B9704A81B87079935
:104FC0000101D7A302D0070107890701109304B498
:104FD00010830101E39104B6E381E39304B8E38312
:104FE00017EF25F00701109B12A4108B1FECEBF0BC
:104FF00074ECE9F005E011ECE9F002E0DAEC0CF019
:105000003AECEEF03FEFEEF065ECEFF085ECF2F00D
:10501000200E89ECF0F00050026E0F0E89ECF0F0DB
:1050200001012C51005C19E1250E025C16E1050E10
:105030004FECF1F00101CAA903D089ECE6F0076A50
:10504000050E0C5C07E1030EE66E100EDF24E66E23
:1050500020ECF2F00A6A010E02D00A6A000EE55254
:10506000FFEFE4F0FAECE4F0FAECECF03B812C8C8E
:105070002D8AD8ECE7F07EECE5F0EE50ED1011E073
:105080000101452B640E455D03E2BEDF00091BE113
:105090000101450703E0B8DF0009FAE10101452BF2
:1050A00012D001014507FF0E455D03E0ADDF0009A9
:1050B0000AE10101452B640E455D03E2A5DF00090D
:1050C000F8E101014507FFEFE4F02A50800B0DE005
:1050D00001013851400B09E02C50100B06E12B5018
:1050E000010B03E1100E2C5D01E3000C010C2FEC11
:1050F000EFF004E033ECEFF001E2010C000C0701EB
:10510000E06B070E1315006E400E136F0050131363
:105110000101389D2BAA38D0020E3A5D02E1070149
:10512000138701013A51020807E2070E3A5D04E2D3
:10513000020E3A5D0701E06F2AAE26D0070E01018C
:105140003A5D0BE12C50100B08E14951780803E25D
:105150006C0E495D496F7DEC56F0080E01013A5D19
:1051600013E3388D4951780804E207011387139B34
:10517000139D01013A51080807E20D0E3A5D04E261
:10518000080E3A5D0701E06F070112911293128930
:1051900082ECE6F011E007011281128312997DEC96
:1051A000E7F003E17851800B05E02C0505E1605143
:1051B000400B02E10701128921AC02D09BEC0FF0F9
:1051C000B4EC2CF0258A12008DECEFF04B6ADA0F6C
:1051D0004A6E060EB7ECEFF0006E009EFE0EDB503E
:1051E000040806E1FD0EDB504F0802E2020E006EDD
:1051F000FFEFE4F00101E351200B03E04451040808
:1052000003E34451040801E2446B040E445D02E1EF
:10521000190E04D0160E4425B8ECE5F0006E0050CF
:10522000E66EE66A3C0EE66E66ECFAF0FCECF3F035
:1052300005EC0CF0258A12000201320E346F395150
:1052400002E0140E346FC80E496F640E506F1EAC2E
:105250002A981E50400B03E02B50800B02E1E2EC39
:1052600018F00201906BFC6B1200FAECE4F0FE0EF9
:10527000DB500EE02AA006D0FE0EDB50030B02E14D
:10528000CBEC07F0280E5CECE7F0FE0EDB06EFD768
:10529000FFEFE4F001C502F50501006B289C010158
:1052A000DE911200A7ECE9F0F5DF17ECE6F002E082
:1052B000080E086E12000850220A01E167D1030AA5
:1052C00001E146D1010A01E1C7D03F0A17E0010A16
:1052D00001E075D1288C2BECEFF007E0200E0601E1
:1052E0004A5D03E0200E69ECE6F01E901F0E086E8A
:1052F00002013D5101E164D1086A17D00501005156
:1053000001E181D017ECE6F014E00501115107E14D
:10531000020E145D0EE18AEC0FF000090AE10201B1
:105320003D5101E13D2B080E086E01011F0EA76FD4
:105330001200050100070251EA6A000FE96E080E2B
:10534000EA22EFCF02F7022B025179ECE5F002E6F8
:1053500035ECEEF001E3026B17ECE6F006E002C775
:10536000E6FFFAEC4FF0E5524BD03C0E0701025D30
:1053700004E12582248C239C12003E0E025D04E190
:105380002592249C238C1200740E025D64E00601B9
:10539000F05107E02A8A02C7E6FF41EC8AF0E552A5
:1053A0002A9A800E0701025D10E2C00E02254A6EA5
:1053B0004B6A000E4B22200E4A5E000E4B5A5FECE9
:1053C000E5F04DECE7F00701026F800E025D03E1AE
:1053D0000201040E676F07010251800805E2800E8A
:1053E000025DFD0F0201676F800E0701025D06E39B
:1053F000220E086E05011F0E056F120002512BE0F0
:10540000200E086E12001DECECF007E007010251BF
:10541000800803E3200E69ECE6F044DF17ECE6F0C9
:1054200006E0289C080E086E0101100EA76F285098
:10543000200B01E1C5D002016A5101E1C1D0199AE6
:105440006ABF198A2A6B010EE66E7F0E6A1541EC5F
:10545000E7F002016A6B12001750800B09E11E5041
:10546000040B06E01E50080B03E08150080B4CE1D2
:105470002850200B09E01750800B06E06DECECF093
:1054800003E0250E675C1FE150EC80F00BDF2194F8
:1054900017ECE6F003E00201010E3D6F28AA90D060
:1054A00002016A6B6AC22AF20601F05101E188D05A
:1054B00007010251800801E283D03088200EE66E99
:1054C00041EC8AF01DD0350E675C09E1010EE66EF5
:1054D000ABEC0FF0E55222ECECF0179E12008FECD3
:1054E000B5F000090FE00D50006E020E49ECF3F02C
:1054F0000D50026E00500D6E0250E66E15EC8FF0EE
:10550000E5521200DEEFB8F017ECE6F006E0080E08
:10551000086E01011F0EA76F1200FE0E0701021593
:105520000EE0238E010E016F02A102D0030E016F67
:1055300002910243210E086E0501200E07D00201E0
:10554000020E676F220E086E05011F0E056F120016
:105550000701015114E00107248003EC80F0086A80
:105560001EA007D0020E086E1BECEBF002E162EC0D
:10557000E9F00101210EA76F1E80239E1200020197
:10558000010E676F238E220E086E12000201675112
:1055900013E02490670703EC80F0030E086E1EB042
:1055A00005D0070E086E006A36EC91F00101220E5C
:1055B000A76F239E1E90120005C508F0120072DE30
:1055C000120086C206F118ECE9F00AE2100E2C5D1A
:1055D0002FECE6F0060E2DECF0F0EFCF06F104D044
:1055E0002CA802D0960E066F0651D880495502E2CB
:1055F00006C149F11200DACFE4FFE2CFDAFFE9CFCA
:10560000E4FFEACFE4FFE652FC0EB36EF30EB26E97
:10561000020125070201255105E10201320E256F25
:10562000010124811E961E94010158A105D081B468
:105630001E8481B21E8604D081B21E8481B41E866F
:10564000020126070201265137E10201050E266FED
:105650000101AB5116E00101AB07020102016651E5
:10566000020B05E01E50040B02E1020166810201FB
:1056700002016651080B05E01E50080B02E1020111
:1056800066850101AC5106E0FF0E0101AC5D02E050
:105690000101AC2B20AE04D00601E42B000EE52363
:1056A00007017D5109E007017D0707017D5104E1F4
:1056B0007EC77DF7010124830101AA5102E00101A7
:1056C000AA0702010D2B010127970101279501016E
:1056D00027A102D001012785010127A302D00101E2
:1056E0002787010127930101279188A202D0010198
:1056F000278188A002D0010127830F0E0101271501
:105700000101266F01012651EA6AC90FE96E060EF2
:10571000EA22EFCF25F1010125A12BD02050080B63
:1057200008E0010101013C51010B03E02850010B8D
:1057300020E02E50400B03E03050200B1AE02150A7
:10574000200B17E0010125AF02D0790601D0792A9C
:1057500001010101CA51100B0CE02050080B09E0B7
:105760002C50200B06E1010125AF02D0070601D025
:10577000072A0101289701012895010128A102D0DB
:1057800001012885010128A302D001012887010118
:1057900028930101289188A802D00101288188AAB4
:1057A00002D0010128830F0E010128150101266F87
:1057B00001012651EA6AC90FE96E060EEA22EFCF0F
:1057C00025F1010125A124D0010101013C51200B4B
:1057D00016E12050080B13E02E50400B08E10101A8
:1057E00001013C51020B0BE02850010B08E12E5047
:1057F000400B0EE0010101013C51010B09E1215078
:10580000200B06E0010125AF02D0070601D0072AD0
:105810009EAA1CD0ABA209D0AB98000000000000EB
:10582000000000000000AB8811D00701C72B070162
:10583000C651C62BEA6A000FE96E0C0EEA22AECF03
:10584000EFFF0701C75102E1C6C7C5F7A1920701E3
:105850005207E552E5CFEAFFE5CFE9FFE5CFDAFFF2
:10586000110001013CAB02D03C9B248A12000701CD
:10587000EFB103D0129A129812001298EFA3128877
:10588000129AEFB3128A12000701EF81E1EC09F0DE
:1058900027EFECF019A602D0199612002CA806D01A
:1058A0000101E0A523D0560E27EFE5F04B0E0A6E5E
:1058B000200E016E12A002D0600E016E01507CEC31
:1058C000F4F0005013E0FF0E005C10E026840101AC
:1058D000B06B45C11FF2FC0E456F12B0452B9BEC1F
:1058E000E7F0E0ECE8F026941FC245F11200220E2A
:1058F000C1EFF3F001018BAD09D0D9752C51615D79
:105900000CE1CD95D9A509D0CD8507D0D9792C51F9
:10591000615D03E1CD99D9B9CD8985EC0CF038EF03
:105920000DF034AC02D07AEF2CF02CA61BD0127004
:10593000129212A012820101CB9F12B0CB8F0701ED
:10594000169F12B0168FB8EC09F0E66AEBECC6F0C1
:10595000E552ACECC5F00201906B258A17859ADF01
:10596000ACEF0CF077EF2CF0B4ECE5F003E017ECC3
:10597000E6F006E01494010157A306D0148404D085
:10598000149401013CB51484149614A4148614983C
:105990001450040B04E182ECE6F001E014881200DC
:1059A00070ECEFF0006A0301C95111E0CCC359F269
:1059B000CDC35AF2800ECD151DE0CCC359F2CDC334
:1059C0005AF20201596D5A1F000E5A2311D044ECAD
:1059D000EDF0595F7A0E5A5B0101A00E505D7A0E10
:1059E000515908E244ECEDF0D88059577A0E5A57D5
:1059F000800E006E060E436E446A59C23EF05AC2D3
:105A00003FF078ECFDF03EC059F23FC05AF2005032
:105A100002015A13010178A717D0BBEC3EF0C0EC8D
:105A200096F002C101F003C102F004C103F005C108
:105A300007F1696A560E65ECE9F0010E696E560EC3
:105A400065ECE9F0DF50696EE552FFEFE4F0FAEC47
:105A5000E4F0FB0EDBCFE9FFFC0EDBCFEAFFEECF7D
:105A60004AF0EECF4BF0EECF4CF0EECF4DF0EFCF53
:105A70004EF099ECE8F04AC0EEFF4BC0EEFF4CC090
:105A8000EEFF4DC0EEFF4EC0EEFFFFEFE4F01EEC68
:105A9000F4F0F3ECE6F09F0EE66E010E40ECE9F058
:105AA000CDEC3AF0D850010B06E0FF0E01019A5DF3
:105AB00002E0010E01D0000EFFEFE4F069ECEFF020
:105AC000005027ECF2F0DAECFDF0D5ECFDF0000927
:105AD000FCE1C450006E1C50040B32E0F3ECF0F01B
:105AE00004E6F90E4A5C000E4B582AE20201F2511C
:105AF0004B6AE8307F0B4A6EC80E39ECF0F045EC8B
:105B0000F1F009ECE6F0C5ECEFF0EECF3EF0EDCFB2
:105B10003FF0CBECF8F03CC0EEFF3DC0EDFF09ECF0
:105B2000E6F0FA0E436E446AEECF3EF0EDCF3FF062
:105B300078ECFDF03EC0EEFF3FC0EDFFEF50006E91
:105B4000020EE15C02E2E16AE552E16EFFEFE4F091
:105B500065ECEFF00050DF6E110E4A6EEA0E4B6EF0
:105B6000010E55ECF1F00150006E009E0EEC97F026
:105B700001AEF2D7E552FFEFE4F065ECEFF0005034
:105B8000DF6E2450100B12E10050E66E8DEC04F035
:105B9000E552800B0BE00101450E196F520E1B6F91
:105BA0001BC11AF1200E1C6F040E016F2B8824A854
:105BB00008D00D0E4A6EEC0E4B6E010E55ECF1F056
:105BC00007D0DFCFE6FF8DEC04F0E552016EDF2A4F
:105BD0002BA802D0019E2B980150006E009E37EC3E
:105BE00097F001AEE4D72498E552FFEFE4F07CECA7
:105BF000F1F003E21FECEFF004D0FE0EDB50410F9A
:105C0000F60F006E0EEC97F0FFEFE4F02AECF4F0E4
:105C1000DB380F0BE66EEBDFE552FE0EDB500F0BB1
:105C2000E66EE5DFE552FFEFE4F0FAECE4F04BEC72
:105C3000EDF0020E0101002783EC96F0DF50006EBC
:105C4000050E0101005F83EC96F0030E0101005F79
:105C5000E552FFEFE4F0FAECE4F04BECEDF0ADECE4
:105C6000E9F0DF50006E0101020E016FA0EC96F02A
:105C7000E552FFEFE4F000C06FF2A2EC93F0FF0EEC
:105C8000005C01E065DF1888120000C070F2AEEC25
:105C900093F0FF0E005C01E070DF188A1200A2ECA6
:105CA00093F0FF0E005C01E053DF188C640E096E68
:105CB00025961200AEEC93F0FF0E005C01E05DDF74
:105CC000188E640E096E25961200FAECE4F09BEC37
:105CD000E7F0F1ECEAF0B6ECE6F0FFEFE4F0FAEC16
:105CE000E4F09BECE7F008EFF1F0FAECE4F0F5EC0F
:105CF00089F00101190EA96FFC0EDBCFADF1FD0E8D
:105D0000DBCFAEF1FE0EDBCFAFF1FFEFE4F0830EA1
:105D10000A6EE00E7CECF4F0800E005C08E2F5EC1C
:105D200089F00101190EA96F0201E00EDF6F120068
:105D30002AECF4F0DBCF4BF0800E4B1407E052EC72
:105D4000EDF04A6C4B1E000E4B2202D052ECEDF0EF
:105D50001AECF3F0FFEFE4F0016A040E015C0DE2CF
:105D600001287EECF0F0EA22B9ECEAF001507EEC7A
:105D7000F0F0B9ECEBF0012AF0D7EA0E66ECE7F0B0
:105D80000301C46F318AFEECF1F00301C56F319A53
:105D90000101DE870480016A040E015C22E20150E9
:105DA0007EECF0F0EA22EECF4CF0EFCF4DF0012880
:105DB0007EECF0F0EA22EE504C5C4A6EEE504D580C
:105DC00027ECF4F08BECF2F0010E7DECE6F007E24C
:105DD0000490050E7DECE6F002E20101DE97012A57
:105DE000DBD70450010B48E001018F51080B03E1A0
:105DF0000201515141E01850020B3EE102015051A5
:105E00003BE1BCC3E6FFBDC3E6FF8BECF2F00F50F5
:105E1000101032E0F40E0F5C010E10582DE2040158
:105E2000440EBB6F0301800EBD1503E00401550E47
:105E3000BB6F2BECEBF0040E7DECE6F002E2310ED2
:105E4000026F140E7DECE6F002E2330E026F3C0EA0
:105E50007DECE6F002E2390E026FDC0E7DECE6F03E
:105E600002E2340E026F020E37ECEFF003E20201A1
:105E7000320E506F2FECCFF012002AECF4F0DBAEB4
:105E800008D0DB50FF0DFE0EF3CFDBFF47ECEBF04D
:105E900007D047ECEBF0DB50FF0DFE0EF3CFDBFF3E
:105EA000DB50FFEFE4F065ECEFF00701875101E014
:105EB00045D1F10501E142D13350040B01E13DD15F
:105EC0000C5004E18650020B01E137D1E30E66EC81
:105ED000E7F00601C16F81ECE7F001E094D0140E09
:105EE0000601E76EC119E8AE02D0C13503D0E75014
:105EF000D880C15502E2140EC16FEC0EE76EC119D5
:105F0000E8AE02D0E73402D0E750C15D02E2EC0E09
:105F1000C16FC051E76EC119E8AE02D0C13503D0E0
:105F2000E750D880C15502E2C02B0BD0C051E76EBC
:105F3000C119E8AE02D0E73402D0E750C15D03E2F8
:105F4000C007C0C6C1F6080E4A6E4B6AC5C63EF011
:105F5000C6C63FF059ECEDF03EC0C4F6C4C64AF0E8
:105F60004B6A4ABE4B684A500601C55F4B50C65B40
:105F7000C1C64AF04B6A4ABE4B684A50C5274B50CF
:105F8000C623C4C6E6FF79DFE552016E010EE66E58
:105F90000E0E012447ECE7F002012B5101E1CDD0B8
:105FA0001A9EFCECE8F002E0000E01D0010E4A6EF1
:105FB0000C5003E1DDECEAF008E00C5004E00101D4
:105FC000CA51040B02E0000E01D0010E4A1804E091
:105FD0000601C151792603D00601C151795ED5EC85
:105FE000EAF005E02050020B02E17950076E06014D
:105FF000C15101E0A2D002012B51320801E39DD032
:10600000320E2B6F9AD0E40E66ECE7F00601C36FF8
:10601000026A016AC151E76EC319E8AE02D0C33506
:1060200003D0E750D880C35505E2C151C35DEFEC02
:10603000E9F0026E0601C351E76EC119E8AE02D065
:10604000C13503D0E750D880C15505E2C351C15DC9
:10605000EFECE9F0016E0601C251D880025402E271
:1060600002C0C2F6C051D880015402E201C0C0F69D
:10607000000EE76EC219E8AE02D0C23503D0E75079
:10608000D880C25505E2010EE66E0D0E47ECE7F032
:10609000010E0601E76EC219E8AE02D0C23503D088
:1060A000E750D880C25505E2010EE66E0C0E47ECB3
:1060B000E7F0020E0601E76EC219E8AE02D0C23563
:1060C00003D0E750D880C25505E2010EE66E0B0EF4
:1060D00047ECE7F0000E0601E76EC019E8AE02D00B
:1060E000C03503D0E750D880C05505E2010EE66EFA
:1060F0000F0E47ECE7F0010E0601E76EC019E8AE9F
:1061000002D0C03503D0E750D880C05505E2010E5B
:10611000E66E100E47ECE7F0020E0601E76EC019BE
:10612000E8AE02D0C03503D0E750D880C05505E2B4
:10613000010EE66E110E47ECE7F03394E552FFEFE7
:10614000E4F065ECEFF00701F10504E1FD0EDB6A18
:10615000FE0EDB6AFC0EDB504DE102013A514AE1D2
:106160000490FE0EDB50140804E2140EF8ECE7F085
:106170000480FE0EDBCF4AF06B51D8804A5403E214
:10618000FE0EDBCF6BF201012B51100B03E0050E6D
:106190000C5C05E10450010B02E0FE0EDB2ADF6A15
:1061A000150EDF5C1AE2006AFE0EDB5004E0FE0E04
:1061B000DB50DF5C0BE301012B51100B09E0050EF6
:1061C0000C5C06E002016B51DF5C02E1010E006E27
:1061D000005046ECE9F0DF2AE3D71450010B6AE0E7
:1061E0000201315167E10C5003E0030E0C5C62E1E7
:1061F000338460D0FC0EDB0431E102013A5106E049
:10620000FD0EDB5003E12350400B57E1FE0EDB5047
:10621000080803E2080EF8ECE7F0FD0EDB500C086E
:1062200005E20C0EF36EFD0EF3CFDBFF03ECE9F09D
:10623000150EDF5C3FE2FE0EDB5004E0FE0EDB508D
:10624000DF5C07E3090EDF5C07E3FD0EDB50DF5C7C
:1062500003E2010E46ECE9F0DF2AEAD7FC0EDB5040
:10626000020828E1FE0EDB50080803E2080EF8ECF5
:10627000E7F0FD0EDB500C0805E20B0EF36EFD0E91
:10628000F3CFDBFF03ECE9F0150EDF5C13E2FE0E4B
:10629000DB5004E0FE0EDB50DF5C07E3090EDF5C41
:1062A00007E3FD0EDB50DF5C03E2010E46ECE9F094
:1062B000DF2AEAD7FE0EDBCF1DF2E552FFEFE4F056
:1062C0007D504DECE9F0A7ECF4F00150080D4A5078
:1062D000F3240A01E26F4B50F420E36F1200010136
:1062E000C451BF5D0CE1C551C05D09E1C651C15D3E
:1062F00006E1C751C25D03E1C851C35D01E0000C76
:10630000010C7D500C5C01E0000C0C500BE1DDEC4D
:10631000EAF001E0010E4A6ED751400B01E0010E98
:106320004A5C2DE0030E0C5C24E10101D65153ECD4
:10633000E6F0785C1EE181ECE7F00CE00101CB5166
:10634000040B01E0010E4B6ED751040B01E0010E6E
:106350004B5C15E081ECE7F00CE10101CA51040B44
:1063600001E0010E4C6ED651040B01E0010E4C5CB5
:1063700006E00C5003E0030E0C5C01E1000C010C84
:10638000AEDF000903E0BDDF000901E1000C010CF4
:10639000F7DF00092FE0050E0C5C01E1010C7D50D8
:1063A0004DECE9F0F2ECECF07D5097ECF1F001509F
:1063B00044ECF4F00C50100DF3CF50F0F4CF51F04A
:1063C0002A0E50260A0E51220701E251080D5050A4
:1063D000F3244E6E5150F4204F6E4EC0E6FF4FC076
:1063E000E6FFA9ECF9F0526E060EE15E525000098C
:1063F00001E1010C000C2CC161F10FC110F11BB2C5
:1064000002D089ECE6F00C507D6E2E50400B03E17B
:106410003550200B17E0010139A306D0D893CCB337
:10642000D883D895CCB5D885D79DCBBDD78DD795FA
:10643000CBB5D785D695CAB5D685CFECF3F041EC70
:10644000F0F01BD07D5004E10101D79DCBBDD78D6D
:10645000030E7D5C12E10101CFECF3F041ECF0F0B2
:1064600081ECE7F006E00101D795CBA506D0D785F2
:1064700004D00101D695CAB5D6852E50400B03E154
:106480003550200B0CE0500EE66EE66AD2ECF3F0CD
:10649000E66E7A0EE66E0A0EDFECE6F00CD0050E24
:1064A0000C5C09E0FEECECF09FECF0F07D5097EC1A
:1064B000F1F091ECF2F0050E7D5C08E07D50EA6AA7
:1064C000CF0FE96E0A0EEA22E2C7EFFF120061C1A8
:1064D0002CF110C10FF1FAECE9F07D500C6E2E504A
:1064E000400B03E13550200B07E095ECECF0D2ECCB
:1064F000F3F0DFECE6F00DD0050E0C5C0AE0A9EC41
:10650000F0F00C50100D61ECE7F044ECEEF091EC83
:10651000F2F0050E0C5C02E03BECF3F01200FAEC3A
:10652000E4F036DF00090FE1BEEC15F0FE0EDB50A3
:1065300002E161DF01D0CBDF2BECECF0258AFAEC35
:10654000ECF03B833B81FFEFE4F02D50100B12E0A9
:1065500074ECE9F00FE0BEEC15F04DDF010E696E52
:106560001982A5EC0DF046EC15F002ECEDF046ECCE
:1065700015F0199212002E8C84ECEEF051EC0AF01A
:106580001B9480ECEEF0696A01013CA90DD0348CBB
:10659000010EE66E1FD9E552A5EC0DF040EC4BF074
:1065A0001FECEBF085EC0CF046EC15F04CEF05F031
:1065B000FAECE4F080ECEEF0CDECE9F012E1CB91F6
:1065C000D7B1CB81CB93D7B3CB83CD95D9B5CD857F
:1065D000CD99D9B9CD89CD91D9B1CD81CD9FD9BF33
:1065E000CD8F2E9C18983CA906D0349CE66AF2D830
:1065F000E552A5EC0DF046EC15F0FE0EDB5002E086
:1066000040EC4BF0E5EC1CF01FECEBF04CEC05F033
:10661000FFEFE4F0BEEC15F0CDECE9F011E09EECFC
:10662000E6F0358A17D8359A46EC15F01D8A9EECAF
:10663000E6F01D9A198457ECE7F01994BFEFEBF0E0
:106640003CA903D087ECEEF0696A04D846EC15F05B
:10665000D0EF10F061C102F010C103F0C4C1CFF25D
:10666000C5C1D0F2C6C1D1F2C7C1D2F2C8C1D3F2FE
:106670007D50006E8BECEEF0D8C1DCF12E50400B5B
:1066800003E13550200B08E095ECECF0580EE66E77
:10669000060EDFECE6F009D0050E005C06E0A9EC82
:1066A000F0F04EECF3F05CECEDF0016A050E005CEE
:1066B00003E000504DECE9F09EDE02C02CF103C077
:1066C0000FF1CFC2BFF1D0C2C0F1D1C2C1F1D2C26D
:1066D000C2F1D3C2C3F100500C6E2E50400B03E147
:1066E0003550200B1EE0010139A30ED0CC93DCB352
:1066F000CC83CC95DCB5CC851396CCB313861394A0
:10670000CCB5138427ECC0F00101CB9DDBBDCB8D54
:10671000CB95DBB5CB85CA95DAB5CA8512ECF0F01E
:1067200019D00C5004E10101CB9DDBBDCB8D030ED4
:106730000C5C10E1010112ECF0F081ECE7F006E0F6
:106740000101CB95DBA506D0CB8504D00101CA950C
:10675000DAB5CA852E50400B03E13550200B0AE014
:10676000500EE66EE66A4EECF3F0D2ECF3F0DFEC9E
:10677000E6F00BD0050E005C08E0FEECECF04EEC11
:10678000F3F09FECF0F05CECEDF001C0E2F7050EE9
:106790000C5C04E0CAECE7F001C0EFFF04900101DB
:1067A0003CB104803C913CB33C813C9304B03C83BD
:1067B000139C3CB1138C139E3CB3138E2EBC03D0A0
:1067C0002BECECF0258AF1EC38F0FAECECF0BF0E93
:1067D0003B6F12008DECEFF00AE0696A01016395EE
:1067E000E4EC23F0010E696E01015D8509D0010E14
:1067F000696E01015D95E4EC23F0696A010163852E
:10680000E4EC23F0FFEFE4F069ECEFF00E0E010191
:10681000305DDF6E060E3125AFECEAF00601F45173
:1068200026E030ECEEF0060ED89010320F32E8047D
:10683000FBE1040EDF02F3508CECF1F0200E90EC43
:10684000EEF002E20F6A106A010EDB504C6E4D6AE8
:106850006BECE7F0070E74ECE8F06EECE8F0FF0E7E
:106860007DECE6F002E20F68106A0FC0F5F6DF502B
:10687000005E59ECF0F006E24A50C808000E4B5496
:1068800001E2006A010EDB504C6E4D6A0050060DAD
:1068900064ECE5F06EECE8F00F50006E0050150867
:1068A00002E2150E006E020EE15C02E2E16AE552C0
:1068B000E16EFFEFE4F065ECEFF00201315105E12C
:1068C0002150010B02E1345102E0000E1DD0AF0E49
:1068D000FAECE5F099DF0050DF6E00C0D4F7090E46
:1068E000016E01012BB901061450010B06E00150A5
:1068F000D880005402E20150006EE66AE66A005059
:10690000E66EBEECE8F0DF50E552FFEFE4F0FAECA3
:10691000E4F0016A0A0E015C19E2FE0EDB50010B85
:1069200006E0270E01248FECE5F0675C0AE0FE0E1E
:10693000DB50020B09E0310E01248FECE5F0675CBF
:1069400003E101500D6E02D0012AE4D7FFEFE4F01D
:10695000FAECE4F0800E0D6E17AE17D0179E1750AC
:10696000010B03E11750100B10E0100E0D6E94ECAC
:10697000E5F0CDDFE5522A0E675C02E1200E0D6ED8
:106980002B0E675C02E1400E0D6EFFEFE4F0FAECB7
:10699000E4F005ECEAF094ECE5F0F7EC0BF0E552EE
:1069A00053ECF3F00101A46FA451640D8AECE5F0FF
:1069B000010EEB50680F5FECF2F058ECF3F063EC73
:1069C000EDF000504C6E4D6A01014C504A5CD26FA4
:1069D0004D504B58D36F2AA60BD09A5163ECEDF073
:1069E0000101D2514A5C0F6ED3514B58106E06D044
:1069F0009A51106AD2250F6ED3511022FBECEEF0A3
:106A0000ACECEFF03EC0A4F13AC09AF1FFEFE4F035
:106A1000FAECE4F005ECEAF0DB502FECE6F0030EC4
:106A20002DECF0F0EF500101A45D02E0000E11D05A
:106A3000FE0EDB502FECE6F015ECECF0EF509A5D1B
:106A4000006E00BE006C040E005C02E2010E01D07C
:106A5000000EFFEFE4F0D6ECF3F0920E4A1810E1CE
:106A60004B500EE1006A3BEC2EF0BD0E006E45EC83
:106A70002EF0096A228602018D6B7E6B299E082A00
:106A8000D6ECF3F0930E4A1845E14B5043E1010E6A
:106A9000E66E5EDFE5520A0E0D5C25E202018D51C5
:106AA000050826E37E51020823E38D2B29BE7E2BA9
:106AB000010E016E070E015C13E20128D4ECE5F033
:106AC000EF50006E060E015C05E1800E0101181505
:106AD0000D10006E63ECF2F000C0EFFF012AEAD760
:106AE0000101189F17D0200E0D5C08E129AE02D0DD
:106AF000268E10D0298E0101188F0CD0400E0D5C0F
:106B000004E1980E086E1B8805D0100E0D5C02E1A2
:106B10009A0E086ED6ECF3F0980E4A1801E07DD07C
:106B20004B5001E07AD0010E016E070E015C0DE2C0
:106B300063ECF2F0EF9E63ECF2F0EF500E0803E12D
:106B400063ECF2F0EF6A012AF0D712C1A4F10A0E49
:106B500001011303F35014259A6F0A0E1503F35025
:106B600016259B6F0A0E1703F3CF9CF19E6B9EC1F7
:106B70009DF1040E02018D5D0DE27E510BE115C108
:106B8000A4F10A0E01011603F35017259A6F9C6BAE
:106B90009CC19BF102017E0508E114C1A4F19BC1D7
:106BA0009AF19CC19BF101019C6B020E02017E5D7A
:106BB0000EE113C1A4F10A0E01011403F3501525CF
:106BC0009A6F0A0E1603F35017259B6F9C6B9A0E53
:106BD000086ED7EC0DF0006E005013E10101A451D6
:106BE00003E19A51370802E2268E120083ECE8F0A6
:106BF0000A0E005C06E10101DD51010B02E03CEFF1
:106C000009F000C02CF157ECE7F09DEC04F058ECD3
:106C10000BF024ECEEF0D8ECE7F0D6ECF3F09A0EA3
:106C20004A1807E14B5005E1189A189853DA0C0EF0
:106C3000086E12008C9804902EB00480695003E016
:106C400004902FBC04803F0E07013715006E04A08E
:106C500002D0008C01D0008E01018EA102D0300E36
:106C6000C66E0050E66E12EC7AF0E55236C7E6FFCB
:106C700012EC7AF0E55239C700F0040E0002F3CFAF
:106C800000F0070138BF0082070138BD008038C717
:106C900001F0040E0102F3CF01F0070137BF0182BA
:106CA000070137BD018004A002D0008C01D0008E06
:106CB0000050E66E12EC7AF0E5520150E66E12ECEE
:106CC0007AF0E5520470200E006E04A002D0280E67
:106CD000006E0050E66E12EC7AF0E552080EE66E99
:106CE00012EC7AF0E5528C880000310EC66E6950C5
:106CF00004E12E9004B02E8003D02F9C04B02F8C82
:106D00001200010178B71FD023EC7AF0080E692435
:106D10004A6EF00E8C144A108C6E93EC5EF08A9AD8
:106D20000000E8EC08F0210EE66E12EC7AF0E55275
:106D3000080EE66E12EC7AF0E5527CDF8A8AF00EDD
:106D40008C161FEC7AF01200010178B71BD00201FB
:106D50000D6B23EC7AF0080E69244A6EF00E8C1449
:106D60004A108C6E93EC5EF08A9A000063DF37C79E
:106D70003AF738C73BF78A8AF00E8C161FEC7AF088
:106D80000DC20EF212006950020DF3CF5BF7F4CF83
:106D90005CF7530E07015B27070E5C236950020D59
:106DA000F3CF65F7F4CF66F75D0E6527070E662310
:106DB00001019A51C80D64ECE5F09B51020D4A5057
:106DC000F3240F6E4B50F420106E9C51310803E2F7
:106DD0000F2A000E1022CC0E0F5E060E105AD8ECB1
:106DE00009F0006E005012E000504CECF2F0400B45
:106DF00003E12850040B0AE00050E66E5AEC0EF056
:106E0000E5520050310802E2D8ECE7F0010EE66EE0
:106E1000AEEC98F0E552320E4B6E4BC044F09CC184
:106E20003FF0BCECFDF03BC04AF00A0E4C6E4CC08B
:106E300044F04AC03FF0FAECF0F0056E47ECE8F0A1
:106E4000EE50ED103CE00150055C44E30F2A000ECB
:106E500010220201C8510F1812E1C95110180FE198
:106E600047ECE8F0CAC2EEFFCBC2EDFF78ECE7F0EA
:106E7000CCC2EEFFCDC2EDFFCEC201F01AD0E66A61
:106E8000AEEC98F0E5520201A007000EA15B47ECC2
:106E9000E8F0EECFCAF2EDCFCBF278ECE7F0EECF30
:106EA000CCF2EDCFCDF201C0CEF20FC0C8F210C0CF
:106EB000C9F247ECE8F0EE50ED100CE109D00550B6
:106EC0004A6E4B6A78ECE7F04A50EE264B50ED22C2
:106ED0001DEC99F02E9A42ECF1F0570EE926070EC0
:106EE000EA22B9ECEAF047ECE8F0EECF4CF0EFCF55
:106EF0004DF04C504A1819E14D504B1816E142EC38
:106F0000F1F0610EE926070EEA22EECF4EF0EFCF48
:106F10004FF078ECE7F0EECF50F0EFCF51F050505B
:106F20004E1802E151504F181AE02E8A47ECE8F053
:106F3000B9ECEAF042ECF1F0570EE926070EB9EC95
:106F4000EBF078ECE7F0B9ECEAF042ECF1F0610E2E
:106F5000E926070EB9ECEBF0040E06ECECF012009B
:106F60000C0E69244A6EF00E8C144A108C6E93EC51
:106F70005EF08A9A00006950E96EEA6AD890E936B4
:106F8000EA36530EE926070EEA22EECF0FF0EDCFD8
:106F900010F0E8EC08F0E66A12EC7AF0E552000135
:106FA0001050040DF350006E060E0FC0E7FF070BE4
:106FB00004E0E742E79EE806FCE1E7500010E66ED9
:106FC00012EC7AF0E55200010F50040DF350E66E1A
:106FD00012EC7AF0E552F2EC08F06950E96EEA6AD8
:106FE000D890E936EA365D0EE926070EEA22EECFA2
:106FF0000FF0EDCF10F0E8EC08F010C0E6FF12EC57
:107000007AF0E5520FC0E6FF12EC7AF0E552010E7D
:10701000E66E12EC7AF0E552F2EC08F08A8A000093
:107020000000F00E8C161200D9CFE6FFE1CFD9FF99
:10703000010178B74BD0FE0EDB5001E0A4DEFD0E5F
:10704000DBCF8FF20C0E69244A6EF00E8C144A10BE
:107050008C6E93EC5EF08A9A0000E8EC08F0FD0E6E
:10706000DB407F0B4A6EFD0EDB50040DF3504A10DF
:10707000E66E12EC7AF0E552FD0EDB40E8403F0B85
:10708000800DF350006E0050E66E12EC7AF0E5527F
:1070900007015139F00B006EFE0EDB5003E0030ECA
:1070A000001201D000820050E66E12EC7AF0E55238
:1070B000F2EC08F0FE0EDB5002E052DF07D00000D9
:1070C00000008A8A00000000F00E8C16E552E7CF1F
:1070D000D9FF120086D8CFEC3EF02682248A120017
:1070E00053C2A3F154C2A2F155C2A1F10101A06B98
:1070F0009F6B20A402D0A9EF3AF0CDEF3AF013C273
:1071000001F014C202F015C203F069EC44F0020170
:107110001351015C06E11451025C03E11551035C5B
:1071200004E0B6EC45F096EC5EF0120084ECF4F06E
:1071300001018EA715D0FE0EDB5008E0FD0EDB50DE
:1071400005E1DF68CAA102D0010EDF6EFE0EDB5042
:1071500007E1FD0EDB5004E0010EDF6ECAB1DF680F
:10716000DF501FE0C4ECE5F0A36BA3C1A0F1A3C105
:107170009FF197ECF2F0FCECE8F002E0000E01D099
:10718000010E4A6EDF0402E0000E01D0010E4A1823
:1071900002E0DFD901D001DA9DEC04F0FAECECF06A
:1071A0003B81E552FFEFE4F00101A36BA26BA16B01
:1071B0000201B351E8244A6E640ED8ECE6F03BC0FD
:1071C000A0F1320E5CECF0F0B3C23FF0BCECFDF08D
:1071D0003FC09FF10201B4A102D0A9EF3AF0CDEF78
:1071E0003AF008AE6ED02C50400B03E02D50200B2F
:1071F00031E0800E0101BF1507E1BF510EE103012F
:10720000E3510101C05D09E2BF6BE3C3C0F1C36B91
:10721000C3C1C2F1C3C1C1F11DD0100E2C5D1AE271
:10722000360EBF5D03E3360EBF6F0DD01E0EBF5D81
:1072300011E32C0EBF5D0EE2250EBF5D02E21E0EB5
:1072400001D02C0EBF6FC36BC3C1C2F1C3C1C1F16A
:10725000C3C1C0F12C50400B03E02D50200B31E195
:10726000800E0101C41507E1C4510EE10301E35191
:107270000101C55D09E2C46BE3C3C5F1C86BC8C1B8
:10728000C7F1C8C1C6F11DD0100E615D1AE2360EFD
:10729000C45D03E3360EC46F0DD01E0EC45D11E352
:1072A0002C0EC45D0EE2250EC45D02E21E0E01D05E
:1072B0002C0EC46FC86BC8C1C7F1C8C1C6F1C8C124
:1072C000C5F118ECE9F023E2E051040B20E0BF51D6
:1072D0001D0809E2DE51200B03E0DE51400B0FE0F8
:1072E000DE8B230E08D0DE51200B03E1DE51400B74
:1072F00006E0DE9B110EE66ED2EC08F0E55274EC6F
:10730000E9F005E02C51615D02E1BFC1C4F12C50F0
:10731000400B03E02D50200B23E02150400B09E1EE
:107320001350080B06E02E50400B12E0CA51100B10
:107330000FE12150400B12E02050020B03E11350EB
:10734000040B06E12050020B09E01350080B06E085
:10735000C4ECE5F0C5DE10ECEAF002D01BECEAF07C
:107360002C50400B03E02D50200B25E12150400B09
:1073700003E01950400B09E01350080B06E02E50B3
:10738000400B09E1D5ECEAF006E12050020B11E0D8
:107390001350040B0EE0A2ECE7F0A2DE9AC1BAF1A2
:1073A0009BC1BBF19CC1BCF19DC1BDF19EC1BEF1B1
:1073B00002D026ECEAF001017851040B09E0800EBE
:1073C000081406E0100E2C5D03E20301280EE76F9F
:1073D0002050020B19E10201B451010B03E1B45139
:1073E000020B12E0050E0C5C07E02150800B0CE054
:1073F000050E0101995D08E12150400B05E0ADEC5F
:10740000E7F0D2DE10ECEAF02E50400B01E0A0D005
:107410002C50400B04E1F4ECE8F001E199D02CC1D0
:1074200000F02C50400B05E02D50200B02E161C113
:1074300000F0800E081401E18BD0100E005C01E317
:1074400087D020EC11F02DBA0DD031ECEAF0C4C198
:107450009FF1C5C1A0F1C6C1A1F1C7C1A2F1C8C1C8
:10746000A3F10CD0ADECE7F0BFC19FF1C0C1A0F11A
:10747000C1C1A1F1C2C1A2F1C3C1A3F183ECE8F083
:107480000101E951200B54E10B0E005C51E22D503B
:10749000200B03E000502C5D06E12D50200B48E14D
:1074A0000050615D45E02DAA0BD000C00FF100C077
:1074B0002CF160B70FD000C010F100C061F10AD00C
:1074C00000C010F100C061F160B704D000C00FF13E
:1074D00000C02CF12CC1CEF159EC0FF02CC1E6FF0D
:1074E000E668FCEC46F0E552E552056E010160B736
:1074F0000FD02DAA06D0050EE66E05246AECE9F041
:1075000005D0050EE66E0550BEECEAF030ECE5F075
:107510000E0E0524BDECE5F00101CD9B00BACD8B2C
:107520000A6AB3EC46F021820201010E346F1200A8
:107530002050010B03E02D50200B09E13150020BCC
:1075400007E02D50200B04E13C51100B01E0D7DD8A
:1075500012000101A3519E279E51090803E20A0E61
:107560009E5F9D2BA2519D279D51090803E20A0EA3
:107570009D5F9C2BA1519C279C51630803E2640EE4
:107580009C5F9B2BA0519B279B51630803E2640ED9
:107590009B5F9A2B9F519A2712000101A3519E5F76
:1075A0009E510A0803E20A0E9E279D07A2519D5F85
:1075B0009D510A0803E20A0E9D279C07A1519C5F7A
:1075C0009C51640803E2640E9C279B07A0519B5FBB
:1075D0009B51640803E2640E9B279A079F519A5FB0
:1075E0001200F00E8C140F098C6E93EC5EF08A9AE8
:1075F000000018C7E6FF12EC7AF0E552E8EC08F05C
:10760000F2EC08F08A8A12002D9069500701196F78
:107610001A6B170E07011927070E07011A23470EC9
:107620004A6E19C7E9FF1AC7EAFF4A50EF126950BC
:10763000EA6A2F0FE96E070EEA22EFCF33F7070150
:1076400033A105D019C7E9FF1AC7EAFFEF94070174
:1076500033A305D019C7E9FF1AC7EAFFEF92070164
:1076600033A505D019C7E9FF1AC7EAFFEF90070154
:1076700033AD05D019C7E9FF1AC7EAFFEF9C0E0E1C
:1076800069244A6EF00E8C144A108C6E93EC5EF0F6
:107690008A9A00006950EA6A170FE96E070EEA221B
:1076A000EF50E66E12EC7AF0E552E8EC08F0F2ECFE
:1076B00008F082A82D808A8A1200A6DF050E85EFC9
:1076C000E5F0FAECE4F0010178B73ED0DFECE7F04A
:1076D000EFCF33F7FE0EDB5006E1470E3CECEAF04D
:1076E000470B4A5C01E090DFFE0EDB5006E1380EEE
:1076F0003CECEAF0380B4A5C21E069500701196F55
:107700001A6B170E1927070E1A23570E4A6E2FEC05
:10771000ECF04A50EF1633A703D02FECECF0EF86D5
:1077200033A903D02FECECF0EF8E33BB03D02FEC5A
:10773000ECF0EF8AC2DF010E78ECE6F09DECF2F09F
:1077400033C7EFFFF00E8C16FFEFE4F00701040ED5
:10775000506FD89040334133423343334433453341
:1077600046334733502FF6D71200010178B7120085
:1077700042ECF1F0530EE926070EEA22EECF67F74E
:10778000EDCF68F742ECF1F05D0EE926070EEA2234
:10779000EECF69F7EDCF6AF7030E07013C156B6F6B
:1077A0006C6B020ED8903F333E333D333C33E806DA
:1077B000F9E167C74AF068C74BF0C3ECE6F0E5ECC7
:1077C000FAF03BC0EDFF3AC0EDFF39C0EDFF38C025
:1077D000EFFF69C74AF06AC74BF0C3ECE6F008EC6C
:1077E000FCF03FC0EDFF3EC0EDFF3DC0EDFF3CC0F3
:1077F000EFFF38C06DF739C06EF7020E0701D89061
:107800003C373D373E373F37E806F9E1020E0F0BB4
:10781000070105E0D89068336733E806FBE1020E04
:107820000F0B070105E0D8906A336933E806FBE1E6
:107830006BC73EF06CC73FF067C743F068C744F0C2
:10784000CBECF8F03C5007016D254A6E3D506E219F
:107850004B6E060E74ECE8F0DDECF0F069C743F017
:107860006AC744F0EDECEFF00701020E486FF10E2D
:10787000496F0301C95107E02DECE8F0D5C14AF783
:10788000D4C14BF704D051C14AF750C14BF73FC7A1
:1078900040F73EC741F73DC742F73CC743F70701F2
:1078A000476B47C746F747C745F747C744F74EDF1B
:1078B00014EC27F044C739F745C738F746C737F700
:1078C00047C736F700010F50070136270001105057
:1078D00007013723000E382339231200D4ECEFF0D0
:1078E0000050016E020E85ECE5F0D4ECEFF0005094
:1078F000026E010E85ECE5F0D4ECEFF0040EE66EBE
:1079000058ECEEF0FAECE6F009E0040E27ECEFF0AC
:107910000250E66EFAECE6F001E0010C000C84EC9B
:10792000F4F0F00E8C1669288C121C84D4ECEFF065
:1079300007013551005C15E23451005C12E322A2CC
:107940000CD02292CBDF000902E0DF2A0AD03C0EE5
:1079500085ECE5F0C3DF000903E0010EDF6E01D026
:10796000DF6A1C94F00E8C16DF50E552FFEFE4F056
:107970006950E8247F0F10240A6E0F50016E120028
:10798000FAECE4F0090EE1260F6A106A770E0F5C3C
:10799000010E105808E2ECDF0068FFEC4CF00F2AF3
:1079A000000E1022F3D7E66A92ECE9F00701336B80
:1079B000335179ECE5F002E670ECE7F001E339D100
:1079C000DFECE7F033C7EFFFC5ECEBF00C0E78EC23
:1079D000E6F01F0E3BECEFF09EECE7F033C700F053
:1079E00083EC96F01AA802D0FFEC04F068EC95F056
:1079F00033C700F0620EDE6EDD6A560E64ECE6F010
:107A0000030EDB6A400E005C63E2DC0E6AECEDF014
:107A100000502F0803E2AA0E6AECEDF0200E005C85
:107A200009E2CC0EFBECEAF00050070803E27C0E02
:107A3000FBECEAF0080E00C0DBFF800E00244A6E6B
:107A40004B6A000EB7ECEFF00A0D020EF3CFDBFF2E
:107A5000030EF4CFDBFF080EDB50006E3C0E72EC21
:107A6000E6F0090E005C03E2500E72ECE6F0005006
:107A7000180808E2210E005C05E2020EDBCFDEFFF3
:107A8000DBCFDDFF0050240803E2280E72ECE6F0A5
:107A900009ECE6F0CC0ED880EE54010EED5404E271
:107AA000CC0EDE6E010EDD6E040EDBCF4AF0050E4D
:107AB000DBCF4BF0DECF4CF0DDCF4DF04C504A5CCD
:107AC0004D504B5805E2040EDBCFDEFFDBCFDDFF70
:107AD00009ECE6F0060EEECFDBFF070EEDCFDBFF85
:107AE00077ECEAF0020EDBCF4CF0030EDBCF4DF06B
:107AF0004A504C5C4B504D5801E398D0180E07018A
:107B0000335D12E1D950060FE96EDACFEAFFDE0EDF
:107B1000D880EE54000EED5407E277ECEAF0E30E65
:107B2000DAECF3F001E27BD00A0E4A6E4B6A060EE5
:107B3000DBCF3EF0070EDBCF3FF0B0ECE5F03EC010
:107B40009AF13AC09BF10A0E01019B03F3CF9BF11E
:107B50009E6B9EC19DF19EC19CF1C3EC36F0B0ECD2
:107B600037F0060EDBCF3CF7070EDBCF3DF7070102
:107B70003E6B3F6BA00E416E860E426E010E436E51
:107B8000446A3CC73CF03DC73DF03EC73EF03FC7AE
:107B90003FF0E5ECFAF038C03CF739C03DF73AC0A9
:107BA0003EF73BC03FF7E1DDA4EC36F0040E78EC85
:107BB000E6F00701C80E356F250E346F77ECEAF05A
:107BC000620EDAECF3F002E21C0E346F1AA803D056
:107BD000060E355F34272282A2DE00091BE0060E66
:107BE000DBCF0FF0070EDBCF10F071ECEDF033C7F9
:107BF00000F0FFEC4CF0D950060FE96EDACFEAFF47
:107C0000CC0EEE180CE1010EED1809E1012AFFEC93
:107C10004CF005D007013451D880005407E2060E1D
:107C2000DB06070E01E35CD7DB065AD70701332BCF
:107C3000BFD60C0E346FDD0E356F760E0F6E010E53
:107C4000106E040E7DECE6F023E292DE3EEC4DF089
:107C5000A1EC98F0FF0E005C07E1420E9CECE5F011
:107C60000FC029F710C02AF7450E0F180DE110506C
:107C70000BE1280E005C03E300502A0805E2450EE4
:107C80009CECE5F000C02BF70F06000E105AD9D778
:107C9000D0EC10F00201800E8A6F6AEC38F0090E09
:107CA000E15C02E2E16AE552E16EFFEFE4F0B6C1A9
:107CB00001F0B7C102F00101000E0D6F0D0E0E6F45
:107CC0000A01D751040DF3500C10036EBDEC0CF0FB
:107CD000066E0C5004E1DDECEAF001E00686030ECE
:107CE0000C5C04E17850080DF350061212000A01F2
:107CF000040EDE6FDF69695005E10C50030802E3F2
:107D0000E05101E1000CD3DF0A01DF6BE051DF5DE0
:107D100030E24DECF0F0EF50015C23E10101E7ECC3
:107D2000E6F0EF50025C1AE1E7ECE6F0EF50035C9E
:107D300012E1E7ECE6F0EF50006E1F0E0014065C57
:107D400007E10050E00BE838E8400A01DE6F010C63
:107D50000D07000E0E5B0D07000E0E5B0D07000EEB
:107D60000E5B040E01010D27000E0E230A01DF2B0E
:107D7000CDD7DF69000C0301C95107E02DECE8F015
:107D8000D4C120F1D5C121F104D050C120F151C19D
:107D900021F10101F10E226F020E236F120070EC2F
:107DA000EFF034BC39D02CBC1AD0696A38D82550D1
:107DB000100B04E10101E351400B0CE0800E0814AC
:107DC00003E03050800B03E01950400B03E0010E3C
:107DD000696E25D8309E21BC20D0199C1ED02DAABA
:107DE00008D02150400B03E02050020B16E1696AD5
:107DF00013D02150400B09E174ECE9F003E1E351A9
:107E0000400B03E0010E696E0AD82150400B05E0DB
:107E10002050020B02E0696A02D878EFEFF070ECB4
:107E2000EFF00101080E9A6F150E9B6FF40E0F6EA6
:107E3000010E106E2150400B06E0A8ECE6F003E0C6
:107E4000B0C201F003D0BDEC0CF0016E0150E66E43
:107E50006CECEAF04A6E4B6A4ABE4B684A5000012D
:107E600003ECEFF09FEC04F001019C6F3AC09DF130
:107E70009E6BA36BA3C1A2F1A3C1A1F1A3C1A0F109
:107E8000A3C19FF12150400B04E0A8ECE6F001E112
:107E9000FAD0695017E03450400B14E10CC05DF289
:107EA000CBC15EF2D7CA5FF25BC261F25CC262F222
:107EB0007D500C6ED7C1CBF160C2D7FA63C25BF2C2
:107EC00064C25CF20C5005E0030E0C5C30E17850AB
:107ED0002EE0FBECEEF05BC23EF05CC23FF0B0EC9B
:107EE000E5F03EC0A1F1A1ECE5F03AC03FF0BCECFA
:107EF000FDF03FC0A2F15BC24AF05CC24BF00A0E3B
:107F0000A4ECF2F04AC0A3F11FEC12F0000903E167
:107F1000CDEC3AF002D0A9EC3AF081ECE7F023E0A6
:107F200077ECEDF01FEC12F0000918E01AD0040E07
:107F30000C5C19E296EC04F001010F0EA16F45EC08
:107F4000F1F0780E4A1804E14B5002E1100EA1271F
:107F50000C0404E06AEC11F0010803E1CDEC3AF006
:107F600002D0A9EC3AF069500EE1C1DE000902E04E
:107F70001C8A03D01CAA07D01C9A6DEC1AF0E66A82
:107F800060EC4BF0E552E5ECEAF005E11C50200B0B
:107F90003FE069503DE1D751DE25FC0FE16F190E3E
:107FA000E15D056E190EE15D04E2190ED880E15520
:107FB000056E0701EFAF07D0A1ECE5F005C03FF07B
:107FC00070ECEAF00AD00550FE0BE8420101A16F07
:107FD000A26B05A002D0050EA26F0C040BE00C50A2
:107FE00003E1DDECEAF006E0030E0C5C08E11BECBB
:107FF000EFF005E10A01E151190808E304D00A0194
:10800000E151190803E2A9EC3AF002D0CDEC3AF0C4
:10801000695023E034BC0AD05DC20CF05EC2CBF1E3
:108020005FC2D7FA61C25BF262C25CF20101E39700
:108030000201D55101019B5D0FE10201D651010101
:108040009C5D0AE10201D75101019D5D05E102013C
:10805000D85101019E5D01E0E387695045E10201CD
:10806000295106E0D65101019C5D02E005013B85E6
:108070009AC1D4F29BC1D5F29CC1D6F29DC1D7F270
:108080009EC1D8F231D0FCEC26F0016E6AEC11F002
:10809000026E010405E0020E015C02E0025014E0F1
:1080A000025002E00250016E01010F0EA16F07ECB9
:1080B000EFF003E0100E0101A12735AC02D097ECE0
:1080C000F2F001040CE00ED0030E015C0DE181EC36
:1080D000E7F002E077ECEDF01BECEFF003E1CDEC24
:1080E0003AF002D0A9EC3AF02CC100F0695005E05A
:1080F0003450400B02E161C100F000500A0801E376
:10810000A8D0100E005C3DECE8F074ECF4F001E156
:1081100085D0EAECF4F001E181D02DDEA00E010162
:10812000205D7A0E2159F10E2259020E235918E2D0
:10813000A00E4E6E7A0E4F6EF10E506E020E516E04
:1081400020514E5C4A6E21514F584B6E225150586F
:10815000235151584AC0D2F14BC0D3F1006A15D017
:1081600020C14AF021C14BF022C14CF023C14DF097
:10817000A00E4A5E7A0E4B5AF10E4C5A020E4D5A20
:108180004AC0D2F14BC0D3F10068590E0F6E020EF7
:10819000106EDEAB04D0640E0F6E020E106E0FC0B8
:1081A0004EF010C04FF0506A516A53ECEEF04C6A3A
:1081B0004D6A5CECF1F04EC041F04FC042F050C04F
:1081C00043F051C044F0E5ECFAF038C020F139C07A
:1081D00021F13AC022F13BC023F1010121C120F17C
:1081E00022C121F123C122F1236BC0EC96F00101E1
:1081F000A06BA0C19FF104C13CF504C1A1F10539F8
:108200000F0B05013D6F0101A26F0F0E0515050152
:108210003E6F0101A36F00C03FF514D087EC08F05A
:108220000101A06BA0C19FF123ECF3F0A16F050E3B
:10823000EB50A26FA36B006AEF50010B01E00068E6
:1082400087EC08F0005003E0CDEC3AF002D0A9EC46
:108250003AF09AC19FF19BC1A0F19CC1A1F19DC1CF
:10826000A2F19EC1A3F1695007E12050020B0AE080
:108270002150400B0AE106D03450400B03E1F4ECEE
:10828000E8F003E0ADECE7F002D031ECEAF00101F8
:10829000DE51200B07E0695003E02C51615D02E1E3
:1082A000020E9A5FE3BD27D01A9E695004E02E505B
:1082B000400B01E11A8EFCECE8F003E0A9EC3AF087
:1082C00002D0CDEC3AF0695016E001013851080BAC
:1082D00012E03C51100B0FE10A0E9A6F330E9B6FA8
:1082E0001E0E9C6F9E6B9EC19DF178A704D0050E5B
:1082F0009A6F370E9B6F01017851080B2CE02150CB
:10830000400B29E1016A3851080B0BE03C51100B7E
:1083100008E08B51400B05E0E351080B02E1020E2F
:10832000016E696A430E65ECE9F0010E016E74ECB2
:10833000E9F003E1E351400B07E08B51400B03E010
:10834000E351080B01E0016A010E696E430E65EC12
:10835000E9F0DF50696E010178A71DD09AC1E6FFF0
:108360006AECE8F0016E9BC1E6FF6AECE8F0026E91
:108370009CC1E6FF6AECE8F0036E0A0E01019D0362
:10838000F3509E25E66E6AECE8F00101076F460E99
:10839000E66ED5D8D0D09B514A6E4B6A0A0ECDEC12
:1083A000F4F001019A510A0DD1ECE7F0010E0F260D
:1083B000000E102271ECEDF03EEC4DF00A6A270E33
:1083C000005C06E1460E0F1803E1105001E1002A9F
:1083D000DFECE7F0EF50005C0AE02A50040B07E105
:1083E000040E06ECECF0DFECE7F000C0EFFF2A949F
:1083F000C3EC36F02EAA09D008AE03D0B0EC37F0AB
:1084000004D0E6C2E6FFE6ECE7F09AC14AF04B6A18
:108410004C6A4D6A400E416E420E426E0F0E436E24
:1084200085ECE7F09BC14EF04F6A506A516A100E1E
:10843000416E270E426E436A446A4EC03CF04FC004
:108440003DF050C03EF051C03FF0E5ECFAF038C0CE
:108450004EF039C04FF03AC050F03BC051F050ECF4
:10846000EBF09CC152F0536A546A556A640E416E37
:10847000426A436A446A52C03CF053C03DF054C063
:108480003EF055C03FF0E5ECFAF038C052F039C08C
:1084900053F03AC054F03BC055F052504A26535066
:1084A0004B2254504C2255504D229DC156F0576AD4
:1084B000586A596A0A0E416E426A436A446A56C053
:1084C0003CF057C03DF058C03EF059C03FF0E5ECDD
:1084D000FAF038C056F039C057F03AC058F03BC0F7
:1084E00059F056504A2657504B2258504C2259505A
:1084F0004D229EC15AF05B6A5C6A5D6A4A505A24FA
:1085000007013C6F4B505B203D6F4C505C203E6F31
:108510004D505D203F6FB5EC3BF0A4EC36F002010E
:108520008A5139ECECF008E14B5006E125BC04D04F
:10853000E66A61EC3BF0E552E552FFEFE4F0D9CF9B
:10854000E6FFE1CFD9FF02010D6B23EC7AF00101C8
:1085500001018E51010B07E001010101E351040B00
:1085600002E1300EC66E0C0E69244A6EF00E8C14B9
:108570004A108C6E93EC5EF08A9AE8EC08F0FE0EDE
:10858000DBCFE6FF12EC7AF0E552FE0EDB50006E18
:10859000FE0EDB50530807E00150E66E12EC7AF055
:1085A000E55201500026FE0EDB50460804E0FE0EA8
:1085B000DB50560815E10250E66E12EC7AF0E552F7
:1085C0000350E66E12EC7AF0E55207C1E6FF12ECBA
:1085D0007AF0E55200500224032401010725006EC1
:1085E000FF0E0002F350E66E12EC7AF0E552FE0E3A
:1085F000DB50530806E1C950006EE66A12EC7AF0CF
:10860000E5528C880000000000000000310EC66EAC
:108610008A8AF00E8C161FEC7AF0E552E7CFD9FF6C
:108620001200D9CFE6FFE1CFD9FFB5C19AF1B6C1AB
:108630009BF1B7C19CF1B8C19DF1B9C19EF1010197
:10864000A46BFE0EDB500A0807E22A96FE0EDBCF73
:10865000E6FFC7EC34F0E5520101006B800E01012A
:108660001615036E800E01011315026E010EEA6EDF
:108670009A5105D89B5103D89C5101D814D0076B4F
:10868000066F0A0E065DD8A003D0066F072BF9D738
:108690000051110FE96E0751EF6EE92A0651EF6E96
:1086A000002B002B000C04D8E552E7CFD9FF1200B5
:1086B0009DC117F19EC118F10101A45105E10A0EF7
:1086C0009A5D02E2100E116F0701EFBB03D00101AA
:1086D000100E186F0701EFAD05D00101100E176FD6
:1086E00017C118F11EBC03D00101138F03D0025033
:1086F0000101131361EC0BF0000903E10101168F76
:1087000003D0035001011613A45109081AE2020113
:10871000495117E0A2EC93F00101020E006F9AC1DB
:1087200000F083EC96F0A4C100F00101006B83EC33
:1087300096F0010EE66EE66A84EC09F0E552E55229
:1087400012000101A45118E00701EF51200B14E1C0
:10875000298C17C118F116C117F115C116F114C1F2
:1087600015F113C114F112C113F111C112F1ABECE7
:10877000F2F03BC011F11200299C1200D9CFE6FFA4
:10878000E1CFD9FF020EE126010EA4C1DBFF2EAC22
:108790000FD02CC1DFFFEFC7F0F7B5C19AF1B6C11A
:1087A0009BF1B7C19CF1B8C19DF1B9C19EF114D044
:1087B00061C1DFFF7D50EA6AE90FE96E070EEA2228
:1087C000EFCFF0F7BAC19AF1BBC19BF1BCC19CF1EC
:1087D000BDC19DF1BEC19EF10101A46BDF500A082D
:1087E00006E22A96DFCFE6FFC7EC34F0E55201013E
:1087F000016B800E01011E15026E010EEA6E9A5188
:1088000005D89B5103D89C5101D816D0076B066F31
:108810000A0E065DD8A003D0066F072BF9D70151C9
:10882000190FE96E0751300FEF6EE92A0651300F2C
:10883000EF6E012B012B000C010EDBCFE6FF0BD8F6
:10884000E552020EE15C02E2E16AE552E16EE552B8
:10885000E7CFD9FF1200FAECE4F0300E01019D25BC
:108860001F6FA45105E10A0E9A5D02E2200E196FF6
:108870000701F0AD03D00101200E1F6F01011B8F16
:108880006FEC0BF0000903E101011E8F03D00250D1
:1088900001011E13A45116E00701F051200B12E153
:1088A0001EC11FF11DC11EF11CC11DF11BC11CF118
:1088B0001AC11BF119C11AF1ABECF2F03B50300FA9
:1088C0000101196FA4C1A5F1FE0EDBCFA4F1FFEFEA
:1088D000E4F0E66A08D8E55231A204D0010EE66E53
:1088E00002D8E5521200FAECE4F0050EE126FE0E85
:1088F000DB500CE1BFC1DFFF010EC0C1DBFF049004
:1089000020B00480040E2CC1DBFF0ED0C4C1DFFFF9
:10891000010EC5C1DBFF049031B20480030E15C205
:10892000DBFF040E61C1DBFF020EDB6A0450010BAA
:1089300001E104D11C0EDF5C01E300D1100EF36EE7
:10894000040EDBCFF4FFF350F45C01E3F7D00E0E1E
:10895000DF5C01E383D0070EDF5C48E2030EDF5CDF
:1089600016E2020EDF5C0DE2DF5005E0460E36EC4B
:10897000E5F001E3E3D0800E64ECE6F00201400E86
:10898000BCD0010EDB500A0801E3D8D00BD0050E95
:10899000DF5C15E2030EDF5C0BE11E0E36ECE5F04A
:1089A00001E3CCD0C00E64ECE6F00201800EA5D04D
:1089B000010EDB50140801E3C1D0100E23D00201D8
:1089C000080E156F050EDF5C0AE1190E36ECE5F0B6
:1089D0000BE3010EDB50320801E3B0D005D05A0E94
:1089E00036ECE5F001E3AAD0100EA6D0090EDF5C4C
:1089F00016E2070EDF5C09E1010EDB50280801E3F7
:108A00009DD0300E64ECE6F007D0300E64ECE6F05A
:108A1000280E36ECE5F032E20201080E6ED00201BB
:108A2000200E156F090EDF5C07E1550E36ECE5F000
:108A300001E384D0300E80D00D0EDF5C09E20A0E17
:108A4000DF5C0AE1010EDB50140801E377D004D0AB
:108A50003C0E36ECE5F072E2080E6ED0160EDF5CCE
:108A600037E2120EDF5C18E20E0EDF5C0AE1010E47
:108A7000DB503C0863E20C0E64ECE6F00201200ED1
:108A80003CD0110EDF5C04E3460E36ECE5F056E216
:108A90000C0E64ECE6F029D00201100E156F120ED8
:108AA000DF5C05E1010EDB50280848E20FD0130E11
:108AB000DF5C0CE0140EDF5C05E15A0E36ECE5F0ED
:108AC0003DE204D0010EDB50320838E2010E34D012
:108AD000180EDF5C14E2160EDF5C0AE1010E64EC96
:108AE000E6F00A0E36ECE5F006E20201100E05D0C3
:108AF000030E64ECE6F00201040E156F1FD00201B4
:108B0000040E156F180EDF5C05E1320E36ECE5F051
:108B100015E20BD0190EDF5C05E1010EDB503208C7
:108B20000DE203D01A0EDF5C02E1030E05D0460E03
:108B300036ECE5F003E2030E64ECE6F0FE0EDB50EB
:108B4000EA6A130FE96E020EEA22020EDBCFEFFF94
:108B5000FE0EDB5003E0030EDBCF15F2050EE15CE9
:108B600002E2E16AE552E16EFFEFE4F007010A6B11
:108B70001F0E0B17116B0D6B0DC70CF7030E0617AD
:108B80001F0E0717096B09C708F72CC100F018EC76
:108B9000E9F002E20FC100F00201135103E020509E
:108BA000010B47E100500A0A3FE0030A39E0010ADD
:108BB00035E00F0A2DE0010A27E0030A20E0010A50
:108BC0001BE0060A14E0010A0FE0020A08E0010AAD
:108BD00036E10701118D11830A890B8B30D0070113
:108BE000118F11830A892BD007010B8D02D0070149
:108BF000118311870A8B23D007010B8D1183070185
:108C00001183118B0A8D1BD007011189118304D0A8
:108C10000701118311890B8F0A8F11D007010B8F68
:108C2000070111850A870BD00701118311850A8579
:108C300006D0E66A01EC15F0E55215C211F72CC119
:108C400000F000500A0802E20FC100F0010160A725
:108C500007D061C100F000500A0802E210C100F024
:108C60000201145103E03150020B35E100500A0AB1
:108C70002FE0030A2AE0010A26E00E0A21E0010A99
:108C80001DE0020A18E0010A14E0060A0FE0010ADA
:108C90000BE0020A06E0010A23E107010689078BBF
:108CA0001FD0070106891CD00701078D0701068B1D
:108CB00017D00701078D0701068D12D00701078F16
:108CC0000701068F0DD00701078F0701068708D01F
:108CD0000701068505D0010EE66E01EC15F0E552A0
:108CE00001013CB905D0FC0E07010613E00E071385
:108CF00005EF0CF032EC0EF02C50040B08E00050A5
:108D00002FECE6F0EF50020B02E125EC0EF0258A85
:108D1000120065ECEFF0830E0A6E0A0EE66E01019A
:108D20000F03F350E66E740EE66E020E30ECE5F0C3
:108D3000DE0EBDECE5F00050DF6EFE0E7CECF4F0D4
:108D40000101DF9D2F9EB90E005C05E1FF0E0201BF
:108D5000745D01E02F8EA30EDF5C02E10101DF8D67
:108D6000E552FFEFE4F070ECEFF0695034E1195098
:108D7000010B31E1CEDF01015751080B03E12C510A
:108D800009080EE228EC05F0FF0805E1800EE66E0A
:108D90003AEC05F0E55228EC05F00101496F08D0E6
:108DA000FF0E8D5D03E1320E8D6F02D08DC149F152
:108DB0005DECF3F02B847FEC28F038EC23F02CA64C
:108DC0000AD0E66AEBECC6F0E5520701169F12B036
:108DD000168FACECC5F02BECECF025A808D038ECE5
:108DE0000DF025A804D0010E696ED0EC10F0696A70
:108DF000D0EC10F078EFEFF065ECEFF0FD0EDB500B
:108E0000100DF350DF6E010E0A6E0201680EC26F84
:108E1000FD0EDB500A080AE2020E0A6E690EC26FEE
:108E2000FD0EDB50F00F100DF350DF6E3EECEFF057
:108E300002E012ECF1F0DF50E552FFEFE4F0020146
:108E4000B25103E0B251330802E20D0EB26FB351DA
:108E5000F6ECE5F005E24CECE8F002E21E0EB36F32
:108E6000B4BFB46B120069ECEFF03EECEFF01BE026
:108E700012ECF1F00F0E89ECF0F00A0E005C07E145
:108E80000101DD51010B03E00A6A000E5DD200C052
:108E90002CF101018B51100B06E00A0E6EECE5F08F
:108EA00002E2FE0EDB682CC10FF10101E0A506D045
:108EB000DE9B450EE66ED2EC08F0E55202018B6BAC
:108EC0000101E09532EC0EF018ECE9F022E2100E10
:108ED0002C5D61ECF3F079EC05F052ECF0F011E070
:108EE000E2ECF0F001010F6FEF380F0B02018B6F16
:108EF000CFECE5F0800B03E00101E085DE8DFADECA
:108F000008D0FE0EDB680101090E0F6F0FC12CF1B6
:108F1000268EF4ECEFF0100E4FECF1F00F0E010185
:108F2000C9150C6EC9390F0B7D6E7D50060802E223
:108F30000C507D6E0C0401E1CA91020E0C5C01E143
:108F4000CA81CFECF3F0786E60B704D02CC161F128
:108F50000FC110F161C110F161510A0817E2100E42
:108F6000615D61ECF3F052ECF0F005E0E2ECF0F062
:108F70000101106F08D0FE0EDB680101090E106FB1
:108F800010C161F1268E61C100F002D059ECEBF006
:108F900000500101615D03E12C51615D0FE09CEC2B
:108FA000F1F0050EE66EDF246AECE9F030ECE5F056
:108FB0000A0E89ECF0F000380F0B7D6E040E95EC74
:108FC000EEF0D60EE66E010E30ECE5F0F4ECEFF0CC
:108FD0003EECEFF003E1C2C20AF002D0100EDF2631
:108FE000100E80ECF4F020ECF2F03EECEFF05CE0E0
:108FF0002CC1E6FFE668BAECE6F00B0E89ECF0F067
:10900000030E0C5C09E01F0E0101CA17E00E0014EC
:10901000CA13CFECF3F0786E0050046E0101CA97CA
:109020000450080B01E0CA870C0E89ECF0F0440EE6
:109030000101CB17BB0E0014CB1342ECEFF0070E6F
:109040000101CC17F80E0014CC1342ECEFF00A0E1D
:109050000101CD17F50E0014CD13C2C20AF00D0E9A
:10906000E66E030EDF24E66EB50EE66E020E30EC01
:10907000E5F09CECF1F00C0E89ECF0F0440E0101EF
:10908000D717BB0E0014D71342ECEFF0070E010107
:10909000D817F80E0014D81342ECEFF00A0E0101B5
:1090A000D917F50E0014D9130201BBBFBB6B0A6AB6
:1090B000BFC107F5C0C108F5C1C109F5C2C10AF5B4
:1090C000C3C10BF5C4C10CF5C5C10DF5C6C10EF584
:1090D000C7C10FF5C8C110F519B42DD0139413965C
:1090E000139A209201013951020B1CE0A8ECE6F022
:1090F00019E10101CC51010B04E01CECB9F00009AD
:1091000011E10101CC51010B05E02C51615D02E13F
:10911000138A20821396CCB313861394CCA509D05E
:10912000138407D028ECEDF00101D895D893CC95A5
:10913000CC9327ECC0F018ECE9F01AE2680E0F258A
:109140005FECF2F000500101BF5D016E01AE03D093
:10915000BF51005C016E015003080AE2050E45ECA8
:10916000EFF0BF0EE66E010EF1ECE5F000C0BFF1CE
:10917000010161510A081AE2680E10255FECF2F055
:1091800000500101C45D026E02AE03D0C451005C08
:10919000026E025003080AE2050E45ECEFF0C40E21
:1091A000E66E010EF1ECE5F000C0C4F1320E73EC96
:1091B000E7F0300E73ECE7F027ECECF0B4EC2CF0B9
:1091C00053EC0EF0139C01013CB1138C139E3CB385
:1091D000138E83EC7FF0139801013CB913882CA403
:1091E000CC9F1294CCBF12840701109B12A4108B49
:1091F0000201BC51030802E3BC5102E1020EBC6F44
:109200004FEC27F02CB602D00101CB9F1290010148
:10921000CBBF12801292CBAF1282B8EC09F00101E1
:109220005851800B05E02C50040B02E025EC0EF0A9
:10923000660E0A6E080E01012C03F328BDECE5F062
:1092400000C042F5FF0E005C02E10501426B010621
:109250003EEC4DF0FF0E005C01E1006A7F0E001451
:109260000501406F01015851100B04E1DD51200B45
:1092700001E1CB9B080E6103F350050FBDECE5F057
:1092800000C043F5FF0E005C02E10501436B0106DF
:109290003EEC4DF0FF0E005C01E1006A7F0E001411
:1092A0000501416F01015851100B0AE1DD51200BFE
:1092B00007E16051080B03E01C50080B01E0D99155
:1092C0000A6A010E69CFDBFF3CA905D0696EFAEC92
:1092D00068F094EC68F0696AFAEC68F094EC68F075
:1092E00015A403D00501FA0E446F010EDB50696E20
:1092F0006A0E01010F250A6EF00EBDECE5F0FF0EBF
:10930000005C01E1006A00C0E0FA040E0002F350C4
:10931000E66EE66A000EE66E0D0E30ECE5F00A6AC7
:1093200022DDACEC0CF01BECEAF026ECEAF0796AFA
:109330001EBC09D00701D36B030E016E2CC100F0D7
:109340005EDB7EECEDF0010EE1ECEAF002E2E16AB8
:10935000E552E16E4A50FFEFE4F065ECEFF00B0EE2
:1093600001012C5D0BE2C0C1E6FFBFC1E6FF65EC69
:10937000F3F0005001012C5D01E0B7D00B0E615DF0
:1093800007E259ECEBF000500101615D01E0ADD066
:109390000A0E2C5D02E249C18DF1F4ECEFF03CECD9
:1093A00027F00101CB9F12B0CB8FCC9F12B4CC8F92
:1093B00039A30DD0F80ECC17CC9120B2CC81CC9330
:1093C00013B6CC83CC9513B4CC8584EC55F02CC16A
:1093D000CEF11BECF1F0050EBEECEAF080ECF4F0FF
:1093E0005AECE5F00A0EDF24016E7D38F00B0C100C
:1093F00000ECE9F0050EE66ECA0EE66E010E95EC85
:10940000EEF05AECE5F0CDECE9F01BE09CECF1F06D
:109410000A0E89ECF0F00F0E00160A0EDF24016E22
:109420007D38F00B001000ECE9F0CDECE9F009E03C
:10943000040EE66ED60EE66E010E95ECEEF05AECDA
:10944000E5F0050E6AECE9F0E66E050EDF2456EC59
:10945000F0F01DBA45D0F4ECEFF001015751080BC4
:1094600003E12C51090805E249C1E6FF3AEC05F099
:10947000E55208ECC5F00101CB51800B01E0010E73
:10948000A1ECEBF03BC1EFFF3EECEFF003E1C2C219
:109490000AF002D0100EDF2684ECEDF0DFCFE6FFFD
:1094A0005AECE5F00A6ABEEC15F0660E0A6E080E7C
:1094B00001012C03F350016E40C500F0A0DA012A2F
:1094C00042C500F09CDA080E01016103F350040F5D
:1094D000016E41C500F093DA012A43C500F08FDA2E
:1094E0000A6A7EECEDF00201306BE552FFEFE4F02A
:1094F00065ECEFF0FE0EDF6E5FECE8F008E02D505B
:10950000400B05E12D50800B02E17F0EDF6EF00E67
:1095100006010D17DF1C0E17E552FFEFE4F0060100
:109520000D9F0E910F971097770E12171397149F98
:1095300012002AECF4F0DBCFE6FF10EC14F0E55259
:10954000E71803E006010D8102D006010D83010139
:109550003DA502D006010E8F01018BA102D00601AC
:109560000E89FFEFE4F01A9E0050050A01E173D066
:10957000010A5BE0070A2AE0010A23E0030A1FE070
:10958000010A01E0120006010D85FCECE8F002E0A2
:10959000000E01D0010E4A6EDDECEAF001E0010E92
:1095A0004A1802E006010D870601F051010801E2A8
:1095B0000E8D01018FAD63D006010E891200E66A9F
:1095C00002D0010EE66EB5DFE552120006010E87ED
:1095D000FCECE8F002E0000E01D0010E05ECEBF02F
:1095E00002E006010D87785003E0030E785C02E18B
:1095F00006010D772BECEFF002E006010E8D33A093
:109600000ED0FCECE8F002E0000E01D0010E05ECFB
:10961000EBF003E006010D8302D006010D8101018C
:109620003DA72DD006010E8F120006010E85010107
:10963000CDA725D0CDA303D006010D8302D006010E
:109640000D8101018F51080B03E10201515117E017
:1096500006010E8D120006010E830201B451040BA7
:1096600004E04D5102E106010E8D0201B4A102D0C9
:1096700006010E890201B4A302D006010E8B12006E
:10968000800E081405E02150010B02E10C5002D0BD
:10969000FCEC26F0006E2CDFB3EF4AF006015051CF
:1096A0000A01DA91040B01E0DA81B4ECE5F007E09D
:1096B0000601525101015799800B01E057891200B0
:1096C000FAECE4F00C50006EFCEC26F0056E6AEC4F
:1096D00011F0046E045006E00450006E21BE02D06A
:1096E0000450056E1B0E00248FECE5F0016E210E78
:1096F00005248FECE5F0026E005005E1DDECEAF0A8
:1097000002E0220E016E055005E1DDECEAF002E018
:10971000420E026E030E005C09E1045007E11BECEF
:10972000EFF004E0200E016E400E026E015012ECCC
:10973000E5F0695006E1FE0EDB5003E0025012EC4A
:10974000E5F0040E005C0DE10101CDA707D0CD517D
:10975000020B02E0270E03D0280E01D0240E12ECDB
:10976000E5F0FFEFE4F065ECEFF034B886D0695037
:1097700002E1B8EC11F00A01DA5106015099010B2F
:1097800001E050890A01DA5106015095010B01E010
:1097900050850A01DA510601010B02E0509B01D00D
:1097A000508B0A01DA510601010B02E0509701D0FB
:1097B0005087F6ECF0F006E10601508D528F529181
:1097C000509F21D0030E005C0EE10601508D509F8A
:1097D00093EC11F0000903E00601509D508F060143
:1097E000528F529110D00601509D508F529F01010F
:1097F00057A902D00601528F06015291010157B9B3
:1098000002D0060152812150800B14E11550100B3B
:1098100011E01550200B0EE10C5009E0030E0C5C1A
:1098200006E0050E0C5C03E05FECE8F003E0159841
:10983000C1EC6AF0030E0C5C03E0050E0C5C02E167
:1098400073EC68F014900C5004E1149001018BB596
:109850001480030E0C5C04E1149001018FB5148098
:10986000149A14A0148A54EC0DF0695004E183ECAE
:109870007FF0E4EC1DF0B4EC2CF03450100B18E148
:1098800001018F51400B14E02150800B11E1695010
:109890000FE1FCEC26F0010804E0FCEC26F00208E5
:1098A00007E10C50DF6E0C6A0EEC1AF0DF500C6E04
:1098B000FAEC1AF02682CFEC3EF0010EE66E00DFE5
:1098C000E55221EC1BF0B2EC23F034B848D0FDECAB
:1098D0001DF0C1EC6AF0EFEC11F049EC26F01D9898
:1098E00035900101E2BB02D025EC09F0050E0C5CBD
:1098F00003E0050E7D5C02E18DEC0CF017EC25F029
:1099000069502DE1B9EC25F0DCEC22F020EC1EF0E2
:10991000D5EC16F0B4ECE5F002E0C3EC23F0B3ECC8
:1099200016F034A402D055EC1EF097ECE7F056C1C7
:10993000E6FFE66A6AECF3F0016E01016081005017
:1099400006E0030E005C04E17850010801E260913A
:10995000F5EC13F0050E005C02E14AEC09F03498D6
:10996000E552FFEFE4F08E9400000000030EE66E77
:1099700012EC7AF0E552040E0A5CE66E12EC7AF014
:10998000E5520150E66E12EC7AF0E55234ECFDF04F
:10999000006E00008E841200D9CFE6FFE1CFD9FF20
:1099A0008E9400000000060EE66E12EC7AF0E5528E
:1099B0008E840000000000008E9400000000020E63
:1099C000E66E12EC7AF0E552040E0A5CE66E12ECDA
:1099D0007AF0E5520150E66E12EC7AF0E552FE0E96
:1099E000DBCFE6FF12EC7AF0E5528E84040EE66ED1
:1099F00006ECFDF0E552E552E7CFD9FF120069EC25
:109A0000EFF00050DF6E010EDB6A38D8DF50005CEB
:109A10002DE0040E0A5C16E2F29EA1980A50AA6E8E
:109A20000150A96EDF50A86EA69EA69CA684550E76
:109A3000A76EAA0EA76EA682F28E040E78ECE6F050
:109A4000A69414D08D8A010EDB2ADFCFE6FFA4DFB7
:109A5000E55289DFDF50005C02E040EC0EF0DF50A1
:109A6000005C04E0050E36ECE5F0EDE3020EE15C8F
:109A700002E2E16AE552E16EFFEFE4F0DAECF1F0C8
:109A8000040E0A5C0AE20A50AA6E0150A96EA69E54
:109A9000A69CA680A850006E13D08D8A010EDB2AEA
:109AA00062DF0050DF6E5FDF0050DF5C02E040EC01
:109AB0000EF00050DF5C04E0050E36ECE5F0EEE35E
:109AC000020EE15C02E2E16AE552E16EFFEFE4F0D2
:109AD000FAECE4F08BECEDF011E0FC0E1FECEEF094
:109AE000BDECE5F0FD0EDBCFE9FFDB2AFE0EDBCFA0
:109AF000EAFF01E3DB2A00C0EFFFECD7FFEFE4F061
:109B0000FAECE4F08BECEDF011E0FE0E1FECEEF061
:109B1000016EFC0EDBCFE9FFDB2AFD0EDBCFEAFF97
:109B200001E3DB2AEF5000ECE9F0ECD7FFEFE4F0C3
:109B3000D9CFE6FFE1CFD9FFE6528E848D9A00009F
:109B40000000060EE66E12EC7AF0E5528D8A0000F7
:109B5000000000008D9A00000000D80EE66E12ECA6
:109B60007AF0E552D7C7E6FF12EC7AF0E552E66AE2
:109B700012EC7AF0E552E66A12EC7AF0E5528D8A40
:109B8000DF6A1E0EDF5C07E2640EE66E35EC29F03C
:109B9000E552DF2AF6D7E552E552E7CFD9FF1200AA
:109BA000D9CFE6FFE1CFD9FF35AE33D08E848D9A81
:109BB00000000000030EE66E12EC7AF0E552D7C703
:109BC000E6FF12EC7AF0E552FC0EDBCFE6FF12EC7A
:109BD0007AF0E552FB0EDBCFE6FF12EC7AF0E552AD
:109BE000FA0EDBCFF3FFDB06F35000090FE034EC95
:109BF000FDF0006EFD0EDBCFE9FFDB2AFE0EDBCFB2
:109C0000EAFF01E3DB2A00C0EFFFEAD700008D8AFC
:109C1000C69EE552E7CFD9FF120069ECEFF0DF6A8C
:109C20000101E99BDF2AFA0EDBCFE6FF53ECF4F0EB
:109C30007EECEAF0FA0EDBCFE6FFF3ECE6F0AC0EDA
:109C4000E66E030EE66E7EECEAF0010EDB6AFA0EBB
:109C5000DB5036ECE5F017E2010EDB50E76E99ECD5
:109C6000E8F0E7502DECF0F0EFCF4AF0010EDB50BA
:109C7000EA6AAC0FE96E030EEA22EF504A5C03E198
:109C8000010EDB2AE4D792ECEDF002E040EC0EF09E
:109C900092ECEDF003E0140EDF5CC4E3140EDF5C25
:109CA00002E2010E03D00101E98B000EE1ECEAF0C3
:109CB00002E2E16AE552E16E4A50FFEFE4F0D9CFEB
:109CC000E6FFE1CFD9FF35AE46D08E848D9A0000F5
:109CD0000000060EE66E12EC7AF0E5528D8A000066
:109CE000000000008D9A00000000020EE66E12ECEB
:109CF0007AF0E552D7C7E6FF12EC7AF0E552FE0E95
:109D0000DBCFE6FF12EC7AF0E552FD0EDBCFE6FF8B
:109D100012EC7AF0E552FA0EDBCFF3FFDB06F350DC
:109D2000000911E0FB0EDBCFE9FFDB2AFC0EDBCFE5
:109D3000EAFF01E3DB2AEF50006E0050E66E12EC02
:109D40007AF0E552E8D700008D8AC69E050EE66ED1
:109D500035EC29F0E552E552E7CFD9FF12000701B3
:109D6000D76B020EE66EE66AE668D20EE66E010E6C
:109D700001ECE8F00101D21D01E1D31D02E067EC26
:109D8000EEF0120069ECEFF0358E0701D76BDF6A59
:109D9000DF2AB1ECF2F001ECE8F0AFECEAF0DB50D6
:109DA00005E00901001D09E1011D07E1010EDB6A63
:109DB00040EC0EF0010E78ECE6F0010EDB5003E112
:109DC000050EDF5CE5E3DF50040802E2010E6DD012
:109DD0000901001D04E1011D02E1020E66D00251DD
:109DE00004250F6E03510521106E000E0F5C400E0E
:109DF000105802E2030E59D006C9D2F107C9D3F1B7
:109E00000101000ED25D380ED35902E2050E4DD08D
:109E1000400E02010F24AC6F000E1020AD6FAC514C
:109E20000101D2250F6E0201AD510101D321106E47
:109E300008C9D2F109C9D3F1800ED25D030ED359FE
:109E400002E2060E32D00FC0AEF210C0AFF2020135
:109E5000AE510101D2250F6E0201AF510101D32194
:109E6000106E0AC9D2F10BC9D3F1BC0ED880D255FD
:109E7000020ED3550FE20FC0A5F310C0A6F30301E5
:109E8000A5510101D2250301A76FA6510101D321DC
:109E90000301A86F0EC9D2F10FC9D3F10101D2514C
:109EA000D31102E1040E01D0000EE1ECEAF002E26F
:109EB000E16AE552E16E4A50FFEFE4F0FAECE4F0BB
:109EC0001F0E0501115D0DE2112B1351EA6A150FEA
:109ED000E96E050E2DECF3F0132B13511F0801E270
:109EE000136BFFEFE4F0FAECE4F0030E785C5BE157
:109EF0000F6A106AFE0EDB500D0803E11F0E0F6E95
:109F0000106AFE0EDB500A0803E11D0E0F6E106A88
:109F1000FE0EDB50090803E1EF0E0F6E106AFE0E15
:109F2000DB50080803E10F68020E106EFE0EDB50D6
:109F30007F0804E1B50E0F6E030E106EFE0EDB50AF
:109F40001F0827E27F0E6EECE5F023E2410E6EEC77
:109F5000E5F00EE3FE0EDB505A080AE3200E4A6ECF
:109F6000FE0EDBCFE7FF4A50E726FE0EE7CFDBFF12
:109F7000020EE66E7A0E0301A7254C6E010EA82193
:109F80004D6EFE0EDB50E00FE82482ECEFF043EC68
:109F9000EAF00F5010102CE010C0E6FF8FDFE55202
:109FA0000FC0E6FF23D0FE0EDB504B6A7A0F4A6EDD
:109FB000060EB7ECEFF0046E2450040B09E10450D8
:109FC000800B06E06F0EE66E79DFE55224840BD03D
:109FD0002450040B08E00450800B05E17F0EE66E70
:109FE0006DDFE5522494049E0450E66E67DFE5526F
:109FF000FFEFE4F065ECEFF0800E6EECE5F003E3CC
:10A00000200EF8ECE7F00201050E3D6FFE0EDB506E
:10A01000740811E1010E3D6F030E785C08E1050143
:10A020001151FC0BE842E842020F02013D6F0501AD
:10A03000006B1E822BD0FE0EDB5028E0DF6A150E6F
:10A04000DF5C11E2B8ECF2F00BE1DF2A0DECE8F096
:10A050009AECEEF0DF2A0DECE8F09AECEEF003D08B
:10A06000030EDF26ECD7150EDF5C04E194ECE5F07F
:10A070003ADFE552200E6EECE5F003E2200EF8EC3C
:10A08000E7F094ECE5F041EC8AF0E552E552FFEFA1
:10A09000E4F069ECEFF024A012D01EB009D0020168
:10A0A000685D1CE30701016B026B68C269F216D0A0
:10A0B0000201682B685180081BE2800E18D01EA098
:10A0C00010D0070E0701015D09E2012B0291024346
:10A0D000020E0201685D02E30701028F0201010E18
:10A0E00006D00201682B6851800802E2800E686F7A
:10A0F0001E9024B01E802450010B03E1020E685D07
:10A1000004E01E50020B01E187D01EA204D007011B
:10A11000CC0E026F0FD0070102910243028F070E8F
:10A12000D8800155016E01500106000903E002913B
:10A130000243F9D700C70AF00201695107081DE27E
:10A1400069513F0802E23F0E696F1DECECF006E03A
:10A15000200E69ECE6F0200E9AECEEF01850080B99
:10A160000CE00701035109E0800E02016925006E31
:10A1700003C701F00701030742DC780E0701025D07
:10A1800018E22A8A02C7E6FF67EC04F0E552DF6EA8
:10A19000DF500EE01DECECF00BE03D5104E0DFCFB2
:10A1A000E6FF28DF04D0DFCFE6FF41EC8AF0E5527E
:10A1B0002A9A18A631D00701035105E002C700F022
:10A1C00003C701F01CDC0701035106E01E50020B1F
:10A1D00003E11C0E025D1DE103510BE01C0E025D4C
:10A1E00008E1CC0E006E030703C701F0FFEC4CF052
:10A1F0001E82189650EC80F0350E675C03E1410E2C
:10A2000027ECE5F0259224BC25820201010E3D6F6A
:10A2100001D003070701026B0A6A020EE15C02E249
:10A22000E16AE552E16EFFEFE4F006015051545D42
:10A2300003E15251555D1DE050C654F652C655F625
:10A24000020E6F5C09E1050E0B5C06E1E66812EC9C
:10A250007AF0E552E66807D052C6E6FF12EC7AF0D3
:10A26000E55250C6E6FF12EC7AF0E5528E8E8E8EE5
:10A270008E9E2850020B2AE02A50010B27E106018E
:10A280005051515D03E15251535D20E0510E69EC94
:10A29000E5F006015051515D09E050C651F6310E0E
:10A2A00069ECE5F050C600F095EC98F006015251CB
:10A2B000535D09E052C653F6320E69ECE5F052C622
:10A2C00000F095EC98F03B0E69ECE5F01200000010
:10A2D00012000601DE6BF00E8C1406092FECEBF079
:10A2E00084AE02D00601DE81F00E8C1404092FEC3E
:10A2F000EBF084AE02D00601DE83F00E8C14070969
:10A300002FECEBF084AE02D00601DE85F00E8C144B
:10A3100005092FECEBF084AE02D00601DE87F00ECB
:10A320008C1402092FECEBF084AE02D00601DE891A
:10A33000F00E8C1401092FECEBF084AE02D0060174
:10A34000DE8BF00E8C1403092FECEBF084AE02D000
:10A350000601DE8DF00E8C142FECEBF084AE02D0F3
:10A360000601DE8FF00E8C1612006FECF3F06EEC2F
:10A37000E5F008E3FE0EDBCFE6FFFD0E9DECECF012
:10A380000AE207D0FD0EDBCFE6FFFE0E9DECECF0FF
:10A3900002E2010E01D0000EFFEFE4F069ECEFF0F5
:10A3A0002FB26CD0DF6A080EDF5C36E2F00E8C1440
:10A3B000DF108C6EB70EFAECE5F000C06FF7070106
:10A3C0006F51190827E2FE0EDB5004E1F00E8C16E7
:10A3D000010E57D0B70EFAECE5F000C070F7070198
:10A3E0007051190817E2B70EFAECE5F000C071F7EA
:10A3F000030EE66E70C7E6FF6FC7E6FFFAECE6F005
:10A4000009E0030EE66E71C7E6FF70C7E6FFFAECDF
:10A41000E6F002E1DF2AC7D7F00E8C16080EDF5CEB
:10A420002AE2DE52010EDD6E080E36ECE5F010E297
:10A43000070EE66E010EDB503B0F8FECE5F0E66E8B
:10A4400070C7E6FFFAECE6F003E1010EDB2AECD779
:10A45000080E36ECE5F00FE26FC772F770C773F7BE
:10A4600071C774F7010EDB50080DF350DF100701C0
:10A47000756F755106D0080EDF5C02E1000E01D049
:10A48000800EE1ECEAF002E2E16AE552E16E4A5048
:10A49000FFEFE4F0FAECE4F01F981F9EFE0EDB5095
:10A4A000005C01E01F8E1F9CFE0EDB50D880005424
:10A4B00001E21F8C020E016E2DA204D01F88FE0E39
:10A4C00000C0DBFF1FAE8FD01F50200B01E0010E3C
:10A4D0004A6E1F50400B01E0010E4A5C01E080D043
:10A4E0001FAC0DD00150D880005414E20150005E22
:10A4F000FE0EDB50D88000540DE21F880BD00128DF
:10A50000E86C005C07E201500026FE0EDB50005CA8
:10A5100001E21F88010157A50FD00050036EDF0E26
:10A52000FAECE5F0F3ECF0F002E628ECEEF002E2F3
:10A530001F9859D00350006E1FA852D0FE0E00C0C5
:10A54000DBFF0494020E6F5C04E1C90E0B5C01E1B9
:10A5500004840450040B11E112EC6EF0000903E0D6
:10A5600049ECEFF03DE0FD0EDB50FF0839E0020161
:10A57000415136E12150200B33E09BECE7F0010123
:10A58000010E016F04A403D0FE0EDB5011D0FD0EAE
:10A59000DB50006EBDEC2DF0500E096EFE0EDB4060
:10A5A000E840E8401F0B006E00501E0802E21E0E3D
:10A5B000006EA0EC96F004B413D0030E0101015D0F
:10A5C000016E0150012AA4ECE5F0200EEF6EDEECE6
:10A5D000F3F0EF50300804E1DEECF3F0200EEF6E04
:10A5E0001F9A1FBC1F8AFE0EDB50FFEFE4F01350D2
:10A5F000040B07E112EC6EF0000903E049ECEFF008
:10A600002EE09BECE7F001012D0E1A6F20A402D082
:10A610002B0E1A6F0201555107E1545105E15351B8
:10A6200003E10101200E1A6FA1ECE5F055C23FF0E5
:10A63000FAECF0F0300F01011B6F300E3B241C6F61
:10A64000300E0201542501011D6F0701EFAB05D04B
:10A65000300E0201532501011E6F01011C8F1200F3
:10A660004EECF4F0FDECE5F0EFCFDFFF01019F6B66
:10A67000A06BA16BA26BA36B1EAE03D0050EA16FE6
:10A680003BD060ECF0F0400B03E12850040B1DE0E0
:10A6900094ECE5F05AEC0EF0E55200C0A1F1005048
:10A6A000630825E20101A16BA02B7D0E005C02E195
:10A6B000190EA16F45ECF1F0FA0E4A1818E14B5053
:10A6C00016E1A02B320EA16F12D060ECF0F0200B3F
:10A6D00002E0A32B0CD060ECF0F0100B07E0020EB0
:10A6E000A26F58A704D0050EA26F01D0A22B2BAEEB
:10A6F00003D0020E85ECE5F0E552FFEFE4F0B10E79
:10A70000006E02018EA502D0B50E006E005015EC51
:10A71000E9F036C100F002018EA502D07CC100F044
:10A72000A0EC96F0300E01011D5D05E19FECEEF00E
:10A7300002E1200E1E6F1200FAECE4F0050E4C6EE2
:10A740004CC044F0FE0ECBECEBF04B6A3D0F4A6E72
:10A75000070EB7ECEFF0006EA2EC93F0010199EC5C
:10A76000EDF00C0E6EECE5F003E20E0E126F0ED063
:10A770000E0E136FFE0EDB50630802E2100E136F15
:10A780000F0E6EECE5F002E2090E146F140E176F57
:10A79000120E186FFFEFE4F0FAECE4F0AEEC93F079
:10A7A0000101012BFE0EDB50006EA0EC96F02C5048
:10A7B000100B07E1640E6EECE5F003E20101200EE0
:10A7C0001A6F2CA807D001014D0E1E6F570E1F6F78
:10A7D0001B8F18D0FD0EDB5003E101011C8F07D049
:10A7E0000A0E6EECE5F003E20101200E1B6F010181
:10A7F000570E1E6FE151010B05E05751080B02E0A7
:10A800002A0E1F6FFFEFE4F0B4EC2CF09BECE7F0A6
:10A8100082ECE6F007E0010EE66E94EC05F0940F92
:10A82000E66E03D0E66A49C1E6FFB6DFE552E552BF
:10A830002CA806D005ECEDF049C1E6FF7DDFE5521E
:10A84000120065ECEFF0B90E15ECE9F035C1DFFF51
:10A8500027ECEBF003E00BECEFF001E1DF6ADF50F7
:10A86000006EA0EC96F0640EDF5C03E20101200EA6
:10A870001D6F0A0EDF5C03E20101200E1E6FE55220
:10A88000FFEFE4F09BECE7F04AC100F0A0EC96F09B
:10A89000640E01014A5D02E2200E196F0A0E4A5D44
:10A8A00002E2200E1A6F930E006EBDEF2DF0020E25
:10A8B0000201955D04E10C0E27ECE5F00AD00D0EC7
:10A8C00027ECE5F0030E0201955D03E10101320E74
:10A8D0001E6F500E096E1200F00E006EB4ECE5F023
:10A8E00002E0F30E006E45EC2EF033C100F0B4EC44
:10A8F000E5F002E054C100F0ADECE9F001011E8F7B
:10A900001200FAECE4F029C100F027ECEBF003E1CF
:10A9100059C100F011D0B4ECE5F00EE055C100F0E3
:10A92000FE0EDB5009E001019751020B05E0975143
:10A93000040B02E098C100F0FFEFE4F0D20E006ECD
:10A94000B4ECE5F00CE027ECEBF009E001019751E5
:10A95000020B05E09751040B02E0F60E006E45EC89
:10A960002EF0010EE66ECDDFE552A0EC96F0300E33
:10A9700001011D5D05E19FECEEF002E1200E1E6F6E
:10A980001200FAECE4F0E1ECF3F0400B03E12850A4
:10A99000040B05E001018F51020B01E18BD0E1ECCA
:10A9A000F3F0200B03E02850040B02E001019E6B42
:10A9B000E1ECF3F0400B03E12850040B57E00101F8
:10A9C000A0510EE0A1510CE1FE0EDB5005E19C51BF
:10A9D00002E19D5101E0A06B9C6B9CC19DF16AD08E
:10A9E0005A0EA15D13E1A1ECE5F09CC13FF0A0EC93
:10A9F000EDF007E1005003E101019D5102E001018A
:10AA0000A16B01019D6B00509C5F54D09C5102E1F1
:10AA10009D5150E09D514A6E4B6A9C510A0DD1ECFC
:10AA2000E7F0A1519EECE9F019ECF4F0D2C143F04B
:10AA3000D3C144F078ECFDF03AC0D0F13BC0D1F185
:10AA40000101D051D11136E0D0510F5ED151105AD1
:10AA5000FE0EDB5001E1A16B0A0E4A6E4B6AACECB4
:10AA6000EFF03EC09CF13AC09DF124D0E1ECF3F050
:10AA7000100B20E0E1ECF3F0200B1CE1020E016E64
:10AA8000010158A702D0050E016E01C0A2F101C05C
:10AA900044F09DC13FF0A0ECEDF004E1005002E075
:10AAA00000C0A2F1FE0EDB5005E0005003E00050B4
:10AAB0000101A25FFFEFE4F0F6ECF4F0E66A61DF7B
:10AAC000E552E5529AC1CFF29BC1D0F29CC1D1F2BE
:10AAD0009DC1D2F29EC1D3F2CDEC3AF001019A5160
:10AAE0000FE10301E35101019B5D0AE2CFC29AF13C
:10AAF000D0C29BF1D1C29CF1D2C29DF1D3C29EF1D2
:10AB00000201842BFFEFE4F0CDECE9F006E1D893ED
:10AB1000CCB3D883D895CCB5D8851200010139A320
:10AB200006D0CC9313B6CC83CC9513B4CC85ECDF94
:10AB300004B05DDD27ECC0F06AEF38F02EBC1200E7
:10AB40000A0E02015403F3504C6E4D6A5551640DC8
:10AB5000F3504C244A6EF4504D204B6E535101017A
:10AB60004A24D46F000E4B20D56F0A0E006E0701E9
:10AB7000EFAB02D0010E08D0EFA907D0140E006E83
:10AB8000010158A702D0320E006E20B403D001019B
:10AB90003EECECF029AA1AD045ECF1F0100ED8806A
:10ABA0004A56270E4B560101D5514B18E8AE02D03C
:10ABB0004B3404D04A50D45D4B50D5591FE200505D
:10ABC00093ECE7F0D4274B50D52318D000504B6AB4
:10ABD000F00F4A6ED80E4B2201014B50D519E8AE4A
:10ABE00002D0D53504D0D4514A5CD5514B5806E239
:10ABF000005093ECE7F0D45F4B50D55B2084800E7F
:10AC0000D51503E020943EECECF045ECF1F0D4C116
:10AC10003EF0D5C13FF059ECEDF04BAE04D03A6CAC
:10AC20003B1E000E3B223A500101D45F3B50D55BE6
:10AC3000FBECEEF0BFECF2F03EC055F23A500101F1
:10AC4000D46FD56B0A0E4A6E4B6ABFECF2F03EC071
:10AC500054F23AC053F22DEF56F00101CAA9308EDA
:10AC6000198C04808EEF55F00A01DA9F54EC0DF038
:10AC7000016A0C5011E1A8ECE6F02AE10701EFBFF0
:10AC800011D00A0E016E7DECE8F03F50006E0150CD
:10AC9000005C1EE200501BD0030E0C5C12E10701A9
:10ACA000EFAF02D0160E13D0030E785C02E1140E43
:10ACB0000ED0785002E11E0E0AD0260E49ECF0F0BC
:10ACC00006D05FECE8F002E0010E01D0160E016E36
:10ACD0000150160802E2160E016E12000A0E010162
:10ACE0000F5D09E12C50100B06E14951500803E2B9
:10ACF000790E495D01E3000C010CF0DF000903E06F
:10AD00000101500E496F1200FAECE4F000AE14D0CD
:10AD1000FF0E0002F3CF84F2840EE96E020EEA6E9B
:10AD2000EFCF3FF0FE0EDBCF44F0BCECFDF03FC0B8
:10AD3000EFFF0201846D09D000C03FF0FE0EDBCFB3
:10AD400044F0BCECFDF03FC084F2FFEFE4F0010101
:10AD50008BAD07D02EAC02D0FCEF04F002010A0E3E
:10AD60003C6F12000101E1A503D0E195CFEFEBF0BC
:10AD70000601D951D995010B01E0D985D951D9974F
:10AD8000020B01E0D987D9918850400B01E0D981AD
:10AD9000D9938850800B01E0D9830F0ED9153FEC71
:10ADA000E6F000A005D000AE02D0DF0701D0DF2B17
:10ADB000DA51DA95010B01E0DA85DA51DA97020B04
:10ADC00001E0DA87DE51DA91020B01E0DA81DE512F
:10ADD000DA93010B01E0DA830F0EDA153FECE6F0AF
:10ADE00000A009D0CFECEBF000AE03D00601E007E5
:10ADF00002D00601E02BDB51DB95010B01E0DB8586
:10AE0000DB51DB97020B01E0DB87DE51DB91080BA6
:10AE100001E0DB81DE51DB93040B01E0DB830F0EED
:10AE2000DB153FECE6F000A009D0CFECEBF000AE74
:10AE300003D00601E10702D00601E12BDC51DC95CD
:10AE4000010B01E0DC85DC51DC97020B01E0DC87C3
:10AE5000DE51DC91200B01E0DC81DE51DC93100B34
:10AE600001E0DC830F0EDC153FECE6F000A00AD019
:10AE70000201320E3B6F00AE03D00601E20702D0A2
:10AE80000601E22BDD51DD95010B01E0DD85DD5191
:10AE9000DD97020B01E0DD87DE51DD91800B01E0E3
:10AEA000DD81DE51DD93400B01E0DD830F0EDD150A
:10AEB0003FECE6F000A00AD00201320E3B6F00AE7C
:10AEC00003D00601E30712000601E32B1200045031
:10AED000010B4A6E0450020B01E0010E4A5C07E0D0
:10AEE000D60EE66EF20EE66E010E5FEFE6F0E00EB5
:10AEF0000101EC15016E1F0EEC15026EEDC103F0A1
:10AF0000015003E0E00E015C54E102506EE001509C
:10AF1000021203501FE12050080B06E03C51010BC8
:10AF200003E02850010B16E02E50400B03E0305098
:10AF3000200B10E02150200B0DE002507926CA5161
:10AF4000100B08E02050080B05E02C50200B02E10C
:10AF500002500726030426E13C51200B12E1205049
:10AF6000080B0FE02E50400B06E13C51020B09E0AC
:10AF70002850010B06E12E50400B14E03C51010B10
:10AF800011E12150200B0EE03C51200B09E0205034
:10AF9000080B06E03C9B289D076A0201320EFD6FFC
:10AFA00002500726020E035C20E102500601DF2753
:10AFB0001200800E015C11E1100E025C16E2070E19
:10AFC0000214400F676E178E1798179002A602D0D2
:10AFD000178801D01780DE951200C00E015C05E1D4
:10AFE000030E025C02E202C0EDF1120019BE120073
:10AFF0008A8C81AE03D00101E99712008150800B49
:10B0000055E10101E951080B51E1F29E8A9C04903F
:10B010000492090E016EEC6B060E5CECE7F0270E55
:10B02000026E0150010803E20101EC91EC4381AE94
:10B0300009D00150010805E202060101EC8F0470FD
:10B0400001D004829EAA04D0020E025E2FECE7F02B
:10B05000025042ECE8F00106E2E1E00E0101EC15DD
:10B06000C0081FE1080E016EF9C206F0020E5CEC8A
:10B07000E7F00F0E936E270E026E06A002D08A8EA6
:10B0800001D08A9E069006429EAA04D0020E025E5D
:10B090002FECE7F0025042ECE8F00106ECE18F0EF5
:10B0A000936E15DF8A8C0101E987F28E120069EC3C
:10B0B000EFF09CDF28A004D079ECCAF08CEF5DF0B3
:10B0C0002450800B4AE13150400B47E120A61BD0B1
:10B0D000A5ECECF0010127990201845102E0010185
:10B0E00027890101279B020184AF02D00101278B30
:10B0F000010127A932D01EAC02D0EEEC0BF0020108
:10B10000640E506F2AD07950006E010127990050CB
:10B1100001E02789279B00BE278B27BB006C020E0E
:10B120006F5C0FE1B90E0B5C03E0E30E0B5C05E115
:10B13000D8900032D890003207D00038E842070B90
:10B1400002D000380F0B006E005006E0278D279FBD
:10B1500027BB278F796A01D0279901012751100B4E
:10B1600009E0CA51100B06E12C50200B52E01E5092
:10B17000400B4FE12050080B1DE03C51200B09E033
:10B180002E50400B06E1CA51100B14E02751100B52
:10B1900011E0ADECECF0010128990201845102E0CC
:10B1A000010128890101289B020184AF32D00101ED
:10B1B000288B2FD00750006E2899005001E0288975
:10B1C000289B00BE288B289928BB006C31AC05D089
:10B1D000D8900032D89000320FD01CA204D0003892
:10B1E000E8461F0B08D033A004D00038E842070B14
:10B1F00002D000380F0B006E00500AE00701280E45
:10B20000D86F0101288D289F28BB288F076A01D09D
:10B2100028992C50200B03E01E50400B0DE001013B
:10B220002751100B01E00DD32851100B01E009D379
:10B230002150200B01E105D3D7CADCFAD6CADDFACA
:10B2400091DDDFC600F00601D999005001E0D989EF
:10B25000D99B00BED98BD9A938D0D9BB006C4DEC95
:10B26000EFF033E0DF6B0201640E506F1350080BF8
:10B270000DE11350040B0AE1020E0101775D0EE1AE
:10B280003C51200B0BE02E50400B08E1298A0601AF
:10B29000D9BB299A53DC22ECECF017D03851010BC2
:10B2A00014E03C51010B11E1E0C279FF0601D9AB7A
:10B2B00004D0E0C279FF0F01796C01012789CAA986
:10B2C00003D07950076E28892884E0C600F0060173
:10B2D000DA99005001E0DA89DA9B00BEDA8BDAA94C
:10B2E0007CD0DABB006C4DECEFF001E176D0E06B86
:10B2F000010E0E6EDABB0E685BECE8F06CE02E50CF
:10B30000400B03E0F4ECE8F066E1050E0C5C03E1B1
:10B31000E0EC0BF060D0020195510EE0030E5FEC03
:10B32000F4F0950EE66E020E21ECE5F057EC54F0C9
:10B33000178E3A0E676E4FD032BC4DD0060150A723
:10B3400025D0358491DC0E040BE1A7ECEDF008E28A
:10B35000190E0124D75D04E2020ED65FD72B11D05F
:10B36000800E0E140EE041EC12F0FF0F0A01D65DC4
:10B3700008E2EEECECF0D880D75503E2020ED627B7
:10B38000D7070A01010ED46F348821D050A523D0ED
:10B390003584EAECECF008E0C80EE66E280EE66EA6
:10B3A000D80EE66E030E0AD05FDC190E0124E66E9D
:10B3B000EEECECF0E66ED70EE66E0A0E21ECE5F050
:10B3C0000A01030ED46F34887CEC20F0010EE66E87
:10B3D000E66E99ECE6F0B4ECEAF0E1C600F00601A6
:10B3E000DB99005001E0DB89DB9B00BEDB8BDBA936
:10B3F00063D0DBBB006C4DECEFF05EE0E16B010E67
:10B400000E6EDBBB0E68050E0C5C03E1E0EC0BF08E
:10B4100053D05BECE8F050E02E50400B03E0F4EC2E
:10B42000E8F04AE1060150AB27D0358434EC56F001
:10B43000800E0E140CE0A7ECEDF009E2EEECECF05F
:10B44000D880D75504E2020ED65FD7070FD00E047E
:10B450000DE141EC12F0FF0F0A01D65D07E2190E73
:10B460000124D75D03E2020ED627D72B0A01020E74
:10B47000D46F348800ECF0F0060150A91BD035845D
:10B4800051EC12F00BECF0F007E24A501408000EF9
:10B490004B5402E251EC12F00BECF0F009E24A508E
:10B4A0003D08000E4B5404E251EC12F051EC12F046
:10B4B0005AEC12F0B4ECEAF0E2C600F00601DC99B6
:10B4C000005001E0DC89DC9B00BEDC8BDCA998D05D
:10B4D000DCBB006C4DECEFF001E192D0E26B010EB1
:10B4E0000E6EDCBB0E682DA418D0B4ECE5F008E1BC
:10B4F000C80EE66E330EE66E010E1CECE5F00AD0C7
:10B50000C80E5FECF4F0540EE66E010E21ECE5F08F
:10B51000ECEC1DF06CEC54F06FD050AD19D0320E45
:10B52000006E01018FAD02D0640E006E0050E66E19
:10B53000080EE66E4A0EE66E010E21ECE5F042ECD6
:10B5400054F04AC103F5E9EC7FF00201178754D0AB
:10B5500050AF52D097ECE7F001018EA503D036EC46
:10B5600009F04AD03450040B25E0000403E0020E39
:10B57000005C20E10E50462746C1E6FFC10E0FECED
:10B58000E5F00E0E27ECE5F046C100F0010146AFF4
:10B5900004D046C100F00001006C00900042A0EC15
:10B5A00096F001012B0E1D6F46AF02D02D0E1D6FC0
:10B5B0001F8F22D002018EA50FD03C0EE66E7C0EAE
:10B5C000E66E010E1CECE5F07CC1E6FFCC0E0FEC44
:10B5D000E5F07FEC53F00FD016EC1EF03C0EE66E5B
:10B5E000360EE66E010E1CECE5F0A6EC16F07FECD4
:10B5F00053F0020119832B842E8E02011E0E306F30
:10B60000E3C600F00601DD99005001E0DD89DD9B15
:10B6100000BEDD8BDDA915D1DDBB006C4DECEFF07C
:10B6200001E10FD1E36B010E0E6EDDBB0E682DA69E
:10B630002FD0B4ECE5F00AE13C0EE66E290EE66E82
:10B64000010E1CECE5F0A1ECE9F01FD027ECEBF0CB
:10B6500006E13C0EE66E590EE66E010E12D00101B7
:10B660009751020B09E09751040B06E03C0EE66E81
:10B67000980EE66E010E05D03C0EE66E550EE66E97
:10B68000010E1CECE5F020EC1EF09EEC54F0D5D041
:10B6900052AFAFD001018EB5B1D034B632D021BE99
:10B6A00004D08D0E006E4FEC2EF0FF0E0E5C0CE100
:10B6B00002013F0ED8800F55000E10551FE2400EBC
:10B6C0000F5F000E105B1AD086C201F02C50100BD9
:10B6D00007E102018651780803E26C0E015C016EFD
:10B6E00001500101CF5D0AE20201480E0F5D710EAB
:10B6F000105904E2400E0F27000E1023E7EC0BF068
:10B700009CD002012D6B780E016E026A2FECEFF0D7
:10B7100002E0DA0E016E2CA804D0960E016E0A0E1D
:10B72000026E0150E66E0250E66E490EE66E010EA4
:10B7300021ECE5F02B84E1EC2AF06EEC56F00009E8
:10B740000BE00101500E496F0E0406E12FECEFF003
:10B7500003E00101790E496F04EC54F0780E016E9C
:10B760007DECE7F002E1500E016E2C50100B10E161
:10B770000E0403E1790E495D06E0800E0E1408E028
:10B780000150495D05E1328E5BECE8F001E01D946B
:10B7900097ECE7F03250800B0EE1020131510BE0E3
:10B7A00000500CE0050E005C09E0030E005C03E1B4
:10B7B000020E785C03E00E50A4ECEEF032AE16D030
:10B7C000329E010EDB6A1AA006D0DB682FEC0BF06C
:10B7D000050E85ECE5F07FEC28F0A8DA010EDB50D1
:10B7E00002E02AEC0BF00E50A4ECEEF00201188BF4
:10B7F00024D052A122D001018EA503D036EC09F04D
:10B800001CD035C1DEF216EC1EF0280EE66E350EA9
:10B81000E66E010E1CECE5F036ECEDF003E0010104
:10B82000355106E00201DE5105E10101355102E02A
:10B83000E5EC1CF0020119852B842E8E02011E0EF0
:10B84000306F1EAC64D00701EF83E1EC09F0010119
:10B850003C91139C3C51010B01E0138C5BEC34F0E8
:10B86000006E00500F0802E20F0E006E100E000274
:10B87000F3CF21F253EC2FF01E9A050E0701D325CA
:10B880000201D880215501E21E8A2B50800B13E162
:10B89000205111E0050E0701D35D0201215D03E295
:10B8A00025EC09F01E881E50100B31E01E50200BB5
:10B8B0002EE0020109D02B50800B0AE11E50800BB4
:10B8C00007E11E50200B04E0FA0E206F1E981FD0D7
:10B8D0002BBE02D022EC09F02CBA17D00C0EE66E6B
:10B8E000050EBEECEAF0E66E06ECE8F00AE007C5ED
:10B8F000BFF108C5C0F109C5C1F10AC5C2F10BC548
:10B90000C3F1E0C279FF0101279B010127891E5085
:10B91000800B0AE101012751100B6FE02050080B4A
:10B920006CE02150200B69E002011E0E306F1EAC4E
:10B9300002D0140E306F2CAA2FD01EBC16D00101DD
:10B940004551630801E2456B800E791406E0FB0E59
:10B95000795C03E2796A000E11D0800E79144CE113
:10B960007950030849E2796A08D0796A2BAE09D088
:10B970000501065141E1320E066F010EAEECEDF00D
:10B980003BD00101A851030837E3010EAEECEDF006
:10B990000101140EA86F30D0178305013B812C8C58
:10B9A0002D8AC4ECE5F00C50E66E30EC53F0E55215
:10B9B000A5ECECF01E50800B05E0795003E1A9ECFA
:10B9C0003AF014D0020184AF09D0EFC7E6FF5CEC77
:10B9D00055F0E5520201E051792608D0845106E085
:10B9E000EFC7E6FF4EECEAF0E051795E02018451C8
:10B9F000DFE12E829DEC04F01E9E01012851100B08
:10BA00005AE02050080B57E02150200B54E002016F
:10BA10001E0E306F1EAC02D0140E306F178305015E
:10BA20003B832C8C7D50DF6E2E50400B03E1D5EC18
:10BA3000EAF002E00C50DF6E2EAC04D02D8AC4EC8C
:10BA4000E5F003D02D9AA2ECE7F0DFCFE6FF30EC73
:10BA500053F0E552ADECECF0020184AF0BD0DF50B7
:10BA60004CECF2F0E66E5CEC55F0E5520201E1516F
:10BA700007260AD0845108E0DF504CECF2F0E66E65
:10BA80004EECEAF0E151075E8451E4E12E822EACE7
:10BA900003D09DEC04F002D0B8ECE7F025A605D069
:10BAA000010E096E0701140E826F0101CAA903D0AD
:10BAB0000701280ED86F2CAC2BD0D5ECEAF00FE0A4
:10BAC0002751100B0CE02851100B03E12C50200BD8
:10BAD00006E02E50400B03E105013B832C9C010145
:10BAE0008BAD03D02C9C08AE198CF1EC38F0010121
:10BAF0003CA9308ECFEC3EF02C9C26822D50200BA2
:10BB000006E02E50400B03E1D5ECEAF001E0248A78
:10BB10000101289927992894020EE15C02E2E16A6A
:10BB2000E552E16EFFEFE4F0FAECE4F0180E0701E5
:10BB30001B171C6BFE0EDB5001E11C81FE0EDB04AB
:10BB400001E11C83E2ECECF001E11B81FE0EDB5015
:10BB5000030801E11B83FE0EDB50040801E11B8595
:10BB6000FFEFE4F0695005E0D5CAE6FFDDDFE552FE
:10BB70001200180E07011D171E6B0A01D55102E1B4
:10BB800007011E810A01D50502E107011E83020E8D
:10BB90000A01D55D02E107011D81030E0A01D55D91
:10BBA00002E107011D83040E0A01D55D02E10701D0
:10BBB0001D851200000000000000E8EC08F0F2EC27
:10BBC00008F082A82D808A8A1200020E42ECE8F06A
:10BBD000DAEF5DF0050EE66EFEEC18F0E552F00EC1
:10BBE0008C148C6EA0D88A9A00001FC700F0010147
:10BBF000E3A915D00050E66E12EC7AF0E5521DC7AD
:10BC000004F0049C07011EB1048C049E07011EB3BE
:10BC1000048E0450E66E12EC7AF0E5521DD0060E4A
:10BC200000C0E7FF070B04E0E742E79EE806FCE1FF
:10BC3000E750E66E12EC7AF0E5523F0E0014040D68
:10BC4000F35007011E11E66E12EC7AF0E5521DC7A3
:10BC5000E6FF12EC7AF0E552ADDFF00E8C14060927
:10BC60008C6E61D88A9A000020C700F00101E9A318
:10BC700015D00050E66E12EC7AF0E5521BC704F0C6
:10BC8000049C07011CB1048C049E07011CB3048EA4
:10BC90000450E66E12EC7AF0E5521DD0060E00C09C
:10BCA000E7FF070B04E0E742E79EE806FCE1E75008
:10BCB000E66E12EC7AF0E5523F0E0014040DF350DC
:10BCC00007011C11E66E12EC7AF0E5521BC7E6FF85
:10BCD00012EC7AF0E5526EDF1200F00E8C140409BB
:10BCE0008C6E21D88A9A000010C7E6FF12EC7AF019
:10BCF000E55260DF1200F00E8C1402098C6E13D82E
:10BD00008A9A000013C7E6FF12EC7AF0E55212C7D8
:10BD1000E6FF12EC7AF0E55211C7E6FF12EC7AF07A
:10BD2000E55253DF1200010E42EFE8F0050EE66E19
:10BD3000FEEC18F0E5522D90DEDF4CDFF5EC13F051
:10BD4000F00E8C1405098C6EEEDFEDDFECDFEBDF1F
:10BD50008A9A0DC7E6FF12EC7AF0E5520CC7E6FFAF
:10BD600012EC7AF0E5520BC7E6FF12EC7AF0E552DE
:10BD70000AC7E6FF12EC7AF0E55227DFF00E8C14CA
:10BD800003098C6ED0DF8A9A00000FC7E6FF12EC21
:10BD90007AF0E5520EC7E6FF12EC7AF0E5520ADFC0
:10BDA000F00E8C140A098C6EBEDF8A9A000009C757
:10BDB000E6FF12EC7AF0E55208C7E6FF12EC7AF0E3
:10BDC000E55207C7E6FF12EC7AF0E55206C7E6FF38
:10BDD00012EC7AF0E552EEDE80DFF00E8C140109F1
:10BDE0008C6EC682C6909FDF8A9A00000000000019
:10BDF000000016C7E6FF12EC7AF0E55215C7E6FF21
:10BE000012EC7AF0E55214C7E6FF12EC7AF0E55234
:10BE1000DCDEC680C692F00E8C161200810E98EC05
:10BE2000E5F0320E096E308834C12AF21200030E9A
:10BE30000A6E2A0EE66E000EE66E0A0E76EFF1F03E
:10BE4000030E0A6EAA0EE66ED2ECF3F0E66E300E2A
:10BE5000D1EFF4F063EFF4F0FAECE4F005013B8F7E
:10BE6000E2ECECF00DE101013CB902D08B9D08D071
:10BE70003C99E66A42EC90F0E55201018B9D34D08A
:10BE8000FE0EDB5024E0F4ECE8F021E1CA993CB965
:10BE900009D03C89010EE66E42EC90F0E5520101BA
:10BEA0008B8D03D08B8D28EC90F0198638EC0DF03B
:10BEB0001B82E6ECB8F00EECB9F01B92076A796AC7
:10BEC000C70EE66EF20EE66E010E5FECE6F0FE0EB9
:10BED000DB5011E1F4ECE8F00EE08B9D28EC90F0E3
:10BEE00038EC0DF06AEC38F0CE0EE66EF20EE66E2F
:10BEF000010E5FECE6F0FFEFE4F012001E50400B85
:10BF00000CE02B50800B09E12250200B06E02B8E19
:10BF1000130E15ECE9F025EC09F0120025A808D065
:10BF2000010EE66E99DFE5520F0E79ECF3F01B86F9
:10BF30001200010124A17DEF67F0010124910201AB
:10BF400022070201225101E0A8D10201640E226FF2
:10BF50000201EC6B0201295102E0020129070101F3
:10BF60008C5106E001018C0701018C5101E13296F0
:10BF7000020130510EE02050080B0BE002013007A7
:10BF80000201305106E11EAC02D01E8E02D02EBE40
:10BF90002E9E300E0401B75D06E10201176B186B8F
:10BFA000196B1A6B02D0A6ECCCF002012A5126E0E4
:10BFB0000501005123E12850400B20E102014A51C4
:10BFC0004B111CE102012A0702012A5117E10D5011
:10BFD000006E02016A5108E07F0E02016A15006ED0
:10BFE000199A02016ABF198A010EE66E0050E66EC8
:10BFF00099EC8FF0E552E55202016A6B02016E077F
:10C0000002016E511EE10701F1050FE102010F0E61
:10C010006E6F560E02011E5D07E2870E006E2488C9
:10C020005AEC2EF00968268E0CD001015251020103
:10C030001E5D07E2870E006E24885AEC2EF0096818
:10C04000268E020128514EE00201280702012851E4
:10C0500047E12250200B44E00E0E675C3AE150ECC1
:10C06000AFF028702892520EE66EE1EC07F0E55230
:10C07000520EE66EE1EC07F0E55228B011D0570EF3
:10C08000E66E6FEC2EF0E5526AEC38F046EC15F0F7
:10C090004E0EE66EE1EC07F0E552E9EC18F013D035
:10C0A000580EE66E6FEC2EF0E55268EC95F0E80E57
:10C0B000E66E06ECFDF0E552E2EC18F0520EE66E8C
:10C0C000E1EC07F0E5523B0EE66EE1EC07F0E552DD
:10C0D00007D028A005D04C0EE66E48ECCAF0E55219
:10C0E0007DEF67F0D7ECC4F0010101013951100B6D
:10C0F00006E11450020B05E01A50200B02E1060184
:10C1000005792950400B01E0010E020F016E295004
:10C11000400B01E0010E050F026E03681EAC10D04B
:10C120000150EA6A110FE96E010EEA22EF7E01501A
:10C13000EA6A110FE96E010EEA22EF50800B036EDE
:10C1400061EC0BF0000923E0FF0E035C11E10250EB
:10C15000EA6A110FE96E010EEA22EF7E0250EA6AE6
:10C16000110FE96E010EEA22EF50800B036E0FD023
:10C170000250EA6A110FE96E010EEA22EF9E0250A8
:10C18000EA6A110FE96E010EEA220350EF126FEC1A
:10C190000BF000091AE0FF0E035C08E10250EA6AA6
:10C1A000190FE96E010EEA22EF7E0FD00250EA6A03
:10C1B000190FE96E010EEA22EF9E0250EA6A190F8A
:10C1C000E96E010EEA220350EF12DBEC04F00009E5
:10C1D00002E006011A772350040B05E02D50100BE6
:10C1E00002E00601127718EC08F000090EE02D506D
:10C1F000400B0BE12D50800B08E10101DEB703D0AD
:10C2000006010E7F02D006010E8F0201435105E0A8
:10C210001450080B02E00601027D34ECC4F0000962
:10C2200003E12F50200B27E02F9AE2EC18F0016A6F
:10C23000030E015C15E2026A040E025C0BE2020EC0
:10C24000006E36EC91F0320EE66E35EC29F0E552D8
:10C25000022AF2D7E66835EC29F0E552012AE8D740
:10C26000E9EC18F001016099268250EC9BF01FEC7C
:10C27000C4F0BBECC3F002013D5102E002013D07F6
:10C280000201905105E02350100B02E102019007DA
:10C290000201455102E0020145072850010B28E048
:10C2A0008150010B03E02150040B22E01AEC16F040
:10C2B000FF081EE12E50400B1BE12150200B18E01F
:10C2C0001950800B15E10201245102E002012407FC
:10C2D000020124510DE12AA003D0CBEC07F0FBD7DB
:10C2E0003B0EE66EE1EC07F0E5520201280E246FEA
:10C2F0000601F45102E00601F4070201FE5102E0DA
:10C300000201FE070201FD5107E00201FD070201E3
:10C31000FD5102E101013C8B010197AD15D10301F3
:10C32000C6070301C65101E00FD1C69AF00E8C1466
:10C3300007098C6EF8DC8A9A0000000000000000FB
:10C340000000000000000000049082B804808A8A87
:10C35000C68AF00E8C160101E0BD12D00301010E59
:10C36000C66F04A00CD00301060EC66F0101E08D5C
:10C370000301CA6BCB6B0301C86B0301C76BE4D02D
:10C38000D8900301CB33CA330301C82B04A003D0D8
:10C390000301CB8F09D00D0E0301C85D05E2030137
:10C3A000C72B070E0301C7170301040EC66F030155
:10C3B000C8510F0801E3C8D00301960EC66F0101F2
:10C3C000E09DCAC30FF0CBC310F000010F1C01E1C8
:10C3D000101C0BE1020E6F5C07E1B90E0B5C04E16F
:10C3E000248A26820601426BAFD00FC00FF010C026
:10C3F00010F00F1E101E10C000F0700E0016003856
:10C400000F0B006E0301C751005C01E09DD00F0EC1
:10C4100000011016000110A603D0F00E000110124A
:10C420000FC0D4F110C0D5F10101D53504E3D451CA
:10C430001708FC0ED55501E387D00101D890D551DE
:10C4400004E6E90ED45D030ED55901E37DD0D0C3D7
:10C45000CEF3D1C3CFF3D4C1D0F3D5C1D1F30A0EFB
:10C460000F6E106A030E0301C95D03E2640E0F6EC6
:10C47000106A0101D4510301CE5D4C6ECF51010110
:10C48000D5554D6E4CC0E6FF4DC0E6FF98EC2EF042
:10C49000E552E552F3CF4AF0F4CF4BF00F504A5C2F
:10C4A00010504B584AE2D0C3CCF3D1C3CDF3FF0EAA
:10C4B0000301C95D02E20301C92B030E0301C95D3B
:10C4C00022E30101D4510301CE5D4C6ECF51010135
:10C4D000D5554D6E4CC0E6FF4DC0E6FF98EC2EF0F2
:10C4E000E552E552F3CF4AF0F4CF4BF0000ED8807E
:10C4F0004A54000E4B540CE20201345109E1C2ECE3
:10C5000005F0000905E0D0EC2CF03488B3EC4BF0DA
:10C51000020E6F5C11E1B90E0B5C03E0E60E0B5CE2
:10C520000BE1248A2682B90E0B5C06E10601080E97
:10C53000426F06011E0E436F07D00301C951020866
:10C5400003E20301010EC96F02014A514B1164E07D
:10C550001CA020D002014A07000E4B5B02014A5189
:10C560004B1117E11A50200B14E01CA210D09EECC6
:10C570000AF054EC05F0EFC2D2F1F0C2D3F10EECA8
:10C580000BF00201280E4A6F230E4B6F02D0A4EC71
:10C590000AF042D02150400B3FE01A50400B3CE0E3
:10C5A0001850080B03E11A50200B36E002014A072D
:10C5B000000E4B5B1A50200B0CE09EEC1DF00009A6
:10C5C0000AE18150010B05E101010101DE51100B6F
:10C5D00002E1000E01D0010E0490E8B004800201D7
:10C5E0004A514B1103E00450010B16E002014A6B63
:10C5F0004B6B0101DE9904A006D002012A6B2AC20E
:10C600006AF250EC80F0A4EC0AF018A604D025924F
:10C6100024BC2582228E21940201505102E00201A5
:10C6200050070201515102E00201510702014F512E
:10C6300002E002014F070201465102E002014607F3
:10C640000201425102E002014207020140510FE0A3
:10C6500002014007020140510AE108504A6E4B6A4C
:10C66000820E4A1801E14B5002E053EC0EF02B50C1
:10C67000200B56E002013B5153E10701DE5102E07D
:10C680000701DE0701012C5107083AE277EC28F098
:10C69000000936E008AE0ED00701DE510AE17EEC5B
:10C6A00014F0D5EC0FF002010F0E456F07015F0E7D
:10C6B000DE6F25D00201455122E10101010139510E
:10C6C000040B04E10A0E01012C5D07E12FEC0BF0D5
:10C6D000060EE66E35EC29F0E5520BEC05F0D5ECD4
:10C6E0000FF0010101013951040B04E10A0E0101AF
:10C6F0002C5D02E12AEC0BF002010F0E456F10D009
:10C70000800E081405E1010101013951040B08E113
:10C710000701DE5105E1D5EC0FF007015F0EDE6F7A
:10C72000020123070201235146E10201280E236F73
:10C730001BAC10D078EC4AF00C50006EB3EC4AF011
:10C7400006010F7706010FA704D07D50006EB3ECF1
:10C750004AF031D01CA803D0060112772CD01DA2BC
:10C7600003D00601147727D01A50200B07E00101EF
:10C7700001013951100B02E1060105792550020B28
:10C7800004E1C3EC0DF0000916E00201405113E191
:10C7900008504A6E4B6A820E4A1801E14B500BE07A
:10C7A0002650040B06E12D50800B05E12D50400B67
:10C7B00002E10601107F0501445129E0C2EC05F0B9
:10C7C000000925E02250100B22E005014407050175
:10C7D00044514A6E4B6AD8904B5004E6960E4A5C20
:10C7E000000E4B580CE3050144514A6E4B6A960EFD
:10C7F0004A1801E14B5002E10501446B08D00601E3
:10C800001C9F140E0501445D02E206011C8F02010B
:10C810003B5102E002013B0702013C5114E00101DF
:10C8200001018B51400B0FE0C2EC05F000090BE059
:10C8300002013C0702013C5106E11B820EECB9F0FB
:10C840001B92076A796A0701D85107E00701D807E8
:10C850000701D85102E1076A796A02013A511EE0E4
:10C8600002013A0702013A5119E1FCEC26F00009F5
:10C8700003E190EC97F012D00701D5510701D611D2
:10C880000DE00701D55102E00701D5070701D65198
:10C8900002E00701D6070201020E3A6F0201395188
:10C8A0000CE0020139070201395107E1178E170E1A
:10C8B000676E2DAC02D00F0E676E0101A95174E0B6
:10C8C0000101A9070101A9516FE1ADC1F6FFAEC198
:10C8D000F7FFAFC1F8FF0800F550006E0201DF510D
:10C8E00007E0830E0A6EDFC201F03EEC4DF00A6AEB
:10C8F0000201AA51AB1120E0010EE66EAAC2E6FFCA
:10C90000ABC2E6FF060EE66E010EE66E0DEC4EF0D3
:10C910004A6E050EE15E4A50016E06C100F002014A
:10C92000AA2B000EAB233550800B05E0015003E02D
:10C9300000507F0801E2006A005015E00101190E65
:10C94000A96F0050E66E41EC8AF0E5520201DF511A
:10C9500003E00201DF2B06D00101AD2B000EAE2358
:10C96000000EAF2321D02950080B03E13150080BF2
:10C9700002E0299619D00201DF5105E00201DF6BC8
:10C98000FA0E096E04D0D8900932D890093224A644
:10C990000BD01C0EE66EED0EE66E010EE66E75EC2B
:10C9A0002EF0E552E552E5520201385106E002014F
:10C9B00038070201385101E1269E0201375109E092
:10C9C000020137070201375104E10601416941C6FE
:10C9D00040F60101A65102E00101A60707018251BC
:10C9E00002E00701820702013F512AE002013F07EE
:10C9F00002013F5125E1000E0601E76EC019E8AEC5
:10CA000002D0C03503D0E750D880C05503E20601FC
:10CA1000C00702D00601C02B000E0601E76EC21946
:10CA2000E8AE02D0C23503D0E750D880C25503E249
:10CA30000601C20702D00601C22B0201050E3F6F9C
:10CA40000301E7516AE00201345167E108BE03D0F7
:10CA50000301E76B62D00301E7070301E7515DE1E2
:10CA600020A20BD0BAC19AF1BBC19BF1BCC19CF111
:10CA7000BDC19DF1BEC19EF10AD0B5C19AF1B6C14A
:10CA80009BF1B7C19CF1B8C19DF1B9C19EF1010103
:10CA90009A514C6E4D6AE80E4D02F3CF4DF0030EE5
:10CAA0004C02F3504D26E80E4C02F3CF4CF0F450FC
:10CAB0004D2601019B510A0D4C50F3244A6E4D50F6
:10CAC000F4204B6E0A0E4E6E4EC044F09CC13FF0F7
:10CAD000BCECFDF03F5000014A240F6E000E4B20CD
:10CAE000106E030E0F0B05E0D89010320F32E806DF
:10CAF000FBE10301E8510F1802E1E95110180DE0C4
:10CB00000FC0E8F310C0E9F3400E016E00011050B1
:10CB100001260FC000F0A7EC91F0020131512EE088
:10CB20000201310721BC25D00101DFA106D002019D
:10CB3000316B0101DF91F2EC27F01B50800B19E003
:10CB4000800E081416E02150010B13E10201316B35
:10CB50001B9E0A01DA8F54EC0DF0010EE66EA7EC75
:10CB600090F0E5520201020E3C6F0201178B0501A5
:10CB70003B850201315102E1248A268202012051C3
:10CB800009E01E50400B06E002012007020120517F
:10CB900001E11E8E0501065102E0050106070201B2
:10CBA000485107E0020148070201485102E146EC02
:10CBB0000AF009506BE00906095068E1189C189EBC
:10CBC00030980101DE951D921C982682248A2898AF
:10CBD00021BA13D0040E0101445D08E101010101F5
:10CBE0008E51100B03E10101E38F05D07EC1E6FFFA
:10CBF000BAEC0EF0E55287EC2EF0218A55EC93F05A
:10CC00007EEC5FF001010101E351100B14E02E50A6
:10CC1000400B11E12250200B0EE0180E675C0BE177
:10CC20001750100B08E0020E0B6E2EEC9BF002EC7E
:10CC30009BF012AC178E0201955103E13250400B6C
:10CC400025E022AA1CD0092A188E020E0201955D49
:10CC500015E1020196514A6E4B6A4B3404E24A5088
:10CC60009608000E4B5408E2AEEC93F0100EE66E00
:10CC700053EC97F0E55202D00201962B07D0329C7C
:10CC80000201955103E0178E3A0E676E02012D5195
:10CC900002E002012D0702012E5102E002012E07DF
:10CCA00002012F5102E002012F070201475102E069
:10CCB000020147070201435102E00201430702015A
:10CCC000445102E0020144070101A85102E00101C0
:10CCD000A8070301E25102E00301E20702014C51FF
:10CCE00002E002014C0702014D511EE02250200BD0
:10CCF0000CE1110E4A6E4AC044F04DC23FF0BCEC4C
:10CD0000FDF03B5002E106010E7D02014D0722506D
:10CD1000200B05E02150400B02E0E3EC05F002019E
:10CD20004D5102E107EC05F0060143510EE006010A
:10CD300043070601435103E106015A0E436F26865D
:10CD40000F0E0601435D01E226960201325110E00A
:10CD50000101E9A503D00201010E326F0201320781
:10CD60000201325102E16BEC84F002011E0E316FC0
:10CD700002014E5113E0010101012751400B0EE168
:10CD800002014E0702014E5109E145C100F019862A
:10CD90003582B5ECB5F00201010E346F0201345159
:10CDA00001E177D0020134070201345101E071D072
:10CDB00069EC44F0B6EC45F096EC5EF04EEC92F087
:10CDC00021A204D021926AEC38F054D02CA602D0D3
:10CDD0004AEC2CF019EC90F046EC15F0E5EC1CF068
:10CDE00025AC0DD025A806D0010E696EE66A61EC6F
:10CDF0003BF0E552696AE66A61EC3BF0E552259C3E
:10CE0000696A01018BAD07D001018B9D010EE66EB1
:10CE10002CEC5FF0E552E9EC18F0640EE66E35ECB0
:10CE200029F0E552010178B71ED00701F1051BE09A
:10CE30003550020B18E125A80DD0010E696E8FEC5C
:10CE40003CF0000907E1480E006E5AEC2EF001019B
:10CE5000320E1F6F696A8FEC3CF0000904E1480E46
:10CE6000006E5AEC2EF0BBECC3F01CA603D0BBEC5A
:10CE700032F01C9619B008D0E1EC2AF07DEC56F0A7
:10CE8000E66A48EC22F0E5521990020117894CEC51
:10CE900005F00201495106E002014907020149512A
:10CEA00001E126820201355102E00201350702014B
:10CEB000415102E0020141070201335102E0020147
:10CEC000330702012C510AE002012C0702012C5108
:10CED00005E1780EE66E67EC18F0E55202012B5181
:10CEE00007E002012B0702012B0502E1A1EC12F081
:10CEF00002013E5102E002013E07120006014F6BA3
:10CF00004FC64EF64FC64DF64FC64CF64FC64BF6C3
:10CF1000120069ECEFF0DE52010EDD6EFE0EDB500A
:10CF200022E185ECF2F0050EE66E200EDF24E66EBF
:10CF30004B0EE66E060E30ECE5F026A406D0FF0E92
:10CF400006014B5D0FE1DADF0DD0050E80ECF4F049
:10CF5000B50EE66E010E30ECE5F00F0E89ECF0F048
:10CF60000050DF6E0A6A26B44BD00101B551630848
:10CF700007E3B5510FE10301E3510101B65D0AE298
:10CF80003E0ECCECF3F0FE0EDB5001E1B7DF010EFC
:10CF9000DB6A22D0FE0EDB501FE12D50800B07E034
:10CFA000DF500A0804E20701EF9BE1EC09F0DFCF54
:10CFB000E6FF11EC43F0E55201018B51100B0CE040
:10CFC0000A0E455D09E2A2EC93F09EECE7F0DFCF9C
:10CFD000E6FFEDECA3F0E5520201395111E1640ED8
:10CFE0000101455D07E2A1ECE5F045C13FF05FECD2
:10CFF000EBF005D04D0E196F030E4515310F1A6F6A
:10D00000016A050E015C31E20150EA6A4B0FE96EDC
:10D01000060EEA22EF504B6A120F4A6E070EB7EC6B
:10D02000EFF0026E2D0E025C05E10101B05102E14C
:10D03000200E026E0201395116E1020E0124A4EC09
:10D04000E5F002C0EFFF26A404D00101610E196FC4
:10D050000AD0015008E12C9A2A0E025C04E12D50FE
:10D06000800B01E02C8A012ACCD72650040B05E165
:10D070000201395102E101011B8F010EDB50E1EC8D
:10D08000EAF002E2E16AE552E16E4A50FFEFE4F0B5
:10D0900071ECEEF0016E4551B0ECE6F0050EE66E77
:10D0A0004B0EE66E060EE66E200E0124D1EFF4F074
:10D0B0003450400B04E00101D951800B09E1345098
:10D0C000400B04E10101CD51400B02E1000E01D003
:10D0D000010E3CEFE9F034AC03D00101D98F12000E
:10D0E0000101CD8D120034AC03D00101D99F120093
:10D0F0000101CD9D1200D8EC09F00101076F020E6D
:10D10000075D01E10707B5ECEDF0EFCF06F1065141
:10D110001F0801E2066B0490CDBD0480695003E056
:10D120000490D9BF04801200CEEC0CF0EFEC1FF09D
:10D13000E2DF300E016E0450010B1AE00701EF51DF
:10D14000010B16E0030E0C5C13E0C5ECF3F0080BCA
:10D1500008E0F3ECF0F004E61F0E4A5C000E4B58BA
:10D1600007E206C1E6FFE90E0FECE5F0310E016EB5
:10D17000015012ECE5F09CDFF3501596E8B01586EF
:10D180001200AEEC93F0110EE5ECE8F0B4DF010113
:10D1900006510F0802E26D0E1B6F065113ECEFF003
:10D1A000310F1D6F030E0615310F1F6F94EF68F0DE
:10D1B000248E2096006845EC2EF0C1EF68F0249E86
:10D1C00004EC0EF034AC02D084ECEEF012003450DB
:10D1D000400B04E00101D951010B09E13450400B2F
:10D1E00004E10101CB51200B02E1000E01D0010E40
:10D1F0003CEFE9F0A0ECE8F0EF04016EC3ECEAF0DC
:10D2000001C03FF0BCECFDF03B50026EC3ECEAF015
:10D2100001C03FF0FAECF0F0036E04900101CBBBCB
:10D220000480695003E00490D9B10480110EE66EC9
:10D23000430E02248FECE5F0E66EA90E2BECE5F030
:10D240004A0E03248FECE5F058ECF2F00450010B89
:10D2500002E0012802E1000E01D0010E000902E007
:10D26000370E01D0360E58ECF2F0006A02B004D04E
:10D2700003280E0DF350006E0050E66EA30E0FEC67
:10D28000E5F0100E4A6E8EECE8F04A50EF1622A838
:10D2900032D0DA0E4B6EEE0E4C6E010E4D6EEDEC92
:10D2A000E7F0EF044E6E4F6A506A4B504E24F36E17
:10D2B0004C504F20F46E4D505020FAECEFF0080027
:10D2C000F5CF4AF08EECE8F04A50EF120450010B13
:10D2D00004E0EDECE7F0EF5002E1000E01D0010EAA
:10D2E0004A6E8EECE8F067ECEBF0DF0EEF14F31013
:10D2F000EF6ECAEC0EF06BDFF3501594E8B01584B6
:10D3000004B002D00501446B1200A2EC93F0170E9A
:10D3100086ECE6F0A0ECE8F0EF5006E151ECEFF01F
:10D320000E0E86ECE6F010D0A0ECE8F0C5ECF2F0C2
:10D330003F280101166F0E0E176FC3ECEAF0FDECEB
:10D34000E7F03B280101186FAEEC93F0910EDCEC96
:10D35000E8F022A823D00101030E016FEDECE7F005
:10D36000EF5003E10107A60E17D0EDECE7F0C5EC96
:10D37000F2F03B50310F01011F6F1F5102E1630EAC
:10D380001F6F070E005C02E23E0E06D00E0E005C20
:10D3900002E2410E01D0440EDCECE8F043EFECF089
:10D3A000308A00ECE7F0209685EF69F0309A04ECC3
:10D3B0000EF034AC02D084ECEEF01200A2EC93F04C
:10D3C000050E0C5C1BE10101030E006F020EE66E00
:10D3D000710E0301A7254C6E070EA8214D6E0201A8
:10D3E000B251E82482ECEFF043ECEAF015EC2EF0B9
:10D3F000040E7EECF3F00101188F29D0030E0C5CB3
:10D400001AE181ECE7F009E0220E49ECF0F086EC3D
:10D41000E6F0B30E86ECE6F01AD06CECEEF001010B
:10D42000006F15EC2EF00101100E146F15510FE175
:10D43000100E156F0CD0E5ECF3F02AC100F083EC70
:10D4400096F00101155102E1100E156F186BAEEC4C
:10D4500093F0AE0E006E81ECE7F002E0B40E006EC9
:10D46000050E0C5C07E1E90E006E0201B4A502D0C6
:10D47000E20E006E0050DCEFE8F0258000ECE7F0F3
:10D4800020969CDF050E0C5C06E0E2EC18F0030E23
:10D49000006E36EC91F01200050E0C5C03E14AECD4
:10D4A00009F004D046EC0AF0E9EC18F0259004EC01
:10D4B0000EF059EF0FF0A2EC93F078501DE0030E40
:10D4C000785C07E11F0E006E010178AD09D03F0EB8
:10D4D00006D02D0E006E010197A102D04B0E006EFA
:10D4E00083EC96F00101115102E1100E116F002B37
:10D4F000A40E006EA8EC2DF0AEEC93F0050E4A6E73
:10D50000EA0E4B6E010E4C6E78504D6E3AECE5F023
:10D51000B6EFE6F0338000ECE7F02096CCDF40EF8A
:10D520004BF0339004EC0EF09EEF6CF0FAECE4F06C
:10D53000F8ECE8F01CE0FE0EDB5002E0350E01D006
:10D54000340E12ECE5F074ECE9F011E02150200B00
:10D550000EE0010E696EF8ECE8F008E0FE0EDB501C
:10D5600002E0350E01D0340E12ECE5F0696AFFEFEF
:10D57000E4F0E66A5DECE9F0A50EC9ECF3F0FEEF2D
:10D58000F1F070ECEFF00701BC51B15D14E1155002
:10D59000100B01E0010E4A6E3450010B4A5C0BE1A6
:10D5A0001550200B01E0010E4B6E3450020B01E0D0
:10D5B000010E4B5C2EE0696AB1C7BCF7349015B818
:10D5C0003480349215BA348215A81DD015AA16D00D
:10D5D000F8ECE8F010E00701B151140D8AECE5F029
:10D5E000C8DF01013CA907D0010E696EF8ECE8F034
:10D5F00001E0BFDF696A010EE66E06D0E66A96DFDB
:10D60000E552330E04D0E66A91DFE552320E73EC38
:10D61000E7F078EFEFF00701B151140D8AECE5F077
:10D620002BEC2EF01CC119F11DC11AF11EC11BF10A
:10D630001FC11CF10101200E1D6F480E1E6F5A0EF6
:10D640001F6F300E195D02E1200E196FC1EF6AF0F5
:10D65000318C2096006845EC2EF00BEF6BF0319C7E
:10D6600004EF0EF0095004E02550080B01E130886A
:10D670000D0E005C03E1AEECF0F009D00A0E005C88
:10D6800003E1B9ECF0F003D0005069ECE6F009508A
:10D6900006E03050100B03E1FA0E096E25861200E9
:10D6A000010E0701D89083378437E806FBE122ACEE
:10D6B00002D0070183810D0E0701855D01E2852BF4
:10D6C0001200229C8650020B01E0228C07017B5144
:10D6D00011E122AC51D07B2B010E836F846B856FDF
:10D6E0003198866F7E51FE0BE8427E257D6F0101E9
:10D6F00024931200010124A33FD0249307017B054A
:10D700003BE122BC2BD031A826D00C0E855D20E257
:10D71000D89084338333000E835D040E845918E25D
:10D720003A0E83254A6E020E842127ECF4F04DEC6C
:10D73000E7F0006E090E005C03E10CEC8AF008D003
:10D74000005006E0610E005C02E3200E005E8ADFFE
:10D7500007017B6B1200318850EF6BF0A1DF31A81D
:10D7600004D00701010E866F06D00701862B865173
:10D770000C0801E27B6B3198120008AE05D0229CA8
:10D780008650020B01E0228C07017B5110E122BC84
:10D7900076D00101249307017C6B08AE70D0020E95
:10D7A0007B277E51FE0BE8427E257D6F12007B05B4
:10D7B0000BE17B2B7EC77DF70101249322AC5FD068
:10D7C0000701080E7B6F1200010124A358D0249397
:10D7D000070E07017B5D47E17B6B22AC41D009500E
:10D7E00004E02550080B01E130887C514D6A3A0F66
:10D7F0004C6E060E4D227F5182ECEFF04DECE7F0BF
:10D80000006E810E005C03E107017F6B20D0800E6B
:10D81000005C04E10701200E7F6F19D00D0E005C43
:10D8200003E1AEECF0F013D00A0E005C03E1B9ECBA
:10D83000F0F00DD00B0E005C02E12A0E06D00A0EAD
:10D84000005C05E0005003E0005069ECE6F0095090
:10D8500009E03050100B06E1FA0E096E2586120021
:10D86000080E7B6F1200080E7B5D04E122AC07D02E
:10D870007B6B12007C917C4322BC7C897B2B120049
:10D88000A2EC93F0810E86ECE6F00C5008E1060164
:10D89000F15105E10101002B640E86EFE6F0E5ECA5
:10D8A000F3F0F1C600F0030E0C5C02E1F3C600F0E9
:10D8B00083EC96F0050EE66E040E13EFE8F0E0DF61
:10D8C000AEEC93F0030E0C5C14E12BECEFF006E0F1
:10D8D000C30E4A6EF20E4B6E010E05D0BE0E4A6E9E
:10D8E000F20E4B6E010E4C6E5FECE5F04CC0E6FFA5
:10D8F0000AD0F60E4A6EE90E4B6E010E4C6EF0C663
:10D900004DF03AECE5F0B6ECE6F049EC26F029EC07
:10D9100012F0006E00500A01D65D04E200C0D6FA93
:10D92000DEECF1F01200318400ECE7F020965FEFBE
:10D930006CF0319404EC0EF09EEF6CF0BCECEDF06A
:10D94000A00E56ECF0F0140E016E3DC100F0FFEF9A
:10D950004CF065ECEFF0E6C64AF0E7C64BF071EC30
:10D96000ECF00601A9ECEEF00BE3E4C64CF0E5C6E2
:10D970004DF00FECEFF0E6514C5CE7514D581FE2D3
:10D98000E451E6250F6EE551E721106ED890103274
:10D990000F32C6ECEAF0030E50ECF2F0FDE14A5013
:10D9A0000601E85F4B50E95B6BECE7F0030E50ECCF
:10D9B000F2F0FDE14A500601E8274B50E923E4C6A6
:10D9C000E6F6E5C6E7F6C6ECEAF071ECECF071ECD1
:10D9D000ECF0A9ECEEF00BE3C6ECEAF029ECE8F091
:10D9E00029ECE8F04A50E45D4B50E55902E2DF6A69
:10D9F00009D0E851E45DE951E55902E2010E01D098
:10DA0000020EDF6EC6ECEAF071ECECF04A50E8254D
:10DA1000EA6F4B50E921EB6FDF50E552FFEFE4F086
:10DA2000229C8650020B01E0228C22AC03D0020122
:10DA3000812B02D00201822B8251EAECE8F001E155
:10DA40004B5008E081514C6E4D6AFF0E4C1822E19C
:10DA50004D5020E18151EAECE8F00DE14B500BE133
:10DA6000805179ECE5F004E6FF0E4A5C000E4B585D
:10DA700005E2802B03D0805101E080070601F151BF
:10DA800005E180C2E6FFE20E0FECE5F00201826BD9
:10DA900082C281F2209E0601EC5109E122AC45D000
:10DAA000010EEC6FE46BE56BED6BEE6B3ED0EC05BD
:10DAB00015E122BC3AD0020EEC6F4BDF006E005035
:10DAC0000BE0070E0601EE5D07E2EE2BED91ED4354
:10DAD0000050010801E2ED8F060119D0020EEC5D45
:10DAE00024E122AC17D0C6ECEAF0030E50ECF2F0C1
:10DAF000FDE106014A50E85D0F6E4B50E959106E8A
:10DB00000F50E45D1050E5590EE2010EEC6FE46B2E
:10DB1000E56B0BD0EA51EA254A6EEB51EB214B6ED7
:10DB2000A9ECEEF002E2030EEC6F030EEC5D68E18F
:10DB3000ED91ED43ED8F070ED880EE55016E01504B
:10DB40000106000903E0ED91ED43F9D7780EED5D94
:10DB500055E2095004E02550080B01E13088EDC67C
:10DB6000E6FF67EC04F0E552006E200E005C03E374
:10DB700000506E0802E22A0E0BD02A8A005069EC8F
:10DB8000E6F00601E451EA5DE551EB5903E2200EAF
:10DB900069ECE6F0040E0601F05D26E12AAA0CD03D
:10DBA000600E3E6E090E3F6EE8C643F0E9C644F0D3
:10DBB00078ECFDF03EC0EFF6E4EC89F0000914E0EB
:10DBC0000101390E1A6F1AC119F16E0E1B6F640E26
:10DBD0000601EF5D07E2A1ECE5F0EFC63FF05FEC78
:10DBE000EBF01A6F01011C8F2A9A095007E03050A0
:10DBF000100B04E12586FA0E096E31860601EC6BE6
:10DC0000208E12000101DF830C5002E109DF07D0F2
:10DC1000209EE9ECEAF002E054DD01D0AEDD010126
:10DC2000DF931200800E081418E02B50020B15E150
:10DC30002150200B12E00201DF510FE10C5004E1F2
:10DC40000601F051010806E3030E0C5C06E12BEC23
:10DC5000EFF003E02A0E18140DE0800E081409E11D
:10DC600017ECE6F006E00601F25103E002013D5137
:10DC700001E0000C010C02014C5103E1120E27ECF3
:10DC8000E5F01200FAECE4F006C201F007C202F07F
:10DC90002DA203D0020EF8ECE7F074ECE9F040E0BE
:10DCA0003851800B3DE1020EF8ECE7F002010A5119
:10DCB00079ECE5F002E670ECE7F015E20A514A6E05
:10DCC0004B6A800EA1ECF1F0036E03504E6E4F6A6A
:10DCD000025023ECE6F0070E0F0B03E054ECF2F0D9
:10DCE000FDE14A50025E02010A51F6ECE5F018E24D
:10DCF0004A508008000E4B5413E20A5182ECEAF0BD
:10DD00004A50036E03504E6E4F6A015023ECE6F00A
:10DD1000070E0F0B03E054ECF2F0FDE14A50015EF8
:10DD200069CFC7F2696AFE0EDB0409E00150E66EB6
:10DD3000A60E0FECE5F00201188335B09CDFFE0E55
:10DD4000DB5009E00250E66EBF0E0FECE5F0020179
:10DD500018851DB890DFC7C269FFFFEFE4F059ECEA
:10DD6000F0F004E24CECE8F001E2006A59ECF0F06B
:10DD700007E24A50E308000E4B5402E2E30E006E45
:10DD80000050AEECEEF00024006E59ECF0F005E22D
:10DD90004CECE8F002E2FA0E006E12001BECF1F01F
:10DDA0002C51615D03E1785041ECF0F09EEF6CF096
:10DDB000A5EC0DF0B9EC25F0DEECF1F0E5EC1CF093
:10DDC00069ECECF02050020B05E0E9ECEAF002E02F
:10DDD00096ECEBF0B3EC4BF04CEF05F065ECEFF0AC
:10DDE000DFEC13F099EC5FF021AA07D00301E651B4
:10DDF00002E0E60702D0ECEC92F014DF000902E04A
:10DE000001DF01D0209E2550200B06E00201345195
:10DE100003E196EC5EF0259A5BECE8F012E03450FA
:10DE2000400B0FE10101CB51200B0DE005014051EA
:10DE30000AE08450040B07E1445105E1280E446FC9
:10DE400002D00501446B02013B5102E069EC51F044
:10DE50000101B15112E12850010B0FE15BEC34F0EC
:10DE6000006E1EAC80EF78F00701D351F00BE83A5A
:10DE7000D35D0024D36F80EF78F0B1051FE1285007
:10DE8000010B1CE184EC8BF053EC2FF05BECE8F021
:10DE900002E180EF78F05FECE8F002E180EF78F0EB
:10DEA0002D50400B02E080EF78F02D50800B02E007
:10DEB00080EF78F0ACEC2EF080EF78F0020EB15DE0
:10DEC00009E12850010B06E14BEC14F0D1EC93F082
:10DED00080EF78F0030EB15D07E12FB480EF78F0AA
:10DEE000D6EC97F080EF78F0040EB15D01E0B9D088
:10DEF0000201355102E080EF78F01750100B03E17A
:10DF00001750010B02E0000E01D0010E2390E8B083
:10DF1000238022AA4ED0B2ECE9F0166E23A036D0B0
:10DF20000101A6511EE1165002E1010E01D0100EB2
:10DF30008009176E2850010B03E10E0E675C05E1A6
:10DF40000201030E286F640E226F28A004D0480E31
:10DF5000B1ECEEF03FD0FBEC09F000093BE01B8494
:10DF600039D0165003E00C0E165C34E1810E176EAA
:10DF7000165001E1229A0201020E356F28A003D04B
:10DF8000540EB1ECEEF00201286B24D0165022E1C1
:10DF90002350010B1FE1229A2850010B06E00C0EC2
:10DFA000675C03E1520EB1ECEEF00201020E356F38
:10DFB00011D032B40FD0E66ACEEC51F0E552000930
:10DFC00009E032840201020E356F640E416FDF6B8F
:10DFD00008AE356B3250040B02E180EF78F002019D
:10DFE000355102E080EF78F03294B2ECE9F0166E31
:10DFF000165002E180EF78F00101280EA66F2A0E7C
:10E00000165C05E12150400B02E01E0EA66F0A0EC1
:10E01000165C09E0090E165C06E0120E165C03E0C1
:10E02000110E165C02E12D0EA66F350E165C02E194
:10E03000FA0EA66F0201020E356F228A176A165079
:10E04000676E28B005D0FBEC09F0000901E01B84E5
:10E0500029B602D00101A96BA5EC0DF02B8480EF4D
:10E0600078F0050EB15D0FE12751100B05E1285145
:10E07000100B02E169EC51F028A080EF78F057EC2A
:10E0800058F080EF78F0060EB15D07E121AA80EF2D
:10E0900078F021EC08F080EF78F0070EB15D01E038
:10E0A000B7D12650800B18E00201385115E1B6ECCB
:10E0B000EEF002011E0E386F269E2850020B0CE077
:10E0C0002A50010B09E1510E69ECE5F0300E69ECC4
:10E0D000E5F0010EC4ECF0F026AC03D062ECE9F000
:10E0E000269C26AA03D046EC0AF0269A0101375155
:10E0F000800B1BE00201485118E11BA404D0040E60
:10E100003BECF1F01B941BA604D0070E3BECF1F0A6
:10E110001B961BA804D0060E3BECF1F01B981BAA23
:10E1200004D0050E3BECF1F01B9A2250080B02E0E4
:10E1300080EF78F02B50400B02E080EF78F0020186
:10E140000B5139E1D70EFAECE5F01F9A1FB01F8A88
:10E15000E66801C2E6FFCBECEAF00201016F1F9016
:10E160001FBA1F801F50100B04E10101E151080B81
:10E1700022E028A006D001C2E6FF470E47ECECF0F3
:10E1800019D001C200F00101E1A703D0DDC300F006
:10E19000E197030E005E59ECF0F004E24CECE8F07D
:10E1A00001E2006A00C006F238BF02D000C007F2E8
:10E1B000E66A68DDE55202010B0548E1CF0EFAEC94
:10E1C000E5F01F9A1FB21F8AE66802C2E6FFCBEC99
:10E1D000EAF00201026F1F921FBA1F821F50100B3C
:10E1E00004E10101E151100B31E028A006D002C288
:10E1F000E6FF480E47ECECF028D002C200F0010127
:10E20000E1A903D0DEC300F0E199030E005E59ECF2
:10E21000F0F004E24CECE8F001E2006A00C00AF21F
:10E2200038AF06D00201800E0A6F00C007F20AD094
:10E2300059ECF0F007E24A50E308000E4B5402E2BA
:10E2400002010A69010EE66E1DDDE552020E0201B1
:10E250000B5D45E1E70EFAECE5F01F9A1FB41F8A4B
:10E26000E66803C2E6FFCBECEAF00201036F1F94FD
:10E270001FBA1F841F50100B04E10101E151200B54
:10E280002EE028A007D003C2E6FF490E47ECECF0D1
:10E29000E55225D003C200F00101E1AB03D0DFC39A
:10E2A00000F0E19B030E005E5ADD00C008F2005052
:10E2B00089ECE8F0006ED9ECEAF00AE208C209F253
:10E2C0000050E66EA70EADECEBF00201188905D008
:10E2D00069CFC7F2696A2EECF2F002011887030ECB
:10E2E00002010B5D01E08AD0EF0EFAECE5F01F9A17
:10E2F0001FB61F8AD9ECEAF009E29E0EE66E05C24F
:10E30000E6FFCBECEAF00201056F07D0E66804C235
:10E31000E6FFCBECEAF00201046F1F961FBA1F86DE
:10E320001F50100B04E10101E151400B67E028A0F0
:10E330000CD0D9ECEAF003E205C2E6FF02D004C239
:10E34000E6FF4A0E47ECECF038D0D9ECEAF037E2C1
:10E350004CECECF005C200F00101E1AD03D0E0C3EC
:10E3600000F0E19D030E005C0701056F0551F6EC1E
:10E37000E5F004E24CECE8F001E2056B0539E84613
:10E380001F0B056F05511D0802E21D0E056F050EDE
:10E390000C5C03E0050E7D5C03E18DEC0CF02ED0EF
:10E3A0002150200B2BE00201415128E1010157BD12
:10E3B00025D0130EE66E6FEC2EF0E5521FD004C28E
:10E3C00000F0E1AD03D0E0C300F0E19D030E005E7C
:10E3D000C6DC59ECF0F004E24CECE8F001E2006A33
:10E3E00000C009F2005089ECE8F0006E69CFC7F276
:10E3F000010E696E2EECF2F002011889030E020183
:10E400000B5D01E12D920B2B030E0B1780EF78F0C3
:10E41000080EB15D02E0E0EF76F02850010B02E05B
:10E42000E0EF76F018BC3DD118A8E0D021AE0FD0B7
:10E43000A85101E0F4D02CA805D0CFC1E6FF9CEC98
:10E4400053F003D0E66AFDECC5F0E552E8D025A014
:10E450003CD027AD7DD016EC09F00C500DE1500EEC
:10E46000E66E1E0EE66E2A0EE66E010E21ECE5F05B
:10E470000101B9ECEEF01CD081ECE7F009E0030EED
:10E48000E66E2F0EE66E010EE66E27EC9DF00DD0C7
:10E49000050E0C5C0DE1330E5FECF4F0B20EE66E8F
:10E4A000020EE66E1DEC9DF0E552E552E552E55296
:10E4B0003DEC6AF0DEECF1F0E5EC1CF002010A0E36
:10E4C0003C6F05013B853B8F43D033A018D027AD6F
:10E4D00013D081ECE7F003E00101977105D0E9EC7E
:10E4E000EAF002E00101787DA5EC0DF0B9EC25F031
:10E4F00049EC26F05BEC6AF00101279D5FD031A466
:10E5000016D027AD25D016EC09F00C5006E1060E0A
:10E51000E66EF10EE66E060E05D01E0EE66EF30EEA
:10E52000E66E060E1CECE5F05FEC6CF011D030AA44
:10E5300011D027AD0DD016EC09F0150EE66E69501E
:10E540004B6A420F4A6E050EE6ECEFF085EC69F07F
:10E55000010134D02D50400B03E12D50800B30E0F1
:10E5600027AD5DD016EC09F00101B0511AE1630E40
:10E57000E66E450EE66E010E06ECE7F045C11FF2B1
:10E5800002014E6BE0ECE8F0000917E02D50800B23
:10E5900014E001018F51100B10E10201100E4E6FBB
:10E5A0000CD0290EE66EB0054B6A4B0F4A6E060E74
:10E5B000E6ECEFF0BEECEEF0E5520101A86B2FD0D7
:10E5C00029A20DD027AD2BD016EC09F0E6686A0E13
:10E5D000E66E030E1CECE5F070ECC5F020D022B620
:10E5E0001ED06FC200F03BEC2EF019D018A205D05F
:10E5F00026A215D02692238212D018A010D026A2CF
:10E6000006D026922CC1E6FF11EC43F0E552020140
:10E61000315105E11B50400B02E140EC4BF01AEC8C
:10E6200016F0006EFF083DE0420E005C03E0450E70
:10E63000005C15E129C70FF02AC710F0450E005CF9
:10E6400004E107012B510F6E106A00683BEC2EF0BD
:10E650000101150E116F030E006F15EC2EF05D0E0B
:10E66000005C16E10101150E116F100E126F020E03
:10E67000006F2CC7E6FF06EC2EF0E5522DC7E6FF33
:10E6800006EC2EF0E5522EC7E6FF06EC2EF0E55222
:10E690007E0E005C06E1A2EC93F0E80E006E3BEC0F
:10E6A0002EF018BE73D318AAA5D12DA603D09EECC8
:10E6B00054F054D32DA403D06CEC54F04FD331A4B8
:10E6C00025D0010128AD17D0010E0E6E28BF0E68AF
:10E6D0000C5005E1BCECEDF027EC9DF008D0010EEC
:10E6E000E66EF20EE66E060EE66E17EC9DF0FCECA2
:10E6F000F3F0DEECF1F02450200B05E1010128518C
:10E70000400B01E184D05FEC6CF081D033A01ED0CF
:10E71000010128AD0DD0010E0E6E28BF0E6878CF16
:10E7200006F1030ED5ECF4F006C178FFCEEC6EF0E6
:10E730002450200B04E101012851400B68E0D8EC83
:10E740006EF05BEC6AF00201198161D025A00CD05B
:10E75000010128AD46D10201B47540EC4BF03DEC0F
:10E760006AF00101289D3DD130AA1AD0010128ADDF
:10E770000DD0010E0E6E28BF0E68150EE66E6950A4
:10E780004B6A400F4A6E050EE6ECEFF02450200B6A
:10E7900004E101012851400B3AE085EC69F037D0E3
:10E7A00024AE1AD0010128AD0ED0010E0E6E28BF86
:10E7B0000E687BEC68F01F0E5BECF4F00101B5EC29
:10E7C000EDF006C1EFFF2450200B03E12851400B70
:10E7D0001EE0C1EC68F01BD031AC1DD0010128ADAA
:10E7E0000DD0010E0E6E28BF0E68C40EE66E0A0E26
:10E7F000E66EB10EE66E070E21ECE5F02450200B1C
:10E8000004E101012851400B02E00BEC6BF0010127
:10E81000289D249AE6D02D50400B03E12D50800B0B
:10E8200034E024AA04D0249ABEECEEF061D00101B9
:10E8300028AD94D2289D010E0E6E28BF0E68006A86
:10E8400026B4002A050E27ECEFF0B00EE66E010E9E
:10E8500021ECE5F00601030E426F0101B0510EE01C
:10E86000B0294A6E010E4A5204E0E846FE0B4A0601
:10E87000FCE10601426F1E0E436F02D048EC68F0C7
:10E88000BEECEEF0E5520101ACD029A215D024AACD
:10E8900002D0249A0ED0010128AD60D2289D010E2D
:10E8A0000E6E28BF0E68E668690EE66E030E1CEC5D
:10E8B000E5F070ECC5F052D221AE1CD00101A85198
:10E8C00001E04CD2CFC101F023A802D0DCEC82F0F1
:10E8D000006A2C50100B05E133ECEFF002E2010E60
:10E8E000006E0050E66E0150E66ECCEC53F0E5523F
:10E8F000E55234D21CA277D0AEEC93F0140EE5ECC6
:10E90000E8F0AEEC04F05A0ED8800054006E0050CF
:10E91000036EA0EC96F00101200E1D6F0201F15173
:10E92000035C03E201012A0E1D6F010128AD58D0DE
:10E93000289D9EEC0AF0E4EC0AF0190E026E01012B
:10E94000DFAF02D01A0E026E28BF09D06E0E020190
:10E950004A5F000E4B5B0250BAECF1F008D06E0E2D
:10E9600002014A27000E4B2302508CECF1F04A5171
:10E970004B1106E0280ED8804A55230E4B5519E25C
:10E98000010128BF0AD00201280E4A6F230E4B6FE7
:10E99000EFC20FF0F0C210F00CD06E0E02014A6F01
:10E9A0004B6B025093ECE7F0EF5D0F6E4B50F0595C
:10E9B000106E0301D2510F5CD351105804E2D651AE
:10E9C0000F26D75110220F50D45D1050D55904E2B4
:10E9D000D6510F5ED751105A10ECECF00EEC0BF044
:10E9E0000101A86BBBD122B6B9D170C200F045ECD1
:10E9F0002EF0B4D118B2B2D118A616D0AEEC93F066
:10EA00000A0E006EBDEC2DF00101040E016F03C76C
:10EA100000F01AAC02D0AEEC04F0A0EC96F01AAC08
:10EA20009DD10101200E70D149ECEFF001E17ED1C2
:10EA30002E50400B01E07AD1060E006E2BA502D0BD
:10EA40000A0E006E0050D880775501E2776B28AD32
:10EA50001FD0289D010E0E6E28BF0E680050E66E76
:10EA6000770EE66E010E1CECE5F0050E0101775DF8
:10EA70000BE12B50200B03E02B50010B05E028BFCE
:10EA800002D0772B01D077070201FC6B0101A86B44
:10EA9000A85101E063D12150200B01E15FD10201B7
:10EAA000DF5101E05BD10A0E0101775D3FE1AEEC81
:10EAB00093F0C3EC18F001012B0E196F000110AE9A
:10EAC0000BD001012D0E196FFF0ED8800F56105676
:10EAD000010E0F26000E1022E70E90ECEEF004E27D
:10EAE000E70E0F6E030E106E0F50101003E10101C0
:10EAF000200E196F6BECE7F0640EA4ECF2F04A50B4
:10EB0000006E0101012BA0EC96F0A4EC04F0300F94
:10EB100001011A6F300E1A5D02E1200E1A6F1C8F70
:10EB2000640E1D6F420E1E6F560E55D0090E775D96
:10EB30001EE1AEEC93F0B7EC18F02BEC2EF00101D7
:10EB4000410E196F460E1A6F560E1B6F300E1C5D6C
:10EB500001E004D1200E1C6F300E1D5D01E0FED0DF
:10EB60009FECEEF001E0FAD0200E1E6FF7D0050EFC
:10EB7000775D03E0060E775D30E1AEEC93F00101C6
:10EB8000500E196F410E1A6F050E775D03E1DDC758
:10EB900000F006D0460E196F500E1A6FE0EC14F01C
:10EBA00000AE04D0006C01012D0E1B6F0101030E9D
:10EBB000016FA0EC96F0300E01011C5D0BE11BC152
:10EBC0001CF1200E1B6F300E1D5D04E11CC11DF1F8
:10EBD000200E1C6F430E1F6FC1D0070E775D04E03F
:10EBE000080E775D01E077D0AEEC93F00101500E96
:10EBF000196F4C0E1B6F1BC11AF1310E1C6F69CFC0
:10EC0000C7F2070E775D02E1696A03D01C2B010E83
:10EC1000696E8FEC3CF0C7C269FF010178A73BD059
:10EC2000AEEC93F0B60EE66EF20EE66E010EE66EF8
:10EC3000B6ECE6F0080E0101775D01E11C2B69CF0F
:10EC4000C7F2696A080E775D02E1010E696E530E24
:10EC500065ECE9F0005003E10201FC5119E00050BD
:10EC600006E00201FC51005C02E000C0FCF2010180
:10EC70002A0E1D6F0201FC390F0B51ECECF0010163
:10EC80001E6F0F0E0201FC1551ECECF001011F6F1D
:10EC9000C7C269FF63D00050150D8AECE5F06BEC3C
:10ECA000E7F0060E50ECF2F0FDE14A50006E005025
:10ECB000DF6E0201345152E1ADECE9F00101200EAA
:10ECC0001D6FDF50480803E3040EDF5C02E22A0EEA
:10ECD0001D6F1F8F43D0020E775D05E1F7EC52F0F8
:10ECE000010E096E3BD0030E775D10E1AEEC93F0A0
:10ECF0001EC200F0A0EC96F0300E0101195D02E199
:10ED0000200E196F1B8F560E1D6F28D0040E775DD5
:10ED100003E1BDEC12F022D0775103E168ECC4F0BE
:10ED20001DD077051BE198ECC4F018D002012A51E0
:10ED30000AE02850400B12E1140E095C0FE2810E2C
:10ED400098ECE5F00BD018A009D024AA03D0249A9F
:10ED5000BEEC43F02EAC02D040EC4BF01AEC16F0B7
:10ED6000006EFF0813E07E0E005C0CE1006845ECCD
:10ED70002EF0AE0EE66EF20EE66E010EE66EB6EC0C
:10ED8000E6F004D00050006E45EC2EF00101A851D1
:10ED900001E0B6D1140EA86F02016B5101E06B07C0
:10EDA000020E6F5C01E0ACD1CD0E0B5C07E0B30E40
:10EDB0000B5C04E0A10E0B5C01E0A2D12682A0D185
:10EDC000090EB15D03E115EC51F09AD10A0EB15D67
:10EDD00008E12850010B05E188EC95F06BEC95F00B
:10EDE0008FD10B0EB15D01E08BD12850010B01E0FA
:10EDF00087D1B25110E1BFEC14F09050800B01E1CB
:10EE000079D19050400B01E175D1909C1E0EE66EB9
:10EE1000F7EC15F06ED1B20511E1800E08140BE18C
:10EE20003951040B01E066D12C51070804E282EC51
:10EE3000E6F001E05FD10BEC05F05CD1020EB25DB3
:10EE40004AE11BEC14F00701DC0ED880DB55000E04
:10EE5000DC5501E34FD182ECE6F001E14BD1DBC799
:10EE60000FF0DCC710F0016A030E015C09E21BEC35
:10EE700014F00701DB510F26DC511022012AF4D7D0
:10EE8000020E0F0B05E0D89010320F32E806FBE1BE
:10EE9000DC0E7DECE6F001E32DD1A70EE66EF20E5E
:10EEA000E66E010EC3ECEDF0010E006EF00E7DEC8F
:10EEB000E6F002E2050E006E33ECEFF004E20050E3
:10EEC000495FD7ECE8F0780E0101495D01E312D10A
:10EED00083EC0FF00FD1030EB25D03E16CEC0FF089
:10EEE00009D1040EB25D39E121AC0CD03250010BD6
:10EEF00009E002018851070805E21450080B02E0FE
:10EF0000640E436F2150400B01E0F4D002013B51ED
:10EF100001E0F0D001015751200B01E0EBD0F00EE1
:10EF20008C1625AE287E28AE02D0030E8C1267EC1C
:10EF30000CF000090DE067EC0CF0000909E067EC4B
:10EF40000CF0000905E0258E150E27ECE5F002D047
:10EF500025BE259EF00E8C16CDD0050EB25D34E197
:10EF6000060150932550020B12E12050020B04E0E1
:10EF7000C0EC31F0000909E01350080B03E1135015
:10EF8000040B05E02BECEEF002E006015083255067
:10EF9000020B01E0AFD01BECEBF001E0ABD00201C3
:10EFA000405101E0A7D0D4ECEBF001E14B5001E17E
:10EFB000A1D02D50800B01E09DD02D50400B01E0E1
:10EFC00099D00601108F96D0060EB25D44E15751DC
:10EFD000040B3FE02050080B3CE0DF0EFAECE5F0BC
:10EFE0002BBC23D0F3ECF0F002E628ECEEF001E3CA
:10EFF00081D01E0E85ECE5F0DF0E70ECF4F0016EB2
:10F00000050E85ECE5F0DF0EFAECE5F0030EE66E9A
:10F01000015027ECEFF0FAECE6F06CE02B8C47ECBB
:10F020000CF002013C0E466F65D059ECF0F00BE29B
:10F030004A50B908000E4B5406E22B9C1E0EE66E99
:10F0400035EC29F056D00201465154E147EC0CF062
:10F0500051D02B9C4FD0070EB25D4CE15BECE8F039
:10F0600049E02150200B46E095ECF4F0C09EF00EF4
:10F070008C160F6A106A01013CB903D0190E0F6E8D
:10F08000106A6BECE7F0FA0ED8804A56000E4B5629
:10F09000C3504A5CC4504B582DE20201EC2BEC519A
:10F0A000030828E2EC6B010158AD07D0589D50ECE5
:10F0B0009BF07CEC1EF0160E19D06950DF6E696A69
:10F0C00002010691064306C2E6FFA60E0FECE5F02C
:10F0D00001013CA908D002010791074307C2E6FFDE
:10F0E000BF0E0FECE5F0DF50696E170EE66E6FECA9
:10F0F0002EF0E5520101B22BB251070801E2B26BCA
:10F100000101B12BB1510B0801E2B16BE552FFEFE8
:10F11000E4F0016A700E015C0EE26A0E4A6EEE0EB9
:10F120004B6E010E4C6E01504D6E88ECF4F000EC0D
:10F13000E9F0012AEFD71200026A300E025C08E201
:10F14000B00E0224016E0A0E00ECE9F0022AF5D797
:10F15000120065ECEFF07A0EDCECE8F068EC95F06C
:10F16000010E0A6EDF6A100EDF5C35E2026A100ED5
:10F17000025C2FE264ECF0F003E0050E025C06E1B5
:10F18000DF50E824860F8FECE5F0006E020403E008
:10F19000060E025C07E1DF50E824860F010F8FECBA
:10F1A000E5F0006E020EDF5C06E3030EDF5C03E0B9
:10F1B0000A0EDF5C0AE10A0E025C02E1110E006E2B
:10F1C0000B0E025C02E1240E006EFFEC4CF0022AF2
:10F1D000CED7DF2AC8D7AC0E016E580E00ECE9F08E
:10F1E000020E0A6EDF6A090EDF5C12E2026A100E7E
:10F1F000025C0CE264ECF0F003E0050E025C02E15C
:10F200001C0E006EFFEC4CF0022AF1D7DF2AEBD780
:10F210000A6A7FDFDF6A200EDF5C09E2100E006EF3
:10F22000800EDF24016EFFEC4CF0DF2AF4D7DF6A9A
:10F230000B0EDF5C03E280DFDF2AFAD7DF6A090EFC
:10F24000DF5C31E2DF28006E0038F00B006E090E43
:10F250000012DFCFE6FFF7EC0BF0E552CBECF2F05B
:10F26000EE52090EBEECF3F015ECECF02C0EBEECF9
:10F27000F3F0030E2DECF0F0010EBEECF3F0040EF3
:10F28000E7ECF0F0050EE7ECF0F0070EE7ECF0F03D
:10F29000080EE7ECF0F0060EE7ECF0F0090ED3EC08
:10F2A000E8F0DF2ACCD718D822D8DF6A060EDF5C58
:10F2B00007E2DF50FDECE5F0010EEF6EDF2AF6D736
:10F2C00063ECF4F0FD0E016EDB0E00ECE9F0010ED4
:10F2D000186EE552FFEFE4F0020E0A6E5A0EE66E6B
:10F2E000000EE66E030EE66EA20ED1EFF4F0730E82
:10F2F000DCECE8F068EC95F0140E45ECEFF0000E55
:10F30000E66E0A0EF1ECE5F00A0E45ECEFF0CA0EDF
:10F31000E66E0A0EF1ECE5F00C0EE66EE66A010E02
:10F32000E66E140EE66E0A0EF1ECE5F00A0E45EC00
:10F33000EFF0200EE66E0A0EF1ECE5F00A01D46B58
:10F34000DA6BDA81D56B380ED66F040ED86F3C0EAF
:10F35000D96F190ED76F016A020E015C0CE20150E1
:10F36000050D82ECF3F0000EE9260A0EEA22360EB5
:10F37000EF6E012AF1D70C6A050E0C5C1AE2070148
:10F38000010EE26FFF0EE25D12E0BEEC15F0F2EC52
:10F39000ECF0C3ECF1F00C5097ECF1F00701E25106
:10F3A00044ECF4F0C3ECE7F00701E207EBD70C2ADA
:10F3B000E3D70701E26B0C6A17EC5FF020EC5FF01B
:10F3C000030E0A6EFE0E016E810E00ECE9F00A6A71
:10F3D0001200240E01013F03F350E66EE66A86EC4C
:10F3E000FBF0E552E552640E0101D8804155E82456
:10F3F0000A0FE66EE66AB5ECFBF0E552E5520C0E3C
:10F40000BD6E006A01013F510AE0020E40253F0334
:10F41000F3504A6E4B6AFF0EA1ECF1F0006E005003
:10F42000BE6E1200FAECE4F094ECE5F0B2ECFCF005
:10F43000E552000902E0C69EF7D7FFEFE4F0C79E51
:10F44000C698C78C1200C78EC688C78C120096EC6F
:10F450005EF02DA003D0210E9CECE5F007010B8798
:10F4600096EC5EF096EC5EF096EC5EF007010B9782
:10F470002DB003D0270E9CECE5F096EC5EF0070172
:10F480000B8596EC5EF007010B952DA002D00101D3
:10F49000E38996EC5EF00701128596EC5EF00701B9
:10F4A00012952DB003D0330E9CECE5F096EC5EF097
:10F4B00007010F8F96EC5EF007010F9F2DB00DD066
:10F4C0000F8B96EC5EF007010F9B2DA003D001017E
:10F4D000E38B03D0240E9CECE5F096EC5EF0070184
:10F4E0001F8996EC5EF007011F9922882DB003D08A
:10F4F0006C0E9CECE5F096EC5EF001012BA11FD0A8
:10F500000701108796EC5EF0070110972C842DA060
:10F5100004D0010178AB11D00DD0010178AB0AD035
:10F520000701108F96EC5EF00701109F0101E28148
:10F530002DB003D0630E9CECE5F096EC5EF001017B
:10F540002BA70ED007010D8796EC5EF007010D97F3
:10F5500020802DB003D02A0E9CECE5F096EC5EF0F6
:10F5600001013B510EE00701168196EC5EF00701A8
:10F5700016912C862DB003D0660E9CECE5F096EC2F
:10F580005EF001013A510EE00701138F96EC5EF038
:10F590000701139F2B8A2DB003D0690E9CECE5F078
:10F5A00096EC5EF0010138A73BD02588070107855E
:10F5B00096EC5EF0070107952DB003D02D0E9CEC64
:10F5C000E5F00701068396EC5EF00701078396ECF1
:10F5D0005EF0070107930101E9932DB0E98396ECF2
:10F5E0005EF0010160A50ED00701098796EC5EF080
:10F5F0000701099731822DB003D0300E9CECE5F065
:10F6000096EC5EF00701208996EC5EF007012099E8
:10F6100031802DB003D06F0E9CECE5F096EC5EF0DF
:10F6200096EF5EF0BEECF1F0020EDB6A81EC12F0B8
:10F630000F0EC16E040E0701042704070407040718
:10F6400004078D8C219A34860201800E8A6FD3ECD8
:10F6500015F00601BA6B800EBB6F40EC0EF00A6A23
:10F66000FB0EBDECE5F000C0F1F707010E6B0F6B70
:10F67000126B206B20C71FF7470E186F18C717F7BC
:10F680000201A069A1690701010E066F076B96ECE4
:10F690005EF096EC5EF00301310EE36F0701090E98
:10F6A000326F32C731F732C730F732C72FF7070E44
:10F6B000516F0301A00ED06F0F0ED16FE50EE66EF5
:10F6C00091ECFCF0E552E668E4ECFBF0E552E6680C
:10F6D0004EECFCF0E552E6682CECFCF0E552050E31
:10F6E000E66ED0ECFCF0E552B5ECECF072DE850E87
:10F6F000E66E70ECFCF0E5520201320E256F000E52
:10F70000A56EA26E9F6EA282D08EE66A040EE66E91
:10F71000210EE66E1DECFBF0FCECF3F0010EDB6A53
:10F72000100E36ECE5F018E23C0E4A6EEF0E4B6E12
:10F73000010E4C6E010EDBCF4DF088ECF4F0E66E5E
:10F74000010EDB50EA6AC90FE96E060EEA220EECE2
:10F75000E6F0010EDB2AE4D70101276B27918850E0
:10F76000010B01E0278127938850020B01E02783DA
:10F7700028918850200B01E0288128938850100B95
:10F7800001E02883E987F28E0601526952C650F6DD
:10F7900015EC51F071EC98F00101D1ECF2F006019A
:10F7A000526B52C650F615EC51F0010E186EA2ECD9
:10F7B00093F0AEEC93F0F5EC89F00601178F4169F8
:10F7C00041C640F6426B148A138012881282148656
:10F7D00014880A01380ED66F010ED76FC5EC1EF0E3
:10F7E0006BEC95F0B2ECE9F0166E380E165C06E1A3
:10F7F00001013989B2ECE9F00009FCE1C80E78ECAE
:10F80000E6F00701D76B358EB1ECF2F0E66E7EECD8
:10F81000EAF0359E40EC0EF00A6A20ECF0F0DF5082
:10F82000005C02E0180E09D0830E0A6E20ECF0F0A6
:10F830000A6ADF50005C04E01B0E9CECE5F033D05C
:10F84000FD0EBDECE5F0DB0E005C03E13A0E165C4C
:10F8500005E17FDC010E64ECE6F01ED0020EBDEC8B
:10F86000E5F000C02BF1370EBDECE5F000C060F113
:10F87000110EBDECE5F000C03AF1120EBDECE5F062
:10F8800000C03BF10F0EBDECE5F000C038F14F0EAB
:10F89000BDECE5F000C078F1B00EBDECE5F0005035
:10F8A000800801E249DC010E696EE66E61EC3BF016
:10F8B000E55281EC36F0E5C2E6FFE6ECE7F0696A76
:10F8C000C5ECEBF081EC36F0E4C2E6FFE6ECE7F0E5
:10F8D000010138B711D0E66ACFEC18F0E552040EFA
:10F8E000AAECEAF0010E78ECE6F0E66ACFEC18F04C
:10F8F000E552280E78ECE6F032880701580E8F6F3B
:10F90000020E906FBC69A5EC0DF0FFEC23F0010135
:10F9100038A707D056ECECF0FFEC23F0696AA5ECB1
:10F920000DF096EC5EF0F29EC2EC4EF00201006F1C
:10F93000000910E0C80E78ECE6F0C80E78ECE6F0AE
:10F94000C2EC4EF00201006F000904E07E0E9CEC58
:10F95000E5F03582A8EC98F00701F10512E003010B
:10F96000010ED96FDB6B73DD0301DB5103E0C80EC1
:10F9700078ECE6F00301DB5104E0D92B040ED95DED
:10F98000F1E3D9C3DAF30301D96BF28E2A9E2BBAC5
:10F990002A8E0101DD95FD0E926E0A0E85ECE5F0D2
:10F9A00092688F0E70ECF4F010080AE20A0E85ECF3
:10F9B000E5F08F0E70ECF4F0100802E20101DD8535
:10F9C0000601D9918850800B01E0D981D9938850E4
:10F9D000400B01E0D98369EC51F020860001126AE6
:10F9E000136A146A156A2D82800E086E176A229AAD
:10F9F000700EE66EE66A290EE66E010E30ECE5F05A
:10FA0000020E0A6E5A0EE66EA20EE66E000EE66E4C
:10FA1000030E30ECE5F0030E0A6E2A0EE66EE66A7F
:10FA2000000EE66E0A0E30ECE5F0AA0EE66E300E21
:10FA3000E66ED2ECF3F030ECE5F0FE0E7CECF4F088
:10FA4000810E005C01E053DC060EE66EF00E74ECF5
:10FA5000F3F030ECE5F0040EE66EA00EE66EF00E6C
:10FA6000E66E060E30ECE5F00601F051040801E206
:10FA7000F06BF251010801E2F26B200EE66E800E8F
:10FA8000E66E910EE66E070E30ECE5F0060EE66EC1
:10FA9000EA0EE66E350EE66E050E30ECE5F0830EEE
:10FAA0000A6EF90EBDECE5F000C086F20201865147
:10FAB000DA0802E2DA0E866FDF0EBDECE5F0010136
:10FAC000DD91720E005C01E1DD817E0E0A6E0F0E8B
:10FAD000E66EE66AED0EE66E020E30ECE5F00A6ABE
:10FAE000020EDB5011E09EEC09F0BB0ED8800F54E3
:10FAF000200E105402E2010178890F0EC2ECEEF0E4
:10FB000003E20101040E446F01017897E385530E6F
:10FB100065ECE9F0001C810B05E0BA0EC95C02E15E
:10FB2000010178870101E3950301DC69D1EC0DF057
:10FB300001018EBB3D9FFF0E0201FB5D02E11E0E27
:10FB4000FB6FFF0EFA5D03E1800EF96FFA6BFF0E9B
:10FB5000F25D02E0F25102E1640EF26F010138A79A
:10FB60003C9978A702D0050E5C6F0501355150080D
:10FB70000BE2280E386F38C535F5050E396F39C5DB
:10FB800036F53A6B3AC537F501018C510A0801E2A6
:10FB90008C6B180EE66EE1EC15F0E552000907E1FA
:10FBA0000301DA51010805E2040EDA5D02E2B5EC68
:10FBB000ECF0E9EC79F046EC0AF0C7ECEEF001016C
:10FBC000DD83B9ECEEF0010178A703D003010A0E42
:10FBD000E36FFAEC28F00401300EB76F010158AB67
:10FBE00003D00401310EB76F04013B0EBE6F050157
:10FBF000006B00C502F500C501F5800E056F070119
:10FC00000C0E346FDD0E356F320EB16F7D6A0C6AEB
:10FC1000E26B88ECE9F00701EF8102ECEDF0E4C261
:10FC2000E6FFE6ECE7F055EC24F0010138A70ED032
:10FC300056ECECF0E5C2E6FFE6ECE7F055EC24F01C
:10FC400002ECEDF001016385E4EC23F038EC25F0E3
:10FC50001A940101DF9F2BAD16D005EC27F00F5051
:10FC600010100EE00F0E0F5C270E105809E21A84D8
:10FC7000680E0F1808E1105006E10101DF8F03D074
:10FC8000600E9CECE5F01AB402D0010197950301D7
:10FC9000B00ED26F0A0ED36FAD0ED46F120ED56FA9
:10FCA000FE0ED66F070ED76F0101DFAF0DD0030137
:10FCB000540ED26F070ED36F910ED46F0F0ED56F07
:10FCC0003E0ED66F080ED76F54EC05F0268057EC29
:10FCD000E7F07FEC28F01880D0EC2CF07AD96AECB1
:10FCE00038F00201320E346F0101040EB36FA30E1F
:10FCF000B46FB3C10BF002016E2B320E326FE66AA5
:10FD000042EC90F0E55261ECC3F0BBECC3F079EC4F
:10FD1000B5F00301DA51010814E2040EDA5D11E2D4
:10FD20009BECE7F09F0EE66EF20EE66E010EE66EBD
:10FD3000B6ECE6F0030E0301DA5D03E10101330ED8
:10FD40001F6F030EE15C02E2E16AE552E16EFFEF34
:10FD5000E4F09A0E0B5C03E30B509D0801E2000CEB
:10FD6000010CE20E0B5C03E30B50E70801E2000C10
:10FD7000010C01013C7B3CBB04803DEC0AF001011D
:10FD8000289D076A120065ECEFF0D5ECF1F0010157
:10FD9000460E196F4C0E1A6F310E0A01D52501015E
:10FDA0001B6F96EC04F0DAECF0F00050EAECE8F0AF
:10FDB00004E14B5002E1CCECEEF09FEC04F0006E5D
:10FDC0003A50DF6EADECE9F001011F8F300E1D5D82
:10FDD00007E11EC11DF11FC11EF1300EDF241F6F90
:10FDE000E552FFEFE4F00A01D651E1EFF4F0FAEC4E
:10FDF000E4F0016A012A0A01D52BD551040801E279
:10FE0000D56BE2ECECF00DE0050E015C0AE2D1EC02
:10FE1000EEF004E0E846FE0BE706FCE10701E11521
:10FE2000E9E07CEC95F096EC5EF0B4ECEAF0FE0EC6
:10FE3000DB5002E0BEEC15F0E66AA7EC90F0E5526C
:10FE4000695002E0D5CAB1F2A8ECE6F01AE0D8ECAD
:10FE500009F0000916E16F5014E1695070ECF0F000
:10FE6000016E0150F6ECE5F00CE24A503808000E45
:10FE70004B5407E2720E15ECE9F0FA0E096EFE0E15
:10FE8000DB6AFE0EDB0403E17EDF640E096EFFEF2A
:10FE9000E4F00C50006E005003E0030E005C1BE128
:10FEA000005005E10101CB7DCBAD0ED007D081EC38
:10FEB000E7F006E00101CB75CBA506D0048004D0A5
:10FEC0000101CA75CAB504803DEC0AF0B3EC4BF0F1
:10FED000E5EC1CF016D0000403E0020E005C11E11A
:10FEE000BEEC15F0000402E1020E01D0010E006E1E
:10FEF000020E005C01E104803DEC0AF000500C6E43
:10FF000027D869EFECF001013C51080B03E0B4EC99
:10FF1000E5F002E0000E01D0010E1592E8B0158266
:10FF2000B4ECE5F004E101013D51800B0CE1B4ECCF
:10FF3000E5F007E017ECE6F004E101013C51800B2D
:10FF400002E1000E01D0010E1590E8B015801200FC
:10FF50000C50006E0050800802E2050E006E060E86
:10FF6000005C01E3006A000402E10101CA91020E93
:10FF7000005C02E10101CA8100500C6E258A21BE9D
:10FF80000CD046EC15F0A8ECE6F002E09CEC05F095
:10FF9000E5EC1CF04CEC05F002D0B3EC4BF0B4EF08
:10FFA0002CF065ECEFF0030EDF6E01018FBDDF6A10
:10FFB0004A514A6E4B6AB00E3E6E040E3F6EB0EC74
:10FFC000E5F03E50D880DF540201656FE552FFEF47
:10FFD000E4F065ECEFF027B012D0320EDF6E0101D5
:10FFE0008FAD02D0640EDF6E080E4A5D02E2080E8D
:10FFF0004A6FDF50D8804A5502E2DFCF4AF1D1DFA5
:020000040001F9
:10000000E552FFEFE4F065C2ABF123AE3AD0006AEF
:1000100001013E510C0803E3050E3E5D02E2090EAC
:100020003E6F050E3E5D4E6E4F6A0201655123EC38
:10003000E6F0140EDAECE5F03EC04AF04A50006EED
:1000400045ECF1F00101AB514C6E4D6AFF0ED880CA
:100050004C56000E4D564B504D18E8AE02D04D3464
:1000600004D04C504A5C4D504B580BE20050D880A5
:10007000AB5507E224A003D00050AB2702D00050BC
:10008000AB5F1850080B08E102013D510601F01169
:1000900006E02850400B03E11E9249EC50F012009C
:1000A000050E15EFE9F0FCDF268E1200180E27EC86
:1000B000E5F0268E1200FAECE4F0050EE12620A20F
:1000C0000FD0BAC1DFFF010EBBC1DBFF020EBCC106
:1000D000DBFF030EBDC1DBFF040EBEC1DBFF0ED094
:1000E000B5C1DFFF010EB6C1DBFF020EB7C1DBFFFA
:1000F000030EB8C1DBFF040EB9C1DBFF82ECE6F0F2
:100100001BE00101DFBD07D0DF50180815E21C0E0F
:10011000DF5C12E245D0190EDF5C42E01A0EDF5CB4
:1001200004E1010EDB505F083BE31B0EDF5C04E1E2
:10013000290E36ECE5F034E32C50100B14E1070ED9
:10014000DF5C0EE1010EDB50360803E282ECE6F0E4
:1001500027E1010EDB50400803E282ECE6F020E0EC
:10016000080EDF5C1DE02C50100B06E12F50800BB9
:1001700003E018ECE9F002E2F36A17D0790EE66EBC
:10018000020EE66E1AECEEF006ECE8F009E11AEC6D
:10019000EEF0740EE66E020EE66E06ECE8F004E099
:1001A00085DF010EF36E01D0F36AF46A050EE15C9F
:1001B00002E2E16AE552E16EFFEFE4F065C301F0AF
:1001C00023A802D075C301F00E0E015C01E2010C00
:1001D000100E015C01E2020C120E015C01E2030C44
:1001E000140E015C01E2040C160E015C01E2050C28
:1001F0001B0E015C01E2060C220E015C01E2070C01
:10020000080C35B603D0D4ECEFF017D0A70E27ECCE
:10021000F2F0016A006A0050D880015402E20150F5
:10022000006EDAECFDF0D5ECFDF00009FCE1C45005
:10023000016E0050D8800154EEE32CA802D000508B
:1002400010D00050020802E2020E005E460E005C72
:100250000BE2240E4A6EEE0E4B6E010E84ECF0F0B3
:10026000F5500F6E106A12000050020D8AEFE5F093
:10027000F00E8C16049035B804807DECE7F006E1B2
:100280002350100B03E0010E85ECE5F0BADF0FC040
:1002900061F310C062F335B81200F00E8C16030E35
:1002A0008C1214A637D0CFC101F023B885D9050E22
:1002B00001244A6E0A0ED8ECE6F03F50016E015060
:1002C00005E12350400B02E0010E016EB4ECE5F0B5
:1002D00003E03550400B05E001C0D5F702010A0EDE
:1002E00008D00701D551015C05E301C0D5F7020133
:1002F0000C0E3A6F63DF0701D66F2C50100B04E130
:1003000035EC0FF0000902E00701D66B89ECEAF04A
:10031000BEECE8F097ECE7F00480005009E03550BF
:10032000400B06E1030E005C04E1020E785C01E183
:100330000490070E016E3250010B03E10450010BD3
:1003400004E0CD0E66ECE7F0016E0F0E0114020121
:10035000886F32B002D0070E881701380F0B016E7C
:1003600004A0016A14A408D0020EE66E88C2E6FF5B
:100370000150E66EBEECE8F02CA80AD001014B510A
:100380000F6E106AE10ED8800F56000E105617D06F
:1003900033ECEFF00CE25E510F6E106A770ED880EE
:1003A0000F56010E10565DECEEF0FDE108D05351F2
:1003B0000F6E106A430ED8800F56010E1056006A59
:1003C0000301FF0ED8806155000E625501E2002A3C
:1003D000005061C34CF062C34DF005E0D8904D323F
:1003E0004C32E804FBE161C33EF062C33FF0E2EC53
:1003F000F1F0D8ECF2F0DDECF0F00FC043F010C0FB
:1004000044F0EDECEFF00050E85003E05DECEEF06E
:10041000FDE10FC0CFF1FA0E7DECE6F003E2010141
:10042000FA0ECF6F310E0101CF5D03E0330ECF5DC9
:1004300002E1320ECF6F630ECF5D03E0650ECF5D3C
:1004400002E1640ECF6F97ECE7F0040E005C23E14D
:10045000100E016E01504A6E4B6AE8C23EF0E9C2CE
:100460003FF0B0ECE5F03EC0EAF20101CF5193EC71
:10047000E7F00201E8274B50E923EA514A6E4B6A44
:10048000E8514A5CE9514B5806E2EA5193ECE7F037
:10049000E85F4B50E95B000406E0020E005C03E0FD
:1004A000030E005C08E10201EB510101D880CF5539
:1004B00002E2CFC1EBF27DECE7F006E12350100B36
:1004C00003E0010E85ECE5F09CDE0FC063F310C085
:1004D00064F3F00E8C1603016C0ED8806355000E89
:1004E000645517E282ECE6F014E0980EE66EF20E28
:1004F000E66E010EC3ECEDF00201640E2D6FC7EC49
:10050000EDF003E054ECF2F0FDE1D9ECEBF0E7ECB8
:100510000BF003016151635D6251645906E3010E02
:100520006325616F000E6421626F61516325676FFF
:1005300062516421686F675167254A6E685168216E
:100540004B6E67C34CF068C34DF0030E0FECEFF039
:10055000E804FCE14A504C240301676F4B504D20E6
:10056000686F6351615D4A6E625164554B6EC5ECB4
:10057000EFF067C33EF068C33FF078ECFDF03EC09B
:1005800067F33FC068F367C365F367C34AF068C3A6
:100590004BF04C6A4D6A4D34000E4D1809E6D88078
:1005A000FF0E4A54000E4B54000E4C54000E4D5496
:1005B00002E203016569120049C101F02C50100BE1
:1005C0000BE133ECEFF008E26C0E015C016E0A0EF9
:1005D0002C5D02E1040E015E1200F6ECF0F007E083
:1005E0003550400B04E1050E005C01E0000C010CED
:1005F0000482F3DF000901E00492358604A23596F7
:10060000359836DE35B8120097ECE7F0049A049876
:100610000496030E005C01E10486000403E0020E70
:10062000005C01E104882350400B01E109D1235013
:10063000100B01E005D13450080B01E101D102019A
:100640002D5101E0FDD01A50010B01E1F9D00482D7
:100650000494C3DF000901E00492040E005C01E190
:100660000484AADF0150FC0BE842E842026E32A08B
:100670001CD00201885107080AE20150E840E84016
:10068000E8401F0B015C525D09E2522B07D0445138
:1006900005E1525103E05207040E446F5251D880D5
:1006A000015405E25251015E02D00201526B0490E6
:1006B0000450040B03E00250EA5D07E30450040B0E
:1006C00070E101500101CF5D6CE20101320E076F54
:1006D0000A0E2C5D02E1040E07270201BA51105DDB
:1006E00002E3000E01D0010E049CE8B0048C480E19
:1006F0000F5D710E105901E394D003016C0E635D20
:10070000000E645901E38DD082ECE6F00CE021503C
:10071000800B05E06C0E01010725495D04E00450E3
:10072000400B01E17ED004B20BD00101CF51015C3E
:10073000020D8AECE5F00F5002010F27105005D092
:1007400004A405D002010F2B000E102369D0020172
:100750002E5167E10A0E2E6F0150EB5D20E2EB5146
:100760001EE004A802D0020E2E6F0450080B12E007
:10077000030E785C06E0020E785C03E08851010805
:1007800009E2320E0F27000E10232F5107E02E91A1
:100790002E4304D00A0E0F27000E10230480EB6BAB
:1007A00040D00450040B05E002500201D880EA5505
:1007B00008E30450040B35E101500101D880CF5506
:1007C00030E2020E036E04A402D0010E07D004A290
:1007D00006D0320E036E04A802D0960E036E0350AC
:1007E0000F6E106A0450020B06E00450080B0EE076
:1007F00002012F510BE001500101CF5D4A6E4B6A9F
:10080000C5ECEFF019ECF4F0DFECF2F002010F515F
:100810000F5C1051105805E20F500F5F1050105B25
:10082000048004A00DD0020111510F1902E11251F0
:10083000101906E0E7EC0BF00FC211F210C212F231
:100840000201305102E00F0E306F12001750100BF2
:100850000CE03A0E675C3EE0170E675C3BE02A0E48
:10086000675C03E10BECEFF035E01750010B06E09D
:10087000190E675C2FE02D0E675C2CE0350E675C6F
:1008800029E0250E675C26E00E0E675C23E0080E6B
:10089000675C20E0390E675C1DE0380E675C1AE08B
:1008A000400E671417E18FECB5F0000913E1090E53
:1008B000675C07E11750100B04E0D8EC1DF000094D
:1008C00009E12150800B05E16F5003E03350200B0C
:1008D00001E0000C010C020E06ECECF0909C460EC0
:1008E0005CECE7F0908E010EE66E8EECFDF0E552CA
:1008F000FDEC1DF017ECE6F003E0720E12ECE5F0F3
:10090000F7EC18F006015091120071C249F172C261
:100910000FF273C210F2E7EC0BF07FEF28F0010149
:10092000AB5103E12C82A7C108F02150010B12E06A
:10093000B4ECE5F00FE11750800B03E06DECECF048
:1009400006E02150040B06E18150010B03E097D92A
:1009500067EC8CF012000101050EAA6F2150010B0B
:1009600005E01A50020B02E0AA6B120034BE13D04D
:100970005CC100F00A0E2C5D05E17851080B02E124
:100980000A0E002602010E51D880005404E20E51D6
:10099000005C0101AA6F1200E7ECF1F00101DF99A0
:1009A000A8ECE6F002E00101DF892550020B04E12A
:1009B0001D50010B01E0238C23BC06D0E66AE66AD9
:1009C000C80E2BECE5F010D00BECEFF00BE134503F
:1009D000080B08E0C7ECEDF003E054ECF2F0FDE1A9
:1009E000D9ECEBF0E7EC0BF002010A0E2E6FEB6B8B
:1009F00021AE1D84C80E2F6FF0EC18F0780E006E3B
:100A000000505CECE7F090EC1DF00201326BB4ECAE
:100A1000E5F003E03550400B07E082EC0BF00009F5
:100A200003E00D0E73ECE7F02150800B06E117ECAC
:100A3000E6F003E0730E12ECE5F0909E349E23EC9A
:100A4000EBF001E0348E06ECF4F03EE12C50080BA4
:100A500030E02350100B2DE101013B052AE016C2C6
:100A6000DFFF41ECC6F0DF500201165D22E0010E0F
:100A700069C3DBFF020E6AC3DBFF030E6BC3DBFF40
:100A8000010EE66EEBECC6F0E552010EDB50030101
:100A9000695D08E1020EDB506A5D04E1030EDB5084
:100AA0006B5D07E0ACECC5F096EC5EF01D82960E37
:100AB000096E3450800B08E01BECEBF005E106EC0E
:100AC000F4F002E12AEC0BF02150800B19E12150E7
:100AD000010B16E1B4ECE5F009E03550400B06E1FE
:100AE00002013D510DE0050100510AE10101DF9BCA
:100AF0001BECEBF003E00101DF8B02D062ECE9F0CC
:100B00001EAC02D0EEEC0BF0218C328234AE02D05F
:100B1000909E6ED0D5CAB0F297ECE7F0360E026E1A
:100B2000380E036E005003E03550400B03E04FC118
:100B3000D5FA12D0A1EC0BF0000904E085C1D5FA7A
:100B400003680AD0050E005C05E10A01D56B036855
:100B5000026802D056C1D5FA0A01D551CEECEDF0AB
:100B6000016E0250015C04E30350D880015403E29B
:100B7000750E9CECE5F0B2EC5DF00101DFB91AD026
:100B8000B5C193F2E6ECF2F03FC094F2F1EC38F02C
:100B9000B5C191F2E6ECF2F03FC092F220A20AD089
:100BA000BAC191F2A1ECE5F0BBC13FF0BCECFDF0A5
:100BB0003FC092F2909E0101DFB91AD020A203D06B
:100BC0000701576B586B02019351915D0EE19451EF
:100BD000925D0AE07DECE7F008E102019429925D64
:100BE00003E09405925D01E12A84308ECFEC3EF063
:100BF000320E5CECE7F0908C9BEC0FF007011B9938
:100C00001B9701013CA904D007011C6B1CC71BF7F3
:100C1000B3ECEBF00201FA0E336F248A2682329293
:100C200023AC02D00601508140EC4BF00201295167
:100C300009E00101DF51080B05E1140E69ECE5F054
:100C40000101DF87040EE15C02E2E16AE552E16E38
:100C5000FFEFE4F065ECEFF0050111071251EA6ACD
:100C6000150FE96E050EEA22EFCFDFFF122B1251AE
:100C70001F0801E2126BDF50E552FFEFE4F052EC87
:100C800029F002012A6B2AC26AF21DECECF007E09F
:100C9000200E01011F5D03E0200E69ECE6F001016A
:100CA000AB6B006A36EF91F065ECEFF00850DF6E49
:100CB00002011E0E316F0501005102012A110BE0E5
:100CC0001E50040B06E01E50080B03E08150080B79
:100CD00002E1D5DF76D308503AE1345101E071D317
:100CE0000101E99521B002D057DE0ED0B4ECE5F059
:100CF00006E002013D5108E00501005105E11BEC51
:100D0000EBF002E162ECE9F00BECEFF014E1020130
:100D1000B4A50FD0330EB25D09E10101DEAF0BD0F7
:100D200002EC05F00201330E4D6F05D002EC05F028
:100D300002D007EC05F00101DFA902D0AA6B37D180
:100D40000ADE050E01018703F350AA2730D10804FB
:100D500030E10101AA5101E030D3209C06ECF4F00F
:100D600002E0208C0FD03450800B0CE11BECEBF038
:100D700009E12AEC0BF00101DFAB02D062ECE9F0F3
:100D80000101DF9B2E50200B03E12050020B04E0F9
:100D9000E4C2E6FF92ECE9F00101280EAA6F23A855
:100DA00002D0AA9FAA4721AE02D0050EAB6F082A37
:100DB0000AD0020E085C09E10101AA5102E1F8EC37
:100DC00082F034EC0BF0ABDDF8D2030E085C42E1AC
:100DD0002CA226D05CC1AAF17DECE7F005E17851A8
:100DE000080B02E10A0EAA27DFB9AA6BAB5104E097
:100DF000050E8703F350AA272C922150010B04E023
:100E00001A50020B01E0AA6BB4ECE5F006E0020117
:100E10003D5103E13550400B03E0006A36EC91F0A0
:100E20000101AA5106E0B4ECE5F00FE03550400BAB
:100E30000CE12050400B05E102013D5102E12FEC95
:100E40000BF00101280EAA6F40D127B8B6D2F8ECFA
:100E500082F0B3D2050E085C68E10101AA5101E0FD
:100E6000ACD2082A279821B059D01C0E016EDFA9F8
:100E700002D0140E016E8751E8240124006E020195
:100E80008C5107E000508C5D04E2090E086E278843
:100E900045D03282909C219C34BE10D0B0C2D5FA8D
:100EA000B2EC5DF00101DFB909D0F1EC38F020A21D
:100EB00003D00701576B586BCFEC3EF007011D992B
:100EC0000101E3A102D007011D8907011D9701015E
:100ED000E3B102D007011D8707011B990101E3A3BC
:100EE00002D007011B8907011B970101E3B302D060
:100EF00007011B8701013CA905D0B1C2E6FF94ECB4
:100F00005DF0E552B3ECEBF0B4ECE5F003E0355006
:100F1000400B03E00101050EAA6F32920101DFA927
:100F200002D0AA6B4AD217DD48D2060E085C41E116
:100F30000101AA5101E041D221B037D02750100B56
:100F400019E13C51080B12E1335110E0E951040B57
:100F50000DE1B4ECE5F003E03550400B07E0010192
:100F60003D51800B03E0E951800B04E00101E99F52
:100F7000B2DC11D033C132F227A80DD0EEECF4F080
:100F800087C13FF0FAECF0F0006E00500201325DD4
:100F900002E200C032F22E50200B03E12050020B7F
:100FA00004E0E4C2E6FF92ECE9F002016B6B082A70
:100FB00004D2070E085C2EE10101AB5119E117AE16
:100FC00015D06DECECF003E055ECB6F00FD0B2ECC0
:100FD0000BF0000904E10101E951040B07E0100ED8
:100FE000675C03E10101E98101D0179EA7C108F008
:100FF00002013D5101E0E1D13A5106E03550400B8C
:1010000003E189ECEAF003D0E66AE66AE66AA1EC5D
:1010100030F037D0080E085C4AE10101AB5106E020
:101020001E50040B03E01E50080B02E1A7C108F09C
:1010300002013D5101E1C1D1F8EC82F034EC0BF03A
:1010400002013E5101E0B9D18AEC0FF0000901E143
:10105000B4D10501020E146F115115E0FBDD006ED5
:10106000020E785C18E0016A0501115102E0F2DD20
:10107000016E0050E66E0150E66EE70EE66E56EC2D
:1010800018F0E5520ED000510FE1006A020E785CB4
:1010900002E1030E006E0050E66EE60EE66E52ECC4
:1010A00018F0E552E55289D102013D6B86D1090E57
:1010B000085C2BE10101AC417F0BAC25D880AC551D
:1010C00006E202018C6B8CC2ACF1050E75D181B6C3
:1010D00074D1010EAC6F320EAA6FDFA902D0280EB8
:1010E000AA6F010E086EB4ECE5F006E002013D5176
:1010F00003E13550400B05E01BECEBF002E162EC44
:10110000E9F001010B0EA76F58D10A0E085C06E149
:1011100022BA9ED0179E0B0E086E9CD00B0E085C58
:1011200001E09BD01750800B3CE12150010B06E001
:101130002150040B03E18150010B33E1B4ECE5F0E5
:1011400003E03550400B0CE02150800B09E1815049
:10115000080B06E01E50040B03E01E50080B21E1B3
:10116000B4ECE5F00CE03550400B09E12150040BE4
:1011700006E18150010B03E0E6ECECF012E02150B7
:10118000800B0CE08150080B0CE01E50040B09E0B2
:101190001E50080B06E08150010B03E006ECF4F052
:1011A0004DE017AE18D06DECECF005E055ECB6F064
:1011B000000911E106D1B2EC0BF0000904E10101D4
:1011C000E951040B08E0100E675C03E10101E981BD
:1011D00002D0179EF6D0B4ECE5F014E03550400B89
:1011E00011E117ECE6F00EE11AAA04D0A4EC0AF023
:1011F000DCEC22F00101895105E089C1E6FF35EC04
:1012000029F0E552ACC18CF20101AC5102E0010EB3
:10121000AC6F27A802D0F8EC82F00701D36B030E65
:10122000086E0101800EA76F2150800B03E117505B
:10123000800B08E021940C0EA76F04D023A802D0E5
:10124000A5ECC7F00101AA5105E12750100B02E1FE
:10125000F8EC82F034EC0BF0B0D00C0E085C01E03E
:10126000ACD022BAAAD0DEECB8F021AEA4D01E5089
:10127000040BFDE01E50080BFAE08150080BF7E06C
:101280002B84189A248A18982682010199510CE01F
:1012900020A203D099C17DFF02D099C10CF0F1ECDE
:1012A00038F0198CA8EC7FF023A803D085EC84F0EB
:1012B0006ED0320E026E7DECE7F002E1040E0226E3
:1012C000140E0301655D5EE22C50100B04E0640E09
:1012D0000101495D0BE02C50100B54E1320E01016D
:1012E000495D04E06C0E0224495D4CE121EC15F0EF
:1012F00010C200F000504C6E4D6A00501BECE6F03E
:1013000049C100F082ECE6F004E06C0E0101495D99
:10131000006E45ECF1F0C5ECEFF0C0ECE5F0000E2E
:101320007DECE6F02CE27D0E37ECEFF028E20F507A
:1013300000ECE9F082ECE6F025E00201710EBA6FF4
:10134000030E5CECF0F0BAC23FF0FAECF0F0006E85
:1013500000500201D880105504E3030E1003F3CFB0
:10136000BAF2100E01012C03F350056E680E0A6EDE
:1013700084ECEDF0055056ECF0F00A6A03D0780EDC
:101380009CECE5F019A803D085EC84F01998219E17
:10139000A8ECE6F003E0B3EC4BF005D0010EE66EEE
:1013A00060EC4BF0E5522398A1ECE9F0010137BF66
:1013B00002D0B6ECEEF0800E086EDF50085C01E063
:1013C0001D8CE552FFEFE4F03050100B0CE10701EB
:1013D000825109E149ECEFF007E0020E6F5C04E096
:1013E0000201DF5101E1000C010C070EE66EE66A16
:1013F000200EE66E440EE66E060EDFEFEBF045C6FD
:1014000044F646C645F647C646F648C647F649C6B8
:1014100048F64AC649F6120049C64AF648C649F691
:1014200047C648F646C647F645C646F644C645F69C
:101430000601200E446F1200FAECE4F00101E551C0
:10144000E61103E00D0EF8ECE7F0E751E81103E0D8
:101450000A0EF8ECE7F032AA02D005ECF0F0010138
:10146000DF51020B0CE0280E0901BD5D08E2BD5101
:10147000BD2BEA6A950FE96E090E2DECF3F0FFEF34
:10148000E4F0DAECF1F01B50010B0AE0800E6EEC98
:10149000E5F004E2FE0EDB50200802E11B905CD078
:1014A000AEDFFE0EDBCF4AF6DB50800804E0850E8F
:1014B0006EECE5F003E30601200E21D0FE0EDB50BA
:1014C000300803E10601630E1AD02A50200B1CE0FD
:1014D0002950080B19E1DF6A150EDF5C15E2B8EC44
:1014E000F2F00FE1DE52010EDD6EDF2A0DECE8F0C6
:1014F00006014A6F84DFDF2A0DECE8F006014A6F2F
:1015000003D0030EDF26E8D7020E6F5C12E0010E57
:10151000DB5004E049C6E6FF8FDFE5524AC600F023
:10152000630E005C02E1300E006E0050E66E84DF58
:10153000E5524ADF000910E09BECE7F044C619F1E0
:1015400045C61AF146C61BF147C61CF148C61DF137
:1015500049C61EF14AC61FF1020EE15C02E2E16AD1
:10156000E552E16EFFEFE4F065ECEFF00850DF6E5E
:101570002492100E085C13E11C0E086E02016651E5
:10158000010B03E11E50040B02E1110E92D06651D3
:10159000040B29E11E50080B01E0ABD024D0110E42
:1015A000085C0AE12480238E0201080E666F248203
:1015B000086A0101120E9CD0120E085C07E124900B
:1015C0002482030E086E0101130E92D0130E085CE4
:1015D0000CE11C0E086E02016651040B04E11E5062
:1015E000080B01E086D0140E64D0140E085C11E1E3
:1015F0002480238E180E086E1E50040B01E079D053
:101600001E50080B01E075D02482086A0101150EF6
:101610006FD0150E085C0BE101012BAF03D0020166
:10162000020E666F239E5AECECF0160E61D0160E79
:10163000085C04E15AECECF0170E5AD0180E085C66
:1016400008E10201020E666F2482086A0101190E88
:101650004FD0190E085C05E1239E5AECECF01A0EEF
:1016600047D01A0E085C04E15AECECF01B0E40D097
:10167000170E085C08E101012BBF03D00201020E26
:10168000666F1B0E16D01B0E085C05E12490238E9E
:101690002482030E2AD01C0E085C2BE12490800EBD
:1016A000086E02016651010B03E11E50040B03E1B9
:1016B000110E086E1ED035AC03D0ADECF4F019D08D
:1016C0001750800B16E11850080B03E0090E685DF7
:1016D0000AE30601F05104E0080E0201685D03E32D
:1016E00002013D5106E02482080E086E0101100E31
:1016F000A76F24A202D003EC80F0DF50085C01E069
:101700001D8CE552FFEFE4F070ECEFF001013CB905
:1017100002D01D9601D01D761D50080B01E0010E70
:10172000696E5751400B18E0D8EC09F0050814E039
:101730000201325111E133510FE134510DE1800EBC
:1017400008140AE02D50080B07E11E50400B04E17D
:101750002550010B01E102D878EFEFF0BEECF1F07B
:10176000D4C7DFFF020EDB6A35A003D0010E64ECA4
:10177000E6F0010E79C1DBFF1DA615D0020EDB6A73
:101780001DA803D0010E64ECE6F001018BBD0BD067
:10179000010E7AC1DBFF8D0E66ECE7F0006E04EC03
:1017A00034F00050DF6ED9ECEAF003E2010E05C719
:1017B000DBFF010EDB50DF5C0EE3020EDB5003E0CB
:1017C0004E0E12ECE5F0020EDB6A0201FA0E336FE8
:1017D00028A80CD009D0020EDB5002E122EC09F05F
:1017E000010E64ECE6F002010A0E336F1DA606D06E
:1017F0001D98020EDB5007E01D8805D03590020EC3
:10180000DB5001E03580030EE15C02E2E16AE55263
:10181000E16EFFEFE4F002016B6BE66AE66AE66AEE
:10182000BEECE8F002013A6B0701D56BD5C7CFF1EA
:1018300021B003D02180CCEC84F0120065ECEFF0F5
:101840000201050E3D6F280E3E6FE5DF020E785C4B
:1018500008E1DF6A010197A102D0060EDF6E92EC6B
:10186000F1F00501040E146FE552FFEFE4F0358C42
:10187000210ED1EFF0F00101DD51020B13E03D51DB
:10188000800B10E12150010B0DE12150100B0AE1FA
:101890002550020B07E1DD933088190E27ECE5F0A7
:1018A000AA0E096E120001013D51800B04E1215086
:1018B000010B01E1000C010C01015751800B05E007
:1018C000020E005C03E0000401E0000C010C65EC7A
:1018D000EFF062EC11F0000909E0030EDF6E010188
:1018E00097A102D0070EDF6E92ECF1F002013251A7
:1018F00002E0010E326F198C0701D36B2190219405
:10190000A7ECE9F0E552FFEFE4F081B003D01B0E45
:1019100027EFE5F081B603D01A0E27ECE5F01200B0
:10192000085039ECECF030E14B502EE11A920101F5
:10193000DFA503D0DF9520EC1EF00101DF51080B7D
:1019400008E02150400B05E1120E69ECE5F00101C1
:10195000DF9735AC02D0ADECF4F021B00BD062ECE7
:1019600011F0000903E0006A36EC91F022966F5006
:1019700001E1208622AE06D0010EE66EEAEC0AF006
:10198000E552229E082A12000850A5ECEAF001E078
:10199000CAD14B5001E0C7D121A0239C1AEC16F00C
:1019A000FF0801E0F4D02E50400B01E0F0D02150B0
:1019B000200B01E1ECD01950800B01E0E8D0285059
:1019C000010B01E0E4D00101E951010B01E0DFD09E
:1019D00002018C6B8CC2ACF11A9297ECE7F0359C4B
:1019E0001D908150080B18E1005006E02050020BBA
:1019F00013E162DF000910E00101010EAC6F1A82F1
:101A0000086A0B0EA76F005003E14DDF000901E0EB
:101A10001D80005033E134D01E50040B03E01E50F3
:101A2000080B30E1005013E02050020B03E144DFCB
:101A300000090DE10601F25125E062EC11F0000908
:101A400006E12050020B1EE117ECE6F01BE01EB48D
:101A500002D0110E05D01EB604D00201666B140E22
:101A6000086E005003E11FDF000901E01D800050F7
:101A700007E0030E0C5C02E1E1DE89D0F8DE87D0DE
:101A8000FADE85D0050100511CE0005003E017ECA0
:101A9000E6F010E0005003E106DF000901E01D80E0
:101AA000005001E1E8DE17ECE6F001E0C7DE1E0EB3
:101AB000086E6DD0268E810E15ECE9F04AEC29F007
:101AC00066D021AE04D0086A01010A0E47D000504A
:101AD00048E08150010B06E02150040B03E1E6ECE5
:101AE000ECF03FE002012A5114E0E6ECECF007E1F3
:101AF00028EC09F000090DE18150010B0AE1020117
:101B00004A6B4B6B2A6B2AC26AF2A4EC0AF050ECC7
:101B100080F006ECF4F007E08150010BFDE0E6EC0C
:101B2000ECF0FAE130D01850080B0FE01A50400BDF
:101B30000CE0800EE66E030EE66E990E2BECE5F0DF
:101B4000B2EC0AF09E0E52ECE7F002013A6B3AC298
:101B5000D5F73AC2CFF1086A01010B0EA76F1D80BD
:101B600016D0005014E12150010B11E18150010BFE
:101B700003E02150040B0BE00101DD9306ECF4F0CF
:101B800004E081A0FED7219412001D8044DE215084
:101B9000200B04E1C3EC0BF0000907E102014751FF
:101BA00004E10101E951010B27E00501006B2190DF
:101BB0002194810E086E0101E951010B02E06F5082
:101BC00007E1A3DEC3EC0BF0000902E009C047F215
:101BD00021EC08F00101E9A10FD0B2EC0BF00009F3
:101BE00007E10101E9910201476B010E096E04D082
:101BF00021AC02D0A7ECE9F00850A5ECEAF001E135
:101C00004B502FE090EC97F002013A6B30AA02D0D3
:101C1000D6EC69F031A402D099EC6CF031AC02D072
:101C20002FEC6BF025A002D04CEC6AF033A002D070
:101C300091EC6AF024AE02D0DFEC68F020A802D06C
:101C4000A1EC12F02D50800B03E12D50400B02E06F
:101C500095EC0FF0269A1BAC02D03AEC0AF01D8CE2
:101C600012002150010B18E002013D5115E11750FF
:101C7000800B06E06DECECF009E0250E675C06E0F9
:101C80002150040B09E18150010B06E015A002D0A0
:101C90000101E98F67EF8CF002013A5104E089EC11
:101CA000EAF0BEECE8F017AE6ED055ECB6F05BECA7
:101CB000E8F017E03050200B14E13150040B11E133
:101CC0002450800B0EE13150400B0BE12550010BED
:101CD00008E13350010B05E13350020B02E16AECDD
:101CE00038F0339220AA4FD0209A01013CAB4BD060
:101CF0009BECE7F0020142510FE1BEEC43F00D0E08
:101D0000675C10E11750010B0DE00C507D5C0AE19F
:101D10000201C80E426F1200426B1C0EE5ECE8F0A7
:101D2000960E096E1200D4ECEBF02DE14B502BE136
:101D30002250200B28E10101E151800B24E109EC44
:101D400008F0000912E165ECF1F00AEC33F00D0E39
:101D500012ECE5F00C5002E03C0E01D01E0EECEC53
:101D6000F2F00101E29B4CEC05F053EC0EF0248AFA
:101D700002011783810E086E09EC08F0000903E0E8
:101D80006AEC38F0268212000D04040F0701006F80
:101D900004A002D0040E00271200189A1AAC11D029
:101DA000A4EC0AF014820201DC0E4A6F050E4B6FA0
:101DB0000101DFAF14D00201E80E4A6F030E4B6F32
:101DC00012000490010139B10480DEDF0701FA0E30
:101DD000036F016B026B0201686B696B1E9012004E
:101DE00000C70AF002016A5104E0800ED6ECEEF062
:101DF0001B800701035117E003510307BDECE5F019
:101E0000CC0E005C10E0FF0E005C0DE0800E005C6C
:101E100006E20050E66E67EC04F0E552006E0050FA
:101E2000D6ECEEF0E6D70A6A12002AECF4F0DBCF2B
:101E30006AF23088006A24885AEC2EF0320E096E5D
:101E400019AA02D002016A8F02012A5102E0010E92
:101E50002A6F179EFFEFE4F069ECEFF019AA02D0A9
